:020000020000FC
:040000000C94820BCF
:100004000C9400000C9400000C9400000C9400006C
:100014000C94760C0C94A40C0C94D20C0C94000D3F
:100024000C94120D0C94190D0C9400000C94000007
:100034000C9400000C9400000C9400000C9400003C
:100044000C94980F0C9400000C9400000C94000085
:100054000C94A40F0C9400000C9400000C94000069
:100064000C941E130C9400000C9400000C940000DB
:100074000C9400000C9400000C9400000C94BC0E32
:100084000C9400000C9400000C9400000C94BC141C
:100094000C9400000C9400000C9400000C940000DC
:1000A4000C9400000C94F50E0C9400000C940000C9
:1000B4000C9400000C9400000C9400000C940000BC
:1000C4000C9400000C9400000C94A9160C940000ED
:1000D4000C9400000C941D180C9400000C94000067
:1000E4001027E80364000A0001000010000110005A
:1000F40001004D6F6E746167004D6F6E646179002D
:100104004469656E737461670054756573646179DD
:10011400004D697474776F6368005765646E657326
:1001240064617900446F6E6E657273746167005424
:1001340068757273646179004672656974616700F9
:100144004672696461790053616D73746167005329
:100154006174757264617900536F6E6E74616700C7
:1001640053756E646179000020427269646765208A
:10017400626F61726420666F756E64002072756EC2
:100184006E696E6720626F61726420686172647761
:1001940061726520746573742E2E2E2E00444332D2
:1001A400632E30342E30392031352E30332E323018
:1001B4003233004443322053577665723A20004468
:1001C4004332635F6F63743230323200444332200F
:1001D40048577665723A2000504F32655F6E6F76ED
:1001E4003230323200504F322048577665723A200E
:1001F4000052616D204572726F720052616D204F22
:100204004B0020204443322074696D653A2000205D
:100214002044433220646174653A20005254432FD1
:10022400545749206572726F72002020696E742ED3
:1002340020656570726F6D206572726F7200202088
:10024400696E742E20656570726F6D204F4B00448B
:1002540043322055494420696E206865783A20006D
:100264004443322055494420696E206465633A2032
:1002740000766F6C74616765206572726F7200201E
:10028400496E70757420766F6C74616765205B6D60
:10029400565D3A200054656D7065726174757265BF
:1002A400206572726F72002054656D70657261749E
:1002B400757265205BB0435D3A2000202064696755
:1002C4006974616C2074657374206572726F723A1C
:1002D400200020206469676974616C2074657374FC
:1002E400204F4B005254432D436C6F636B20657257
:1002F400726F72005254432D545749206572726FC5
:10030400720052544320697320776F726B696E6771
:10031400006F766572616C6C2073756363657373CB
:10032400006F766572616C6C206661696C757265CC
:10033400006578742E20656570726F6D2065727229
:100344006F72006578742E20656570726F6D20334E
:1003540032206B42204F4B006578742E2065657007
:10036400726F6D203634206B42204F4B00657874D9
:100374002E20656570726F6D2039366B42204F4BAD
:10038400203F3F3F006578742E20656570726F6D65
:1003940020313230206B42204F4B0000676F7420B5
:1003A4006D6462204E414B006D646220726573700F
:1003B400206572726F720072657065617420737467
:1003C4006F70006D6462206F6666006D6462206FFA
:1003D4006E006D646220737461727420706F6C6C53
:1003E400696E67006D64622073746F7020706F6C47
:1003F4006C696E67006D646220726570656174007B
:10040400656D70206F666600454D5020636F756E94
:100414007472793A2000454D50207363616C653ADB
:100424002000454D5020646563696D616C733A200A
:1004340000656D702070617920737461727420009E
:10044400656D70207061792073746F702000656D24
:100454007020676F742068436F696E2000656D704B
:1004640020676F7420636F696E2000656D70207261
:100474006420657272002D64796E5072302D002DE7
:1004840064796E5072312D002D64796E5072322D64
:10049400002D64796E5072332D002D64796E507284
:1004A400342D002D64796E5072352D002D64796ED3
:1004B4005072362D002D64796E5072372D002D2D1B
:1004C4002D2041544220476D6248202D2D2D002DB2
:1004D4002D2D205053412031323536202D2D2D0025
:1004E4002D2D2054657374205072696E74202D2D47
:1004F400004C4F474F3A0051523A00426172436FE9
:10050400646520322F353A0031323334353637388A
:10051400393031323334353637383930002D2D2DDA
:100524002D2D2D2D2D2D2D2D2D2D2D2D2D2D2D2DF7
:100534002D2D2D00202020202074686973206973DC
:1005440020612074696E792074657874006E6F720E
:100554006D616C20746578740074686973206973C4
:1005640020612068696768207465787400202042DF
:100574006F6C6420546578742000756E6465726CC9
:10058400696E656420746578740020696E7665729E
:10059400732074657874007072696E746572207467
:1005A400656D706C61746520002D2D2D20656E6461
:1005B400206F662066696C65202D2D2D00444F57F1
:1005C400206E6F7420736574007468697320697396
:1005D400206120322F35626172636F6465003C20B4
:1005E400536C61766520526573706F6E7365004459
:1005F4004332635F6F63743230323200504F32657E
:100604005F6E6F763230323200444332632E3034C0
:100614002E30392031352E30332E32303233000033
:100624007468697320697320616E204154422061AB
:1006340063636573732063617264000044436D6196
:100644006B655265736574002D00776F6B656E2062
:100654006279206D646200776F6B656E2062792029
:10066400636F696E00776F6B656E206279207074BA
:10067400750074726967676572696E672068656181
:100684007274626561742E2E2E00706F776572200D
:10069400646F776E006C696768742077616B6500BE
:1006A40066756C6C2077616B650073746172746934
:1006B4006E6720626F6F746C6F616465722E2E2E8C
:1006C4000000746573742063616E63656C6C6564AB
:1006D400007374617274696E6720436F696E436856
:1006E40065636B657220746573742E2E2E007769B2
:1006F4006C6C2062652073746F7070656420616631
:100704007465722032307320776974686F75742051
:10071400636F696E00496E7365727420636F696EEE
:100724007320706C656173653A00656D7020696E45
:100734002069646C6520737461746500656D702054
:1007440073746F7000656D702077616974696E678A
:1007540020666F7220636F696E7300207E3E207680
:10076400616C75653D00636F696E207465737420F8
:10077400656E640072756E6E696E67207374617263
:100784007475702074657374732E2E2E0052616D0F
:10079400204F4B0052616D206572726F7220666F3C
:1007A400756E6400426F617264206877204F4B005D
:1007B400426F617264206877206572726F722000E4
:1007C400527463206572726F722000527463206FDA
:1007D4006B00556964206572726F722000556964FC
:1007E400206F6B00557070657220646F6F722069A2
:1007F40073206F70656E005661756C7420646F6F42
:1008040072206973206F70656E0042617474657242
:100814007920646F6F72206973206F70656E004475
:100824006F6F7273206F6B0054656D7065726174C5
:10083400757265206572726F72200054656D706503
:10084400726174757265206F6B00566F6C746167AA
:1008540065206572726F722000566F6C74616765F3
:10086400206F6B00496E746565206572726F72202B
:1008740000496E746565206F6B004578746565206A
:100884006572726F7220004578746565206F6B0025
:10089400436F696E20657363726F77206572726F40
:1008A400722000436F696E20657363726F77206FE7
:1008B4006B005072696E746572206572726F72207B
:1008C400002020206E6F207061706572002020204F
:1008D4006E6F74207265616479002020206E6F2031
:1008E400726573706F6E736500202020696E746585
:1008F400726E616C206572726F72002020206865D0
:100904006164206F70656E005072696E7465722048
:100914006F6B002020206C6F77207061706572000F
:100924004E6F20636F696E207361666500436F6963
:100934006E2073616665206F6B004E6F2062696C78
:100944006C20626F780042696C6C20626F78206F53
:100954006B004D6462206572726F72004D64622098
:100964006F6B004D6966526561646572206F6B0040
:100974004D6966526561646572206572726F72209A
:1009840000436865636B696E67206D6F64656D2CE9
:1009940020706C7320776169742E2E2E00436F696A
:1009A4006E20636865636B6572206F6B00436F69CB
:1009B4006E2063686B206572726F722000466F75DB
:1009C4006E64204552524F52287329005379737430
:1009D400656D206F6B00444332632E30342E303902
:1009E4002031352E30332E3230323300444332201E
:1009F40053577665723A2000444332635F6F6374E1
:100A040032303232004443322048577665723A20FD
:100A140000504F32655F6E6F763230323200504F85
:100A2400322048577665723A20004D6F64656D2018
:100A34006F6B0072656769737465726564005369EE
:100A4400676E616C20004D6F64656D206572726F16
:100A540072200077726F6E67207479706500534955
:100A64004D206E6F742072656164790074657374CF
:100A7400696E67207072696E7465722E2E2E000086
:100A840041542B4353510041542B435245473F009B
:100A940041542B434C54533D3F002B4353513A2074
:100AA400002B435245473A20004154004F4B00610C
:100AB400742B6970723D3131353230300041544508
:100AC400300041542B434C54533D310041544900B0
:100AD40053494D37303030470041542B4353494D2F
:100AE4003D3F000006046F04DF045705D7055E068A
:100AF400EC0682072008C5087109250AE10AA40B3F
:100B04006E0C400D170EE90EA80F4610B8103011E8
:100B140006046F04DF045705D7055E06EC0682075A
:100B24002008C5087109250AE10AA40B6E0C400DC2
:100B3400170EE90EA80F4610B81030110001020379
:100B44000405060708090A0B0C0D0E0F001000001F
:100B54006410B71DC8206E3BAC30D9269041DC76BA
:100B6400F4516B6B5861B24D3C7105502083B8ED64
:100B740044930FF0E8A3D6D68CB361CBB0C2649B88
:100B8400D4D2D38678E20AA01CF2BDBD417462506F
:100B9400736131323536507475355F21003778A76B
:100BA40030203F3F660041544256414C5545434135
:100BB400524456303032000076616C6964204D69CD
:100BC40066617265636172642053657276696365F8
:100BD40020646F6F720076616C6964204D69666190
:100BE400726563617264205661756C7420646F6F02
:100BF400720066696C6520697320746F6F20626986
:100C0400672C206D6178203830306279746500700B
:100C14006C6561736520776169742E2E2E00736C88
:100C2400656570206D6F6465206F666600736C6522
:100C34006570204F4B002D2D2D2D2D2D2D2D2D2D5F
:100C44002D2D2D2D2D2D2D2D2D2D2D2D2D2D2D2DD0
:100C54002D2D2D2D2D2D2D2D2D2D2D2D2D2D2D2DC0
:100C64002D2D2D2D2D2D2D2D002D2D2D2D2D2D2DDD
:100C74002D2D202044657669636520436F6E747260
:100C84006F6C6C65722048656C7020536372656587
:100C94006E202D2D2D2D2D2D2D2D2D007C2D2D2D2A
:100CA4002D2D2D2D2D2D2D2D2D2D2D2D2D2D2D2D70
:100CB4002D2D2D2D2D2D2D2D2D2D2D2D2D2D2D2D60
:100CC4002D2D2D2D2D2D2D2D2D2D2D2D2D2D007C2E
:100CD400007C202020275027203D20446973706C1D
:100CE4006179204D616368696E6520536574746928
:100CF4006E6773007C202020275327203D20446901
:100D040073706C61792044657669636520537461FE
:100D14007465007C202020275727203D20446973D8
:100D2400706C61792057616B6520536F75726365D0
:100D3400007C2020202754787827203D20446973A4
:100D4400706C6179205469636B6574206E722078CD
:100D540078203D2030312E2E3332007C2020202775
:100D64007427203D2052756E20636F6D706C65741E
:100D7400652073797374656D20636865636B2028DF
:100D840031377329007C202020277027203D2050F4
:100D940072696E7420546573747469636B6574004E
:100DA4007C202020276327203D2052756E20636F0E
:100DB400696E2074657374007C20202027752720B9
:100DC4003D206F70656E20757070657220636F765C
:100DD4006572202020277627203D206F70656E20C5
:100DE4007661756C7420646F6F7220636F766572C0
:100DF400007C202020276C27203D206C6564206F18
:100E04006E203373202020276F27203D206C6564DB
:100E1400206F6666007C202020273027203D207329
:100E24006C656570206F6666202873746179206133
:100E340077616B652920202020273127203D2073EE
:100E44006C656570206F6E202864656661756C74CE
:100E540029007C202020277327203D207369726598
:100E64006E206F6E20666F7220313073007C2020FC
:100E7400202764787827203D205072696E742054AE
:100E840069636B6574206E72207878203D20303160
:100E94002E2E3332007C202020276B636363636330
:100EA40027203D20656E6361736820616D6F756EE8
:100EB400742028356469676974732920696E206316
:100EC400656E74007C20202073656E64206A736FE5
:100ED4006E2D66696C652077697468202253454ECF
:100EE400442046494C452D427574746F6E004D6123
:100EF4006368696E652053657474696E67733A003C
:100F0400437573746F6D65724E723A20004D616360
:100F140068696E654E723A202000426F726F756781
:100F2400683A20202020005A6F6E653A2020202045
:100F340020202000416C6961734E723A20202020E9
:100F4400004D79506C6163653A20004D617374659E
:100F54007220496E746572666163653A0043757206
:100F640072656E742042617564726174653A200022
:100F740020202020303D393630302020313D31349E
:100F84006B342020323D31396B322020333D3338ED
:100F94006B342020343D35372C362020353D31311B
:100FA400356B322020363D3233306B34004372636C
:100FB40020636865636B3A20005061726974793A02
:100FC40020002020202020202F2F2070617269749F
:100FD400793A20303D6E6F2020313D6576656E2074
:100FE40020323D6F64640044617461626974733AD1
:100FF40020002020202020202F2F206461746120D5
:10100400626974733A20303D356269742020313D41
:1010140036626974202020323D37626974202020B2
:10102400333D38626974202020343D39626974008C
:1010340053746F70626974733A200020202020205A
:10104400202F2F20303D3173746F7062697420201B
:101054002020313D3273746F70626974730044658B
:1010640076696365733A005072696E746572202004
:10107400203A2000436F696E43686B2020203A2099
:10108400004D6966617265202020203A20004D6180
:10109400696E73537570706C793A20004D6F646596
:1010A4006D20202020203A20004372656469744337
:1010B4006172643A2000457363726F7720202020A8
:1010C4003A200052656A4D6F746F7220203A2000F6
:1010D400536875747465722020203A200042696C4C
:1010E4006C2020202020203A20005661756C744C1E
:1010F4006F636B203A20004175746F416C61726DAF
:10110400203A20004175746F4F70656E20203A209C
:10111400005374617465206F6620616C6C204465B3
:1011240076696365732028313D4F4B2020317878F0
:101134003D7761726E696E6720203278783D657202
:10114400726F72290052616D3A2000496E744565D0
:101154003A200045787445653A20005274633A2079
:10116400004272642048573A200050726E3A2000C0
:101174004D6F64656D3A20005369676E616C3A2067
:10118400005265676973743A20004D646242757356
:101194003A2000436F696E43686B3A2000457363DD
:1011A400726F773A20004D6966526561643A200097
:1011B40043437465726D3A200052656A6563743AFC
:1011C40020005661756C743A200042696C6C626F41
:1011D400783A2000566F6C743A200054656D703A6A
:1011E40020005077724F6E5473743A2000446F6F2E
:1011F4007253746174653A2000446F6F725761735F
:101204004F70656E3A20004368616E6765723A20DC
:1012140000436F696E536C6F743A200042696C6CC2
:101224003A20004C617374205265736574206279AE
:101234003A2000416C6C20436865636B65643A2016
:1012440000416C61726D3A2000444332632E3034A5
:101254002E30392031352E30332E323032330044A3
:1012640043322053577665723A2000444332635F19
:101274006F6374323032320044433220485776650B
:10128400723A2000504F32655F6E6F7632303232E0
:1012940000504F322048577665723A2000616C6CDA
:1012A4002064796E616D69632076616C7565733A4B
:1012B400006B657074206177616B652062793A20F8
:1012C40000646F6F725F6F70656E3A2000757020F6
:1012D400006D6964646C652000646F776E20002083
:1012E400616C6C20646F6F727320636C6F736564E0
:1012F400206E6F77200020202F6F6E416C61726D1D
:101304000020202F43426368616E67650020202F10
:101314004E6F436F696E626F780020202F556261B3
:1013240074745B565D3D0020202F54656D705BB076
:10133400435D3A2000006572726F7220696E20630B
:101344006F6E6669672066696C6500636F6E6669B7
:101354006720757064617465207375636365737366
:10136400006572726F7220696E2073657269616CB8
:101374002066696C650073657269616C20757064C0
:101384006174652073756363657373006572726F4E
:101394007220696E206465766963652066696C6590
:1013A4000064657669636520757064617465207393
:1013B400756363657373006572726F7220696E2062
:1013C400636173682066696C650063617368207586
:1013D400706461746520737563636573730065720B
:1013E400726F7220696E207072696E7478782066EC
:1013F400696C65007072696E7478782075706461C8
:1014040074652073756363657373006572726F72BC
:1014140020696E2074696D652066696C6500746965
:101424006D6520757064617465207375636365739D
:10143400730077726F6E672066696C6500746974F7
:101444006C65003F3F3F444332435F636F6E6669A0
:1014540067003F3F3F444332435F73657269616C89
:10146400003F3F3F444332435F64657669636500F0
:101474003F3F3F444332435F636173682020003F32
:101484003F3F444332435F707269003F3F3F4443F0
:1014940032435F74696D6500637573744E756D00D6
:1014A4006D6163684E756D00626F726F7567680079
:1014B4007A6F6E6500616C696173006C6F6361744F
:1014C400696F6E0063726343686B00626175645296
:1014D400617465006461746100706172697479009B
:1014E40073746F70007072696E74657200636F69F3
:1014F4006E43686B006D6966526400736F6C617251
:10150400507772006D6F64656D0063726564697411
:101514004361726400657363726F770052656A4D4C
:101524006F746F7200736875747465720062696CAD
:101534006C5264007661756C744C6F636B006175FA
:10154400746F416C61726D006175746F4F70656E7C
:101554000072657365727665006C6F63616C436FCE
:10156400696E416363657074004E616D65206F66DA
:1015740020437572006C6F63616C20746178207213
:1015840061746500666F726569676E436F696E5654
:10159400616C75650043757272656E63794E616D39
:1015A4006500666F726569676E2074617800546FB8
:1015B4006B656E4368616E6E656C0042696C6C733A
:1015C40028372E2E3029007375726368617267653F
:1015D40000646973636F756E74006578636867523D
:1015E40061746500637572722E796561720063754A
:1015F40072722E6D6F6E746800637572722E646FF2
:101604006D00637572722E686F7572006375727205
:101614002E6D696E00637572722E73656300637557
:1016240072722E646F770070726F6A6563740074EF
:1016340065787400697373756564007374796C00FC
:1016440066656564007661726900677261660000B0
:1016540063617368207374617274207061796D655D
:101664006E7400636173682073746F7000636173D8
:10167400682072656164790063617368206C6173CA
:101684007420636F696E00206361736820676F74F0
:1016940020636F696E3A200020746F74616C3A2085
:1016A4000063617368207374617274436F6C6C209F
:1016B400776974682000636173682073657475705A
:1016C400200073746F70207061796D656E74206191
:1016D400742000000A000000000000000000000068
:1016E40000000000000000000000000000000000F6
:1016F4000000000000000100DB19D8160000000003
:10170400F894EE27EFBBF1E0F5BFE5BFE09374007A
:10171400E09375008DE0A2E0BB27ED938A95E9F78D
:1017240080E090E2A0E0B2E0ED930197E9F7EAEF00
:10173400F6E1D0E0DBBF87919791009781F0A79104
:10174400B79107901790C791D791BF01DBB7F0010C
:10175400CBBF07900D920197E1F7FB01EBCFE0E0DF
:10176400EEBBEFEFEDBFE1E2EEBFC0E0DAE00C94D8
:10177400256B0E94D9B81A2F2B2F3C81343010F4DA
:101784000C94C50B30E03295307F330F330F307C2F
:1017940030937C00E7E9E0937A00012FAEE7B0E0F4
:1017A400EC91E02BEC93EFEF0E27E0B3E023E0BBEA
:1017B400122F2227012FADE7B0E0EC91E02BEC9340
:1017C400EFEF0E27A7E0B1E0EC91E023EC930E9449
:1017D400E0B825960895E0E0E0937A0008950A932E
:1017E4000A2F003110F40C94FA0BE0E009910895EB
:1017F400083010F40C94050CE0917B00E860E09351
:101804007B00077005C0E0917B00E77FE0937B00DD
:10181400083010F00C941D0CE0917C00E87FE093FC
:101824007C00ACE7B0E0EC91E02BEC93E0917A0023
:10183400E064E0937A00E1E0099108950E94DAB847
:1018440000E010E0E0917A00E0712E2F81E791E052
:101854000197F1F7203011F00C943A0CF80131960D
:101864008F01E436A0E0FA0710F00C943A0C01C0A2
:1018740001C0E8CFE0917A00E061E0937A00009142
:10188400780010917900F8010E94E1B82396089538
:10189400E0E0EDBBE093680008950A930A2F00305E
:1018A40011F00C945E0CE0916A00E2600E948BA43B
:1018B400EE7FE0936A00EC9A013011F00C94680C0E
:1018C400E0916A00E360E0936A00EC9A023011F060
:1018D4000C94720CE0916A00EC7FE0936A00EC9A3D
:1018E40009910895EC9808950E9490A40E94586F5D
:1018F4000E94A2A418950A930A2F003011F00C94A8
:101904008C0CE0916A00E8600E948BA4EB7FE0936A
:101914006A00ED9A013011F00C94960CE0916A0083
:10192400EC60E0936A00ED9A023011F00C94A00C84
:10193400E0916A00E37FE0936A00ED9A09910895CB
:10194400ED9808950E9490A40E946E6F0E94A2A434
:1019540018950A930A2F003011F00C94BA0CE091F8
:101964006A00E0620E948BA4EF7EE0936A00EE9A24
:10197400013011F00C94C40CE0916A00E063E09330
:101984006A00EE9A023011F00C94CE0CE0916A00D9
:10199400EF7CE0936A00EE9A09910895EE98089519
:1019A4000E9490A40E94836F0E94A2A418950A9397
:1019B4000A2F003011F00C94E80CE0916A00E06802
:1019C4000E948BA4EF7BE0936A00EF9A013011F040
:1019D4000C94F20CE0916A00E06CE0936A00EF9AD8
:1019E400023011F00C94FC0CE0916A00EF73E09368
:1019F4006A00EF9A09910895EF9808950E9490A4BF
:101A04000E94966F0E94A2A418950E94B4A40E94FA
:101A1400B4A40E94B4A4A8E6B0E0EC91EC930895B9
:101A24000E9490A40E94E56F0E94A2A418950E94AF
:101A340090A40E94E86F0E94A2A418950D9400F04F
:101A440008950E94BAA4F99B01C0FDCF22BD11BD27
:101A5400F89A00B50E94BFA408950E94C4A4F99BFB
:101A640001C0FDCF09851A852F81388540E0F90131
:101A7400A42FB0E0AE17BF0710F00C944C0D0E94D9
:101A8400C9A4AD81BE81EE27A40FBE1FE0B5EC93BF
:101A94004F5FEDCF0E94DFB82B9608950E94D8B80F
:101AA4002A2F3D814E81F99B01C0FDCF1FB742BD56
:101AB40031BDF89A00B5201711F40C94660D20BDC1
:101AC400E4E0EFBBE2E0EFBB17FF01C078940E94B3
:101AD400DFB8279608950E94D0A4F99B01C0FDCFDA
:101AE4000C851D852A853B85EFB7EE8340E0F9011F
:101AF400A42FB0E0AE17BF0710F00C949A0DA88580
:101B0400B985EE27A40FBE1F5C910E94C9A4E0B55D
:101B1400EF83AF815A1711F40C94980D50BDE4E093
:101B2400EFBBE2E0EFBBF99B01C0FDCF4F5FDFCF1E
:101B3400EE81E07811F40C94A00D78940E94DEB844
:101B44002E9608950A932B9823982A98229A2998D6
:101B5400219A289A209A02E0E02FE03011F00C94A8
:101B6400B80DE1E0EDBDE0E5ECBD35C0E13011F0CC
:101B74000C94C10DE0E0EDBDE0E5ECBD2CC0E2301D
:101B840011F00C94CA0DE1E0EDBDE1E5ECBD23C01C
:101B9400E33011F00C94D30DE0E0EDBDE1E5ECBDD4
:101BA4001AC0E43011F00C94DC0DE1E0EDBDE2E587
:101BB400ECBD11C0E53011F00C94E50DE0E0EDBD95
:101BC400E2E5ECBD08C0E63011F00C94ED0DE0E068
:101BD400EDBDE3E5ECBD09910895E0E0ECBD0895A9
:101BE400E0E0E4BDE5BDE0936E00E093B000E09377
:101BF400B100E0937000E093B600E3BDE093800091
:101C0400E0939000E093A000E0932001E093810032
:101C1400E0939100E093A100E0932101E09382001E
:101C2400E0939200E093A200E0932201E0936F001E
:101C3400E0937100E0937200E093730008951A93A7
:101C44000A931CE0E3B70E2FAE2FE5E0EA23AE2F94
:101C5400E5E00E9476B9E03011F40C94420EE12FD5
:101C6400E1501E2FEF5FAE2FEAE00E9480B9E03012
:101C740011F40C943E0EF3CFE0E00991199108950C
:101C8400E0E0E4BDE1E0E5BDE0E0E7BDE6EBF0E087
:101C9400DF01E0E0EC93E6BDE6B5AE2FE7E30E949A
:101CA4007BB9E03011F40C94580EF6CFE0E00991C2
:101CB400199108950E94D9B89D017894E0E0F0E06C
:101CC4008F010E94210EF80131968F013197F8019E
:101CD400FF93EF93F901AF91BF910E948BB9E0306C
:101CE40011F40C94760EEDCFE7E0F0E08F018F0154
:101CF4000E94E0B8249608950E94D7B8AD01FA0175
:101D04009F01E0E0F0E08F01E4E6F0E0DF010E94F3
:101D14005C0EF80131968F013197F801FF93EF9330
:101D2400F901AF91BF910E948BB9E03011F40C948A
:101D34009C0EEACFE8E0F0E08F018F010E94DEB84C
:101D440026960895E0E0E0939000E09392000E94CC
:101D5400D6A4E0917100E260E0937100E2E0E093C8
:101D64009100E8E4E0939900E0E0E0939800EFEF5D
:101D7400E8BB08950E9490A40E94D6A4A0E0BAE013
:101D84000E94DCA40E94E06FA4E0BAE00E94DCA4FC
:101D9400A091040AB091050AA436E0E0BE0710F44D
:101DA4000C94DF0EE0E0E093040AE093050AA2E05D
:101DB400BAE00E94DCA40E94DF6FEFEFE8BB0E9450
:101DC400A2A41895A0919100A03011F40C94F10EE6
:101DD400A0917100A03011F40C94F10E02C0E0E067
:101DE4000895E1E0089518950A930A2F083210F433
:101DF4000C94FF0EE1E009910895E02F0E94E2A403
:101E0400EA0FFB1FA091000AB091010AA083B183DD
:101E1400E0E0099108950E94D7B85A2F583210F47F
:101E24000C94180F0E94E8A426960895452F20913B
:101E3400000A3091010AE42F0E94E2A40E94EDA45A
:101E440010F40C94300FE42F0E94E2A40E94F4A436
:101E5400DF01F901EA1BFB0B8F0107C0E42F0E948D
:101E6400E2A40E94F4A40E94F9A4F8010E94DEB83E
:101E7400269608950A930A2F043110F40C94450F02
:101E8400E1E009910895E02F0E9403A5EA0FFB1FEA
:101E9400A091020AB091030AA083B183E02FF0E07D
:101EA400E258F54FA1E0A08309910895AA930E94F6
:101EB400D8B84D81443110F40C94660FE0E0F0E0A2
:101EC4000E94DFB826960895E42FF0E0E258F54F1B
:101ED400E081E03011F00C94750FE0E0F0E00E9436
:101EE400DFB8269608952091020A3091030AE42F60
:101EF4000E9403A50E94EDA410F40C948C0FE42F0F
:101F04000E9403A50E94F4A4DF01F901EA1BFB0B64
:101F14008F0107C0E42F0E9403A50E94F4A40E942D
:101F2400F9A4F8010E94DFB8269608950E9490A4AF
:101F3400E0E0E0938500E09384000E94E36F0E9458
:101F4400A2A418950E9490A4E0E0E6BD0E94E46F6C
:101F54000E94A2A418952C970A930E9409A50E9496
:101F64000EA50E9413A50E9413A5EAB1E360EAB985
:101F7400EBB1E360EBB9E0916400EF77E0936400C8
:101F8400E4E0E093BC00E985FA856B857C850E94DA
:101F94001CA50E9421A50E9426A50E942BA50E9493
:101FA4002EA5E051F040604070400E9433A50E948D
:101FB4006CB90E941CA500E00E9426A5A030E1E0B7
:101FC400BE07E0E08E07E0E09E0710F40C94F40FE7
:101FD4000E9426A5E4E0F0E060E070E00E942BA5FA
:101FE4000F5FEACFED81E093B8000093B900088158
:101FF4002D960895E0E0E093BC00E0916400E06871
:10200400E0936400EAB1EC7FEAB9EBB1E360EBB9C9
:1020140008950E9436A50F5F1F4F81E38A95F1F75B
:10202400E091BC00E07811F00C941F100436E0E05D
:102034001E0714F00C941F1001C001C0ECCF04362D
:10204400E0E01E0714F40C942B10E1E009911991BF
:102054000895E0E00991199108950E943BA5022F8B
:102064004093BB00303011F40C943C10E4EAE0934C
:10207400BC0003C0E4E8E093BC000E940B101E2FD8
:10208400113010F40C944B10EAE00E94DFB827964C
:102094000895E091B900E87F0E1711F40C945A10DA
:1020A400E4E9E093BC00E1E00E94DFB827960895DC
:1020B400E0E00E94DFB8279608950E94DAB80E94F3
:1020C400FC0F509A51985998AAE0B0E00E9440BC85
:1020D400E9B1E1700E2FE9B1E2701E2F103011F05A
:1020E4000C94901020E058988AE08A95F1F7589A59
:1020F4008AE08A95F1F7E9B1E2701E2F2F5F103064
:1021040011F00C948A10203210F00C948A1001C043
:1021140001C0E9CFA2E0B0E00E9440BC103011F44D
:102124000C9496100E94AD0FA2E0B0E00E9440BC57
:102134000E94E1B8239608950E94D0A40E9441A56C
:1021440011F00C94A8100770000F202B0E944CA5CE
:1021540011F40C94B0100E9457A508950E945CA538
:1021640011F00C94BA10E2E00E94DEB82F960895A4
:10217400313011F00C94C1100E9465A508955030BF
:1021840011F40C94CD100E946AA511F40C94CD1096
:102194000E9473A508950E9478A511F40C94D5109B
:1021A4000E9473A50895E0E0EE83EF830E9481A569
:1021B400AE17BF0710F00C94F3100E9486A5AE0F63
:1021C400BF1FEC91EA93E0E0EA93A8E20E948BA59A
:1021D40011F40C94F0100E9490A508950E9495A506
:1021E400E5CF0E949BA508950E94A3A50E94AAA5DD
:1021F4000E949E100E2F013010F40C9403110E94C3
:102204005F10013010F40C940D111F5F153010F0A5
:102214000C940D1101C001C0E9CF7894013010F481
:102224000C941411E02F0E94DEB82B9608950E949E
:10223400D0A40E9441A511F00C9423110770000F43
:10224400202B0E944CA511F40C942B110E9457A52D
:1022540008950E945CA511F00C943511E2E00E94EF
:10226400DEB82F960895313011F00C943C110E9481
:1022740065A50895503011F40C9448110E946AA584
:1022840011F40C9448110E9473A508950E9478A536
:1022940011F40C9450110E9473A508950E94B4A5E2
:1022A400A0E10E948BA511F40C945B110E9457A528
:1022B400089521602A93E0E0EA93A0E40E948BA5AC
:1022C40011F40C9468110E9465A508954150E0E052
:1022D400EE83EF830E9481A5EA17FB0710F40C94A8
:1022E400C3110E9481A5EA17FB0711F00C947E111B
:1022F400E4E8E093BC0003C0E4ECE093BC000E947B
:102304000B10E03011F40C948A110E9490A50895EA
:10231400E091B900E87FE03511F00C9499110E9426
:1023240081A5AE17BF0710F00C94991101C008C025
:102334000E9486A5AE0FBF1FE091BB00EC931EC0A8
:10234400E091B900E87FE83511F00C94B1110E94D6
:1023540081A5EA17FB0711F00C94B11101C008C064
:102364000E9486A5AE0FBF1FE091BB00EC9306C090
:10237400E4E9E093BC000E9490A508950E9495A50D
:10238400A9CF0E949BA508950E94A3A50E94AAA577
:102394000E9419110E2F013010F40C94D3110E94D5
:1023A4005F10013010F40C94DD111F5F153010F034
:1023B4000C94DD1101C001C0E9CF7894013010F410
:1023C4000C94EF1110E0E8851E1710F00C94EF1137
:1023D4000E94B9A5EC931F5FF6CFE02F0E94DEB8F0
:1023E4002B960895A091C40DA23010F40C94FF1103
:1023F400AE3F10F00C94FF1101C005C0E091C40D74
:10240400EF5FE093C40DA0912E0EA23010F40C9453
:102414001012AE3F10F00C94101201C005C0E091F0
:102424002E0EEF5FE0932E0EA0915E11A23010F4F9
:102434000C942112AE3F10F00C94211201C005C07F
:10244400E0915E11EF5FE0935E11A091C811A2309C
:1024540010F40C943212AE3F10F00C94321201C0FE
:1024640005C0E091C811EF5FE093C81108950A9385
:102474000A2FE02FE13011F00C944312EFE309919D
:102484000895E23011F00C944A12EFE20991089594
:10249400E33011F00C945112E7E109910895E4300E
:1024A40011F00C945812EFE009910895E53011F001
:1024B4000C945F12E7E009910895E63011F00C9452
:1024C4006612E3E009910895EFE5099108950E94E9
:1024D400BEA5E093C000E0E0E093C100E093C20039
:1024E400E093C500EAE2F3E0E093C20DF093C30D7C
:1024F400A091C20DB091C30D139710F00C948812E3
:10250400E3E0F0E0E093C20DF093C30DA32F0E942B
:102514003912E093C400E22FE13011F00C949812C8
:10252400E091C200E260E093C20022C0E23011F008
:102534000C94A212E091C200E460E093C20018C0BF
:10254400E33011F00C94AC12E091C200E660E09329
:10255400C2000EC0E43011F00C94BA12E091C20033
:10256400E660E093C200E091C100E460E093C10042
:10257400E12FE13011F00C94C412E091C200E86044
:10258400E093C200E02FE13011F00C94CF12E091FF
:10259400C200E062E093C20009C0E23011F00C9482
:1025A400D812E091C200E063E093C200E42FE1306E
:1025B40011F00C94E312E091C100E861E093C100D2
:1025C40009C0E23011F00C94EC12E091C100E8690A
:1025D400E093C1000E94DFB829960895E0E0E093FB
:1025E400C10008950A930A2FE091C000E07211F02F
:1025F4000C94FD12F9CF0093C600099108950E942E
:1026040036A50E94C7A50E171F0710F00C941113CE
:10261400A5E9BAE00E94CCA50F5F1F4FF2CFE0E01E
:10262400E093BF0DE093C00DE093C10DE1E0E093B2
:10263400C40D0991199108950E94D1A50E94D9B899
:10264400A091C40DA13010F40C942B13E2E0E0939C
:10265400C40DE091C100E47011F40C9465130E9460
:10266400C7A532970E94D8A510F00C945313E0919B
:10267400C100E27011F40C9447130E94DFA5319756
:10268400EB56F54FA1E0A08307C00E94DFA5319768
:10269400EB56F54FA0E0A0830E94DFA50E94E2A5BF
:1026A40002C00091C600E091BF0DE2501E2FF0E081
:1026B400EB56F54F0E94EAA5EB56F54FE081F0E0AA
:1026C4002E2B3F2B0EC00E94C7A50E94D8A510F048
:1026D4000C9471130E94DFA50E94E2A502C0009130
:1026E400C600E091C000EC710E2F013010F40C9480
:1026F4008213A091C10DA03011F00C94821301C07B
:1027040002C00093C10D0E94E0B824960E94F2A575
:1027140018950E94F9A508950E94D7B8AD01A0911B
:10272400BF0DB091C00D4A175B0710F00C949C13B9
:10273400FA0102C00E94F9A59F0100E010E002170F
:10274400130710F00C94AF130E94FEA5A5E9BAE09C
:102754000E9405A60F5F1F4FF2CF0E940BA6A4365E
:10276400E0E0BE0710F00C94BB130E94F9A50E9490
:1027740010A60E94DEB8289608950E9417A60E940B
:102784001EA610F40C94C913A22F0E94F412003D4B
:10279400E7E01E0710F00C94D413213010F40C94CD
:1027A400D41301C001C0EBCF78940E94DFB8259602
:1027B40008950E9426A600E010E00217130710F007
:1027C4000C94ED13F801E40FF51FA0810E94F4129C
:1027D4000F5F1F4FF2CF0E94DEB8289608950E9423
:1027E400BEA5E093C800E091C900EC79E093C9006C
:1027F400E091C900E861E093C900E091CA00EE737A
:10280400E093CA00E0E0E093CD00E4E6F0E0E0937A
:102814002C0EF0932D0EA0912C0EB0912D0E13972B
:1028240010F00C941B14E3E0F0E0E0932C0EF09312
:102834002D0EA32F0E943912E093CC00E22FE13039
:1028440011F00C942B14E091CA00E2600E942EA6B1
:1028540022C0E23011F00C943514E091CA00E46017
:102864000E942EA618C0E33011F00C943F14E0919E
:10287400CA00E6600E942EA60EC0E43011F00C944B
:102884004D14E091CA00E660E093CA00E091C900EB
:10289400E460E093C900E12FE13011F00C94571487
:1028A400E091CA00E860E093CA00E02FE13011F043
:1028B4000C946214E091CA00E062E093CA000FC075
:1028C400E23011F00C946C14E091CA00E063E093E0
:1028D400CA0005C0E091CA00EF7CE093CA00E42F6F
:1028E400E13011F00C947C14E091C900EF77E0938F
:1028F400C90009C0E23011F00C948514E091C900BC
:10290400E068E093C90089E18A95F1F70E94DFB895
:1029140029960895E0E0E093C90008950A930A2FE8
:10292400E091C800E07211F00C949914F9CF00936F
:10293400CE00099108950E9436A50E9436A60E176E
:102944001F0710F00C94AD14A5ECBDE00E94CCA5BB
:102954000F5F1F4FF2CFE0E0E093290EE0932A0EC1
:10296400E0932B0EE093C911E1E0E0932E0E099160
:10297400199108950E94D1A50A93A0912E0EA13019
:1029840010F40C94CB14E1E0E093C911E2E0E0937D
:102994002E0EE091C900E47011F40C94F8140E9416
:1029A40036A632970E940BA6AE17BF0710F00C9400
:1029B400F514E091C900E27011F40C94E9140E943A
:1029C4003BA63197EB53F24FA1E0A08307C00E94CE
:1029D4003BA63197EB53F24FA0E0A0830E943BA6A5
:1029E4000E943EA602C00091CE0010C00E9436A6EE
:1029F4000E940BA6AE17BF0710F00C9406150E9498
:102A04003BA60E943EA602C00091CE00E091C80001
:102A1400EC710E2F013010F40C941715A0912B0EAD
:102A2400A03011F00C94171501C002C000932B0EB6
:102A340009910E94F2A51895E0912B0EE03011F057
:102A44000C9427150E9446A60895E0912B0EE07180
:102A540011F40C943015EFEFFFEF0895E0912B0E75
:102A6400E87011F40C943915EEEFFFEF0895E0913E
:102A74002B0EE47011F40C944215EDEFFFEF089562
:102A840008950E94D7B8AD010E940BA64A175B07B0
:102A940010F00C944F15FA0102C00E9446A69F0143
:102AA40000E010E00217130710F00C9462150E9466
:102AB400FEA5A5ECBDE00E9405A60F5F1F4FF2CF57
:102AC4000E940BA6A436E0E0BE0710F00C946E152D
:102AD4000E9446A60E9410A60E94DEB82896089579
:102AE400A0912E0EA53010F40C947D15E0E0E09337
:102AF4002E0EE1E00895E0E0089508950E944BA6AB
:102B040000E010E02F81388540E050E00E94B926B3
:102B1400E03011F00C9495154436E0E05E0710F0B7
:102B24000C94951501C007C0A1E0B0E00E9440BC20
:102B34004F5F5F4FEBCFF8010F5F1F4FA985BA8539
:102B4400AE0FBF1FEC91EE83AE810E94901402176A
:102B5400130710F00C94AF15D7CF0E94DEB82B9654
:102B640008950E946FBA0E94D8B800E010E020E0F7
:102B740030E00E94B926E03011F00C94C8152436D8
:102B8400E0E03E0710F00C94C81501C007C0A1E0B6
:102B9400B0E00E9440BC2F5F3F4FEBCFF8010F5FC6
:102BA4001F4F0E9426A50E9451A66BBF469141303B
:102BB40010F40C94E015A42F0E949014003DE7E05B
:102BC4001E0710F00C94EB15413010F40C94EB1527
:102BD40001C001C0CCCF78940E94DFB82996089533
:102BE4000E94BEA5E093D000E0E0E093D100E09322
:102BF400D200E093D500EAE2F3E0E0935C11F093B5
:102C04005D11A0915C11B0915D11139710F00C94BB
:102C14001116E3E0F0E0E0935C11F0935D11A32F53
:102C24000E943912E093D400E22FE13011F00C94A9
:102C34002116E091D200E260E093D20022C0E2309B
:102C440011F00C942B16E091D200E460E093D200D2
:102C540018C0E33011F00C943516E091D200E66010
:102C6400E093D2000EC0E43011F00C944316E091CE
:102C7400D200E660E093D200E091D100E460E093FA
:102C8400D100E12FE13011F00C944D16E091D20007
:102C9400E860E093D200E02FE13011F00C94581674
:102CA400E091D200E062E093D20009C0E23011F07A
:102CB4000C946116E091D200E063E093D200E42F1B
:102CC400E13011F00C946C16E091D100E861E093CE
:102CD400D10009C0E23011F00C947516E091D100D6
:102CE400E869E093D1000E94DFB829960895E0E0F6
:102CF400E093D10008950A930A2FE091D000E07286
:102D040011F00C948616F9CF0093D600099108951A
:102D14000E9436A5E0915C11F0915D110E171F071A
:102D240010F00C949C16AFE2BEE00E94CCA50F5F9D
:102D34001F4FF0CFE0E0E0935911E0935A11E09374
:102D44005B11E1E0E0935E110991199108950E94ED
:102D5400D1A50A93A0915E11A13010F40C94B5167C
:102D6400E2E0E0935E11E0915C11F0915D110E944C
:102D740056A6AE17BF0710F00C94CC16A9E5B1E126
:102D84000E94DCA43197E15DF14FDF01E091D600B0
:102D9400EC9302C00091D600E091D000EC710E2FAC
:102DA400E0915B11E03011F00C94DA1600935B11A2
:102DB40009910E94F2A518950E945BA608950E94AD
:102DC400D7B8AD010E9456A64A175B0710F00C94C1
:102DD400ED16FA0102C00E945BA69F0100E010E01C
:102DE4000217130710F00C9400170E94FEA5AFE21F
:102DF400BEE00E9405A60F5F1F4FF2CF0E9456A6A9
:102E0400AA32E3E0BE0710F00C940C170E945BA6F4
:102E14000E9410A60E94DEB828960895A0915E1123
:102E2400A43010F40C941B17E0E0E0935E11E1E091
:102E34000895E0E0089508950E9417A60E941EA632
:102E440010F40C942817A22F0E947D16003DE7E091
:102E54001E0710F00C943317213010F40C94331720
:102E640001C001C0EBCF0E94DFB8259608950E94EF
:102E7400C4A400E010E02D813E81F8010F5F1F4FD4
:102E84000E9460A64C91A42F0E947D16021713077E
:102E940010F00C944E17F1CF0E94DFB829960895D4
:102EA4000E94BEA5E0933001E0E0E0933101E0939D
:102EB4003201E0933501E4E6F0E0E093C611F093CB
:102EC400C711A091C611B091C711139710F00C94BB
:102ED4007117E3E0F0E0E093C611F093C711A32F5C
:102EE4000E943912E0933401E22FE13011F00C9486
:102EF4008117E0913201E260E093320122C0E230B6
:102F040011F00C948B17E0913201E460E0933201EC
:102F140018C0E33011F00C949517E0913201E6608B
:102F2400E09332010EC0E43011F00C94A317E09149
:102F34003201E660E0933201E0913101E460E09314
:102F44003101E12FE13011F00C94AD17E091320121
:102F5400E860E0933201E02FE13011F00C94B817EF
:102F6400E0913201E062E093320109C0E23011F0F5
:102F74000C94C117E0913201E063E0933201E42F35
:102F8400E13011F00C94CC17E0913101E861E09349
:102F9400310109C0E23011F00C94D517E0913101F0
:102FA400E869E093310181E38A95F1F70E94DFB883
:102FB40029960895E0E0E093310108950E9436A532
:102FC4000E9465A60E171F0710F00C94F017AFE5CA
:102FD400B1E10E94CCA50F5F1F4FF2CFE0E0E09378
:102FE400C311E093C411E093C511E1E0E093C8116B
:102FF4000991199108950A930A2F003011F40C9441
:103004000918E0913101E160E093310105C0E091DC
:103014003101EE7FE0933101099108950A930A2F5B
:10302400E0913001E07211F00C941918F9CF00937B
:103034003601099108950E9490A40E94D9B8A091E4
:10304400C811A13010F40C942A18E2E0E093C811DE
:10305400E0913101E47011F40C9467180E9465A6A4
:1030640032970E946AA610F00C945218E091310134
:10307400E27011F40C9446180E9471A63197E15A3B
:10308400FE4EA1E0A08307C00E9471A63197E15AC9
:10309400FE4EA0E0A0830E9471A60E9474A602C006
:1030A40000913601E091C311E2501E2FF0E0E15A85
:1030B400FE4E0E94EAA5E15AFE4EE081F0E02E2B7E
:1030C4003F2BD9010E9481381BC00E9465A60E9433
:1030D4006AA610F00C9474180E947CA610F00C944C
:1030E400741801C005C00E9471A60E9474A602C093
:1030F400009136010E947CA610F40C94821800E022
:10310400E0913001EC710E2FE091C511E03011F027
:103114000C948E180093C5110E94E0B824960E9466
:10312400A2A41895BA93AA932997E0E0ED83EE83BD
:103134000E94D7B80B8D1C8D00FF02C0E1E0EC8724
:103144000436E0E01E0710F00C94B318E1E0EB87BE
:10315400E4E6F0E0E01BF10BAF01F695E7959F0183
:1031640008C0E0E0EB8704561040F801F695E795B7
:103174009F012436E0E03E0710F40C94DC18E3E0F1
:10318400EA87D901E4E6F0E00E94D7B9AF014987A4
:10319400D9010E9481A6ED87FE87AD85BE850E9478
:1031A40086A6AD85BE85EAE0F0E00E941BBAAF01B9
:1031B4004F831DC02A30E0E03E0710F40C94F3184E
:1031C400E2E0EA87E0E0E987D9010E9486A6D90116
:1031D400EAE0F0E00E941BBAED87FE87ED85EF83FD
:1031E40006C0E1E0EA87E0E0E987E8872F83E98524
:1031F400E05DE9870E948DA6A985A03311F00C94A7
:103204000B19E0E2E987A885A03311F00C940B199F
:10321400E887EC85E03011F40C941319E5E3EE83B0
:1032240002C0E0E3EE83EA85A98DBA8DEC93E985CB
:10323400AF89B88DEC93E885AD89BE89EC93EF81B5
:10324400AB89BC89EC93EB85A989BA89EC93EE81AF
:10325400AF85B889EC930E94DEB86D960895BA9351
:10326400AA9360970E94D7B8EB8DE987E98DE88728
:10327400EA8DEF83E88DEE83EC8DFD8DFA93EA936E
:10328400EDB7FEB7FA93EA932F93EDB7FEB7FA932F
:10329400EA933F93EDB7FEB7FA93EA934F93EDB7F2
:1032A400FEB7FA93EA935F93FE017596FA93EA9355
:1032B400DE0156960E9494185F914F913F912F9191
:1032C40000E00A3010F00C946D190E9494A6E0E01E
:1032D400EC930F5FF6CF00E0E985E03011F40C9435
:1032E4007919EB85E03011F40C94791901C006C00A
:1032F4000E949BA6AE0FBF1FEDE2EC93E885E03081
:1033040011F40C9495190E949BA6EA0FFB1F3083BD
:103314000E949BA6EA0FFB1F40830E949BA6EA0F14
:10332400FB1F508317C0233010F40C949E190E9485
:103334009BA6EA0FFB1F3083223010F40C94A719CC
:103344000E949BA6EA0FFB1F40830E949BA6EA0FE4
:10335400FB1F5083EF81E03011F40C94C5190E94D7
:103364009BA60E94A1A6EA85E03011F40C94C11931
:103374000E949BA6AE0FBF1FE5E3EC9304C00E941E
:103384009BA60E94A6A6EE81E03011F40C94D619F7
:103394000E949BA6AE0FBF1FE8EFEC930E949BA672
:1033A400AE0FBF1FE3E4EC9300E00E9494A61C91CF
:1033B400E02FAE89BF89F0E0EA0FFB1F10830F5F97
:1033C4000A3010F00C94EB19113010F40C94EB1932
:1033D40001C001C0EACF0E94DEB86E9608950E9433
:1033E40026A60217130714F00C94121A0E94ABA617
:1033F400F801E40FF51FE081EA1711F40C940B1A9D
:10340400F801E40FF51FA081AF3311F40C940B1AEB
:1034140001C003C00E94B2A608950F5F1F4FE1CF01
:10342400E1E00E94DEB82A9608950E94B7A6003013
:10343400E0EF1E0710F00C942F1AF801E20FF31FAF
:10344400E081E03011F00C942C1AF8010E94E0B8ED
:10345400249608950F5F1F4FEACFE0E0F0E00E944A
:10346400E0B824960895BA93AA93EF97EF97EF974D
:103474002F970E94D7B8DE01AC52BF4F0D90BC917C
:10348400A02D0E94171A9F01DE01AE52BF4F0D906E
:10349400BC91A02D0E94171AAF012436E0E03E072C
:1034A40014F00C94651AFE01EC52FF4F0190F08168
:1034B400E02DFA93EA93FE01E459FF4FFA93EA935D
:1034C400D9010E94061B4436E0E05E0714F00C9418
:1034D400761AFE01EE52FF4F0190F081E02D0E941A
:1034E400BDA6DA010E94061B00E010E0E0E00E94A5
:1034F400C4A6DE01A659BF4FA00FB11FAC91EE8147
:10350400EA1711F00C94C21AE1E00E94C4A6D80193
:10351400A40FB51F2A173B0714F00C94941A0E94A9
:10352400C9A60895E0E0DE01A053BF4FED93EC93EC
:103534000E94D1A6A417B50714F00C94C21AF8017E
:103544000E94D1A6EA0FFB1FDE01A659BF4FAE0FA2
:10355400BF1F1C90FE01E053FF4F0190F081E02D4E
:103564000E94D8A6EC91E11511F40C94BC1AE0E089
:103574000E94C4A6DE01A053BF4F0E94DCA4D8CF92
:103584000E94DDA6E03011F40C94D71AE02F0E94BB
:10359400E2A6EA0FDE01A253BF4FEC930E94DEB80D
:1035A400EF96EF96EF9669960895F80131968F019C
:1035B400E217F30714F00C94E01A98CF0E94C9A6FE
:1035C40008950E946FBA0E9436A50030E0EF1E07EE
:1035D40010F00C94001BF8010E94E7A60E9451A66B
:1035E4006BBFE691E03011F00C94FD1AF8011981DB
:1035F4000881269608950F5F1F4FE7CFE0E0F0E0C3
:1036040019810881269608950E9426A6022E032A6F
:1036140011F00C941B1B0E94ABA6A13010F40C9467
:10362400181B0E94ECA60F5F1F4FF5CF0E94F9A64E
:103634000EC000E010E00217130710F00C94271BD3
:103644000E94ECA60F5F1F4FF6CF0E94F9A60E94BE
:10365400DEB82A9608950E9426A6022E032A11F0A7
:103664000C94421B0E94FFA6E13010F40C943F1B03
:103674000E9407A70E940CA7F5CF0E94F9A610C0CC
:1036840000E010E00217130710F00C94501B0E9486
:1036940007A7D001EC930F5F1F4FF4CF0E94F9A648
:1036A4000E94DEB82A9608950E9426A6022E032AB6
:1036B40011F00C946B1B0E94ABA6A13010F40C9477
:1036C400681B0E9411A70F5F1F4FF5CF0E941FA711
:1036D4000EC000E010E00217130710F00C94771BE3
:1036E4000E9411A70F5F1F4FF6CF0E941FA70E94D1
:1036F400DEB82A9608950E94D0A4488559852C8561
:103704003D8500E010E00217130710F00C949C1B99
:10371400FA01E00FF11FEE83FF83AA85BB85EA0F50
:10372400FB1F0F01F801AE85BF850E9426A70F5F1E
:103734001F4FE9CF0E94DEB8609608950E94D0A47E
:103744000E851F852A853B8548855985E0E0EE83F3
:10375400EF83AE81BF81A417B50710F00C94C61B8C
:10376400EE81FF81E20FF31FAC85BD85EA0FFB1FDD
:103774000F01EE81FF81E00FF11FA889B9890E9432
:1037840026A70E9495A5E5CF0E94DEB8629608950B
:103794000E9426A600240216030610F00C94D41BE3
:1037A400215030400E942CA76BBFA691A13010F489
:1037B4000C94E31B0034E0E01E0710F00C94E31BB0
:1037C40001C00BC0F901E00FF11FE40FF51F0F0159
:1037D4000E942CA70E9432A7E5CF0E94DEB82C9647
:1037E40008950E94D8B89D014D8100E010E000E0EA
:1037F40010E00217130710F00C94071CF8010E9444
:1038040035A740830F5F1F4FF4CF0E94DFB828967F
:1038140008950E94B7A60E943AA76BBFA691A13053
:1038240010F40C941A1C0E9440A70E9432A7F3CFF4
:10383400F801E20FF31FA0E0A0830E94E0B82896ED
:1038440008950E94B7A60E943AA76BBFA691A13023
:1038540010F40C94321C0E9440A70E9432A7F3CFAC
:103864000E94E0B828960895BA93AA9327970E94D5
:10387400D8B830E040E000E0073010F00C944C1C65
:10388400AC85BD850E9445A70E944CA7E0E0EC935F
:103894000F5FF2CF1E852F8500E0012E022A11F062
:1038A4000C94581C0E9451A70E94A6A6222312F031
:1038B4000C946A1C0E9451A7AE0FBF1FEDE2EC935B
:1038C400E12FF22FAFEFBFEF0E94BFB91E2F2F2FB2
:1038D40000240116020614F00C94881CE32FF42F24
:1038E4003F5F4F4F0E9457A7BF01A12FB22FEAE0BD
:1038F400F0E00E941EBADB01EC93A12FB22FEAE0A4
:10390400F0E00E94EAB91E2F2F2FE2CF0024031605
:10391400040614F00C949D1C0E9451A7EA0FFB1F8F
:103924000F01E32FF42F31973E2F4F2F0E944CA706
:103934000E945CA7EBCF0E94DFB8609608950E94B6
:1039440061A70C3010F00C94B11CA32FB42F0E946B
:1039540045A70E946AA7E0E0EC930F5FF2CF0E94B4
:103964006FA711F00C94BA1C0E947BA7A0E3A0835C
:10397400A885AA2312F00C94CD1C0E947BA7ADE26B
:10398400A0830E942EA5AFEFBFEF8FEF9FEF0E94A1
:10399400C4B90E941CA50E9426A50E94B4BA14F0C2
:1039A4000C94E61C0E9481A7FF93EF930E948AA7C0
:1039B4000E9430BAAF91BF91EC930E948AA70E94F3
:1039C40013BA0E941CA5E7CF00240116020614F0C6
:1039D4000C94F31C0E947BA70E9491A70E945CA7F1
:1039E400F3CF0E94DFB8699608950E9461A70C3056
:1039F40010F00C94071DA32FB42F0E9445A70E941A
:103A04006AA7E0E0EC930F5FF2CF0E946FA711F07A
:103A14000C94101D0E947BA7A0E3A0830E9426A5FE
:103A24000E94B4BA10F00C94271D0E9481A7FF9342
:103A3400EF930E948AA70E942CBAAF91BF91EC9396
:103A44000E948AA70E942BA5E9CF00240116020632
:103A540014F00C94341D0E947BA70E9491A70E942D
:103A64005CA7F3CF0E94DFB869960895AA93A5973F
:103A74000E94D7B8E9A9FAA96BA97CA90E9498A7C2
:103A8400ECA5E88B1DA51B3010F40C944A1D1AE01C
:103A9400E889E03011F00C94501D10E0A889A032A0
:103AA40010F40C945A1DA03810F00C945A1D02C046
:103AB400EEE2E88B0EA50D3010F40C94621D0CE0C0
:103AC400E0E0EE87EF87AE85BF851D9714F00C9478
:103AD400781D0E949DA70E94A6A6EE85FF85DE01A3
:103AE4005E960E94A6A60E94A2A7EDCF0E94A8A758
:103AF400DE0155960E94F71CDE0151960E94171AAA
:103B0400EA87FB87AA85BB851B9714F40C948E1D4A
:103B1400EAE0F0E0EA87FB87EA85FB85309711F05D
:103B24000C949A1DE0E3E98BE1E0F0E0EA87FB877F
:103B340050E0113010F40C94281EEA85FB85A12F67
:103B4400B0E0AE17BF0714F40C94F51DE0E3EE8F5C
:103B5400E889EF8FE2E0F0E0EE87FF875E5FAA85F9
:103B6400E12FEA1B2E2F520F213010F40C94C31DA9
:103B74000E94A2A73197DE015E960E94A6A621505C
:103B8400F3CFE0E0EC87ED87AE85BF851C9714F09A
:103B94000C94DD1D0E94A2A731970E94AFA70F01CC
:103BA400EC85FD853196EC87FD873197DE015196D2
:103BB4000E9426A7E9CFE0E0EE87EF87AE85BF85B8
:103BC4001C9714F00C94F41D0E949DA7EA0FFB1F90
:103BD4000F01EE85FF85DE015E960E9426A70E94F6
:103BE400A2A7ECCF2BC0EA85E11B2E2FEBE0F0E07F
:103BF400EE87FF87E22FAE85BF85F0E0EA17FB076B
:103C040014F00C94171E0E949DA7EA0FFB1F0F01CE
:103C1400EE85FF853197DE0151960E9426A7EE8539
:103C2400FF853197EE87FF87E5CFE22FF0E0DE01D5
:103C34005196EA0FFB1FA889A0835F5FE52FAA8531
:103C4400BB85F0E0EA0FFB1FEA87FB87EBA5E030BA
:103C540011F40C942F1E40E301C040E2EA85FB8579
:103C6400A02FB0E0EA17FB0714F00C946F1EAA858E
:103C7400E02FEA1B3E2FEBE0F0E0EE87FF870E9487
:103C84009DA7EA0FFB1FBF010E94B4A70E9474BA4C
:103C9400EA1BFB0BDE0151960E94B9A7EE85FF8556
:103CA4003197EE87FF870E94B4A7AE17BF0714F4BD
:103CB4000C945D1EE4CFE0E0EE87EF870E94B4A78A
:103CC400AE17BF0714F00C946F1E0E949DA7EA0F55
:103CD400FB1F40830E94A2A7F1CFE0E0EE87EF87AD
:103CE400AE85BF851C9714F00C94861EEE85FF8567
:103CF400AFA5B8A9EA0FFB1F0F010E949DA70E9460
:103D040026A70E94A2A7ECCF0E94DEB8E5960895EC
:103D14000E944BA63D854C855B85383110F40C948C
:103D2400941E30E04C3310F40C94991E40E05C3344
:103D340010F40C949E1E50E0E985EE8310E020E020
:103D44001C30E0E02E0714F00C94B11EE12FF22F8A
:103D54000E9460A6E0E0EC931F5F2F4FF1CF0A852D
:103D6400003011F40C94DE1E303011F40C94BF1E9C
:103D74003C3011F40C94BF1E08C0AF81B885E1E358
:103D8400EC931196E2E3EC9316C03C3010F00C94E3
:103D9400CE1E0E94BFA70FC0A32FAC500E94D1A774
:103DA400AF81B885EC93A32FAC500E94D6A7AF8106
:103DB400B8851196EC9302C00E94BFA7AF81B88565
:103DC4001296EAE3EC93A42F0E94D1A7AF81B885A1
:103DD4001396EC93A42F0E94D6A7AF81B8851496AE
:103DE400EC9315E020E0EE81E03011F40C94101F08
:103DF4000E94DBA70E9460A6EAE3EC930E94DBA783
:103E04000E94E0A70E94D1A7DB01EC930E94DBA7EC
:103E14000E94E0A70E94D6A7DB01EC93003011F4C6
:103E24000C94311F0E94DBA70E9460A6E0E2EC9391
:103E34003C3010F00C94251F0E94DBA70E9460A662
:103E4400E1E4EC9306C00E94DBA70E9460A6E0E5D3
:103E5400EC930E94DBA70E9460A6EDE4EC93E1E002
:103E64000E94DEB82E960895BA93AA9326970E94CC
:103E7400D7B8E989EF70E05DE987E989E07FE295E9
:103E8400EF70E05DEA870B891A8928891D3010F0EC
:103E94000C94511F103011F40C94511F01C011E007
:103EA400003210F00C945B1F003011F40C945B1F73
:103EB40001C001E0233310F00C94651F2B3010F483
:103EC4000C94651F01C021E0EE85E03011F00C94E4
:103ED4006E1FEEE2EE830FC0AE85A13011F00C949C
:103EE400761FEFE2EE8307C0AE85A03210F40C9487
:103EF4007D1FEE85EE83A02FEAE00E94C9B93E2F14
:103F0400A02FEAE00E9418BA4E2FA12FEAE00E94E7
:103F1400C9B95E2FA12FEAE00E9418BAEB870E946C
:103F2400E7A7E8870E94ECA7EF83305D405D505D12
:103F3400EB85E05DEB870E948DA6EF85E03011F004
:103F44000C94AF1F0E94F1A7EC85FD855383EB858C
:103F54000E94FDA70E9402A84DC0E13011F00C940C
:103F6400BC1F0E941CA8EC85FD85338344830E94FA
:103F740002A840C0E23011F00C94CD1F0E942AA880
:103F8400EC85FD855583EB850E943FA83087EC8541
:103F9400FD8541872FC0E33011F00C94DA1F0E9495
:103FA400F1A70E944BA80E9452A80E9459A822C0BF
:103FB400E43011F00C94E91F0E941CA80E944BA845
:103FC4000E9452A83087EC85FD85418713C0E530F7
:103FD40011F00C94FC1F0E942AA8EC85FD85358302
:103FE4004683EE81AC85BD851796EC93EC85FD8503
:103FF4000E9459A8AC85BD851A96E0E0EC930E9416
:10400400DEB8649608950E94D0A4A885B9850E945C
:10401400171A0E9460A8A030E1E0BE0710F40C94C7
:104024001720EFEFF0E0EE83FF830E9465A80E9463
:10403400E31A5E2F00E010E00E946AA810F00C94CE
:104044006A200E94ABA60E946FA86BBFE691EA1794
:1040540011F00C946720E52FF0E0E00FF11FDF0171
:10406400EE81FF81EA17FB0710F00C943E20E0E09C
:104074000E94DEB82E96089520E030E040E0451717
:1040840010F00C945B20E42FF0E0E00FF11FA88502
:10409400B985AE0FBF1F0C90E42F0E9465A80E9443
:1040A40074A8E01511F40C94592021E030E04F5F1E
:1040B400E6CF022E032A11F00C946720E02FE40FC0
:1040C4005E2F0E94DEB82E9608950F5F1F4FB4CF67
:1040D400E0E00E94DEB82E9608950E94DAB82A2FF6
:1040E400022F02950F700F70AAE00A9F002DE22F95
:1040F400EF701E2F010F0E94BFA408950E94D9B82B
:104104003A2F032FA02FEAE00E94C9B91E2F12955F
:10411400107FA02FEAE00E9418BA2E2F120FE12F71
:104124000E94E0B8249608950A930A2F003310F4ED
:104134000C94A1200A3310F00C94A12001C003C0F8
:10414400E1E009910895E0E0099108950991089545
:104154000A930A2F0E949620E03011F40C94B620A2
:10416400E02FE05309910895E0E009910895099141
:1041740008950E94D7B84A2F5E81F52FE0E08F01A1
:104184000070E42FF0E0F0709F01022B132BF80174
:104194000E94DEB82796089528970E94D9B80A2F5E
:1041A4001C852D853E85E32F0E947CA80E9484A84F
:1041B4000E9489A80E948EA8E22F0E947CA80E94D7
:1041C40092A8E12F0E947CA80E9492A8E02F0E944E
:1041D4007CA8EC83FD836E837F830E9489A80E9460
:1041E400FDB80E9484A8E885F9856A857B850E94CC
:1041F400E0B82F9608950E94D9B82A2F3C81E22F67
:10420400E0531E2FE32FE0530E2FAAE00A9F002D48
:10421400010FE02F0E94E0B825960895BA93AA935F
:104224002B970E94D7B8A989BA890E94171A1E2F02
:10423400E989FA890E949FA8A6E0B0E00E94061BC3
:1042440010E0E0E0E88B0E94A6A8A03310F40C94E0
:1042540032210E94A6A8AA3310F00C94322102C085
:10426400E1E0E88BE889E03011F00C943A211F5F1B
:10427400153010F00C944421A889A03011F00C944E
:10428400442101C001C0DFCF163010F00C944F213F
:10429400103011F40C944F2104C00E94E8A46396DA
:1042A4000895153011F00C946B21E989FA89E481A1
:1042B400E88BA989BA8913965C91A989BA8912965F
:1042C4004C91A989BA8911963C91A989BA892C91F2
:1042D40047C0143011F00C948021E989FA89E381F4
:1042E400E88BA989BA8912965C91A989BA89119631
:1042F4004C91A989BA893C9120E332C0133011F062
:104304000C949221E989FA89E281E88BA989BA8916
:1043140011965C91A989BA894C9130E320E320C0BD
:10432400123011F00C94A121E989FA89E181E88B1A
:10433400A989BA895C9140E330E320E311C01130CC
:1043440011F00C94AE21A989BA89EC91E88B50E361
:1043540040E330E320E304C00E94E8A46396089598
:10436400E22FE0530E2F0A3010F40C94BA2100E02F
:104374000E94ADA8A0E1B7E20E94B2A8EE83FF8339
:10438400E32FE0530E2F0A3010F40C94CA2100E0FE
:104394000E94ADA8A8EEB3E00E94B2A80E9435A77F
:1043A400EE83FF83E42FE0530E2F0A3010F40C94B5
:1043B400DC2100E00E94B7A8E4E60E94BEA8EE83D8
:1043C400FF83E52FE0530E2F0A3010F40C94EB21F9
:1043D40000E00E94B7A8EAE00E94BEA8EE83FF8333
:1043E400E889E0530E2F0A3010F40C94FA2100E00F
:1043F4000E94ADA80E9435A7EE83FF830E94DEB819
:1044040063960895BA93AA932A970E94D7B85A89B3
:104414000B891C8930E0E52FE1502E2F283010F451
:104424000C94152227E0422FE22F2150F0E00E9445
:10443400D8A6E02FEF70EC93F8010E9463B98F01C6
:104444003F5F341710F00C942822EECFE22F0E9425
:10445400C3A800834F5FE42FF0E00E94D8A6E0E0F9
:10446400EC9330E00E94C9A8AC91AA3010F40C94EB
:1044740040220E94C9A8EC91E95FEC93E32FA8893C
:10448400B9890E94CCA80E94C9A80E945CA73F5F7A
:10449400341710F00C944F22E5CFA889B989EE2780
:1044A400A30FBE1FEC930E94DEB8659608950E9488
:1044B400D9B88D012C813D810217130710F00C949B
:1044C4006522F80101C0F9010E94E0B8269608951A
:1044D4000E94D1A811F00C947F22E02FE37011F414
:1044E4000C947922ECE11981088123960895EDE179
:1044F400198108812396089527C0113011F40C9472
:104504009C22133011F40C949C22153011F40C9459
:104514009C22173011F40C949C22183011F40C9442
:104524009C221A3011F40C949C221C3011F40C942B
:104534009C2205C0EFE11981088123960895EEE1DC
:104544001981088123960895198108812396089575
:10455400AA9321970E94D7A8498528853F812030B6
:1045640011F40C94C6222D3010F00C94C622303075
:1045740011F40C94C622303210F00C94C622443646
:1045840010F00C94C62204C00E94E8A42A96089550
:1045940051E0223010F40C94DA225A93A42F0E9492
:1045A4006A22EE83F0E00E0F1F1F21505F5FF1CFF0
:1045B400E32F0E94DCA80E94DEB82A9608950A938D
:1045C4000A2FE02FE37011F00C94EB22E1E0099143
:1045D4000895E0E009910895AA931A930A930A8131
:1045E400102FE02FEC5F1E1710F00C940523E12F21
:1045F400E37011F00C940323E12F198108812396B1
:1046040008951F5FEECF1981088123960895AA9318
:104614001A930A930A81043010F00C941623E0E0F4
:104624001981088123960895E02FE37011F00C940A
:104634002023E02F19810881239608950450102F18
:10464400E02FEC5F1E1710F00C943423E12FE3707D
:1046540011F00C943223E12F1981088123960895D7
:104664001F5FEECF1981088123960895AA931A93A8
:104674000A931B81EB81E1500E2FA8E10A9F002DC4
:10468400EA810E0FE02F19810881249608950E9473
:104694003BA54A93A32F0E9438230E2F11270E9473
:1046A400E1A80E94DFB8279608950E94D9B82A2F5E
:1046B4003C81E32FE1500E2F11270E94E9A80E94AC
:1046C400E0B8259608950E943BA54A93A32F0E9423
:1046D40057238F010E94E1A80E94DFB8279608950E
:1046E4000E94D7B82A2F3E814F8158855A934A9306
:1046F400A32F0E94AA228F01015010400E94E9A812
:104704000E94DEB82996089524970E94D8B80A2FEB
:1047140019852A853B854C854A933A932A93A12F80
:104724000E947223662777270E9433A53197604041
:1047340070400E9433A50E94F1A80E941CA50E940B
:10474400F8A80E9433A50E94DFB82D960895AA9375
:104754000E94D9B82D813E810D811E81EC81E0300B
:1047640011F40C94BC23012F1127E02F0E94E0B810
:1047740027960895E02F0E94E0B8279608950E9496
:10478400E0B827960895AA9324970E942EA50E9424
:1047940001A9EC81E03011F00C94D323E88129962F
:1047A40008950E9404A9A13011F00C94DC23E8813F
:1047B400299608950E9404A9A23011F00C94E523CF
:1047C400E881299608950E9460BAE8E00E9443B9FE
:1047D4000E9401A9E881299608950E94D8B84A2F19
:1047E400242F332700240216030614F00C94FC2310
:1047F4002150304000E010E00217130714F00C942D
:104804001B24F801AD81BE81AE0FBF1F0C90319601
:10481400AD81BE81AE0FBF1FEC91E01511F40C9475
:104824001824E0E00E94DFB8279608950F5F1F4F19
:10483400E3CFE1E00E94DFB8279608950E94DAB83A
:104844001A2F2B81A22F0E949620E03011F00C9495
:104854003024EFEF0E94E1B824960895A12F0E941E
:104864009620E03011F40C944324A22F0E94AA2035
:104874000E2FAAE00A9F002DA12F0E94AA200E0F3E
:1048840004C0A22F0E94AA200E2FE02F0E94E1B89C
:1048940024960895AA930E94D8B83D81AE81BF8121
:1048A4000E94171A2E2FE31B1E2F112311F00C94B4
:1048B4006024E1E00E94DFB82896089500E0011723
:1048C40010F00C947B24E32FE00F4E2F421710F0CE
:1048D4000C947924E02FAE81BF810E94CCA8AE81D4
:1048E400BF81EE27A40FBE1FEC91D001EC930F5FA4
:1048F400E6CF012F021710F00C948924AE81BF81FA
:10490400EE27A00FBE1FE0E2EC930F5FF3CFE0E0D1
:104914000E94DFB82896089524970E940DA92AE0E2
:1049240010E01A3010F00C94A524A32FB42FEE2716
:10493400A10FBE1F0E9412A911F00C94A324212FD1
:1049440002C01F5FEECF213010F40C94AE242B3044
:1049540010F00C94AE2404C00E9417A9299608955F
:1049640010E0E0E0ED83EE83EF83E8870E942EA55C
:10497400AAE0B0E080E090E00E9499B90E941CA5F2
:10498400E12F1F5FF0E0E30FF41FA0810E94AA2033
:104994000E2F0E94F8A80E941CA5121710F00C9468
:1049A400D424E4CF0E942EA50E94DFB8299608954E
:1049B4000E94D9B88D012C813D811A930A930E94DB
:1049C4001EA9E32FE13011F00C94FE24213011F0E4
:1049D4000C94F324E6EFF0E060E070E00E9424A978
:1049E4000AC0223011F00C94FD24EDEFF0E060E0F9
:1049F40070E00E9424A99BC0E23011F00C941825A9
:104A0400213011F00C940D25E4E0F1E060E070E059
:104A14000E9424A90AC0223011F00C941725EDE05D
:104A2400F1E060E070E00E9424A981C0E33011F05D
:104A34000C943225213011F00C942725E5E1F1E0A6
:104A440060E070E00E9424A90AC0223011F00C94A6
:104A54003125EEE1F1E060E070E00E9424A967C036
:104A6400E43011F00C944C25213011F00C944125C4
:104A7400E8E2F1E060E070E00E9424A90AC022307C
:104A840011F00C944B25E3E3F1E060E070E00E9448
:104A940024A94DC0E53011F00C946625213011F0A5
:104AA4000C945B25ECE3F1E060E070E00E9424A943
:104AB4000AC0223011F00C946525E4E4F1E060E0D2
:104AC40070E00E9424A933C0E63011F00C948025D4
:104AD400213011F00C947525EBE4F1E060E070E016
:104AE4000E9424A90AC0223011F00C947F25E3E52A
:104AF400F1E060E070E00E9424A919C0E73011F0F1
:104B04000C949925213011F00C948F25ECE5F1E0FB
:104B140060E070E00E9424A90AC0223011F00C94D5
:104B24009925E4E6F1E060E070E00E9424A90E9487
:104B3400E0B826960895759A749A769A779AE091D1
:104B44000401E068E09304015D9A559A5D985F9AC8
:104B5400579A5F980895E0E00895E0E0E1B9E2B97A
:104B6400E4B9E5B9E7B9E8B9EAB9EBB9EDB9EEB931
:104B7400E0BBE1BBE3BBE4BBE0930101E0930201D2
:104B8400E4E1E0930401E0930501E0E0E093070130
:104B9400E0930801E0930A01E0930B0108950A935E
:104BA4000A2F00FF03C05D9A559A01C05D980991D0
:104BB40008950A930A2F00FF03C05F9A579A01C011
:104BC4005F98099108950A930A2F6B9A003011F4A3
:104BD4000C94EE25739A01C0739809910895639B10
:104BE40002C0E1E00895E0E008950E9429A9E86088
:104BF400E0930101003011F40C940626E0910201C7
:104C0400E860E093020105C0E0910201E77FE093D0
:104C14000201099108956F980E942EA9679B02C012
:104C2400E0E00895E1E008951A930A9300E010E0AB
:104C3400649901C011E0A49B01C010E0103011F48C
:104C44000C9425260061659901C00062669901C033
:104C54000064679901C00068E02F099119910895D3
:104C64000A930A2F9A9A003011F40C943B26A29AC4
:104C740001C0A298099108950A930A2F003011F4F3
:104C84000C944826A0E00E94322603C0A1E00E94B2
:104C94003226099108959A9B03C0A29B01C001C0CA
:104CA40002C0E1E00895E0E008956E980E942EA904
:104CB400669B02C0E0E00895E1E008950E9429A9FE
:104CC400E061E0930101003011F40C946F26E0914F
:104CD4000201E061E093020105C0E0910201EF7E70
:104CE400E093020109910895E0910001E07111F44B
:104CF4000C947E26E1E00895E0E008950E9432A934
:104D0400E064E0930A01003011F40C948F26E091E2
:104D14000B01E064E0930B0105C0E0910B01EF7B14
:104D2400E0930B0109910895E0910901E07411F4F5
:104D34000C949E26E1E00895E0E008950A930A2F7A
:104D44000E948C14539A003011F40C94AB265B9A95
:104D540001C05B98099108950E948C1452980E9496
:104D64002EA94A9B02C0E1E00895E0E008950E9464
:104D74000A2DE03011F00C94C126E0E00895239848
:104D84000E942EA91B9B02C0E0E00895E1E0089573
:104D940023980E942EA91B9B02C0E1E00895E0E045
:104DA40008950A930A2F249A003011F40C94DC26F7
:104DB4002C9A01C02C98099108950A930A2F229ADB
:104DC400003011F40C94E8262A9A01C02A9809911B
:104DD40008950E9432A9E062E0930A01003011F4C0
:104DE4000C94FA26E0910B01E062E0930B0105C0FC
:104DF400E0910B01EF7DE0930B0109910895E0919F
:104E04000901E07211F40C940927E1E00895E0E04F
:104E140008950A930A2F0E947916E0910101E26035
:104E2400E0930101003011F40C941E27E09102017B
:104E3400E260E093020105C0E0910201ED7FE0939E
:104E44000201099108950E947916E0910101EE7F13
:104E54000E9437A9E0910001E17011F40C94342709
:104E6400E1E00895E0E008950E9429A9E064E09358
:104E74000101003011F40C944527E0910201E06433
:104E8400E093020105C0E0910201EF7BE09302018F
:104E940009910895E0910101EF7D0E9437A9E09105
:104EA4000001E07211F40C945927E0E00895E1E068
:104EB400089538980E942EA9309B02C0E0E008951E
:104EC400E1E008950A930A2F399A003011F40C9402
:104ED4006D27419A01C0419809910895419B02C0F0
:104EE400E1E00895E0E008953A980E942EA9329BEB
:104EF40002C0E1E00895E0E00895E0910101EF7758
:104F04000E9437A9E0910001E07811F40C948C27F9
:104F1400E1E00895E0E008950E947F2708950A9350
:104F24000A2F0E94DC17E0910401E260E09304017F
:104F3400003011F40C94A427E0910501E260E093A1
:104F4400050105C0E0910501ED7FE093050109919C
:104F540008950E94DC17E0910401EE7FE0930401C0
:104F64000E942EA9E0910301E17011F40C94BC2776
:104F7400E1E00895E0E008950A930A2F279A0030AB
:104F840011F40C94C7272F9A01C02F980991089502
:104F94002F9B03C0279B01C001C002C0E1E008951C
:104FA400E0E008950A930A2F9C9A003011F40C94BF
:104FB400DD27A49A01C0A49809910895A49B02C076
:104FC400E0E00895E1E008956C980E942EA9649BA6
:104FD40002C0E0E00895E1E008950A930A2F9B9A45
:104FE400003011F40C94F827A39A01C0A3980991F6
:104FF40008956D98759A0E942EA9659B02C0E0E001
:105004000895E1E008950A930A2F269A003011F4D6
:105014000C940E282E9A01C02E98099108952E9B67
:1050240003C0269B01C001C002C0E1E00895E0E096
:1050340008950A930A2F259A003011F40C94242819
:105044002D9A01C02D98099108951D9B02C0E1E09D
:105054000895E0E008950A930A2F569A003011F05B
:105064000C9436285E9805C0013011F00C943B284E
:105074005E9A099108954E9B02C0E1E00895E0E034
:1050840008950E9432A9E068E0930A01003011F00B
:105094000C945228E0910B01EF77E0930B0109C0C7
:1050A400013011F00C945B28E0910B01E068E0936F
:1050B4000B0109910895E0910901E07811F40C9431
:1050C4006528E1E00895E0E0089554980E942EA92F
:1050D4004C9B02C0E1E00895E0E008950A930A2F92
:1050E4003B9A003011F40C947928439A01C04398F8
:1050F400099108953C980E942EA9349B02C0E1E0D6
:105104000895E0E008950A930A2F003011F00C94FA
:105114008E283D9845980DC0013011F00C949528C7
:105124003D9A459806C0023011F00C949B283D9896
:10513400459A099108953D98459A0E942EA9359B58
:1051440002C0E0E00895E1E008950A930A2F0030D8
:1051540011F00C94B0283E9846980DC0013011F01F
:105164000C94B7283E9A469806C0023011F00C946D
:10517400BD283E98469A099108950A930A2F3E9AAB
:10518400003011F40C94C828469A01C0469809913D
:1051940008953E98469A0E942EA9369B02C0E0E0EC
:1051A4000895E1E008950A930A2F003011F00C9459
:1051B400DE289898A0980DC0013011F00C94E528D1
:1051C400989AA09806C0023011F00C94EB28989895
:1051D400A09A099108950A930A2F989A003011F41D
:1051E4000C94F628A09A01C0A09809910895989863
:1051F400A09A0E942EA9909B02C0E0E00895E1E0ED
:1052040008950A930A2F003011F00C940C299998F0
:10521400A1980DC0013011F00C941329999AA1980A
:1052240006C0023011F00C9419299998A19A099199
:1052340008950A930A2F999A0E942EA9003011F416
:105244000C942629A19A01C0A198099108959998CE
:10525400A19A919B02C0E0E00895E1E008950A93C9
:105264000A2F003011F00C943A290B9813980DC0B2
:10527400013011F00C9441290B9A139806C00230A6
:1052840011F00C9447290B98139A099108950A93E5
:105294000A2F0B9A003011F40C945229139A01C06E
:1052A4001398099108950B98139A0E942EA9039BB1
:1052B40002C0E0E00895E1E008950A930A2F003067
:1052C40011F00C946829099811980DC0013011F05F
:1052D4000C946F29099A119806C0023011F00C94AD
:1052E40075290998119A099108950A930A2F099A20
:1052F400003011F40C948029119A01C0119809917D
:1053040008950998119A0E942EA9019B02C0E0E019
:105314000895E1E008950E9432A9E260E0930A0151
:10532400003011F40C949C29E0910B01E260E093AD
:105334000B0105C0E0910B01ED7FE0930B01099196
:105344000895E0910901E27011F40C94AB29E1E0B5
:105354000895E0E008950E9432A9E460E0930A0110
:10536400013011F00C94BC29E0910B01E460E0934E
:105374000B0105C0E0910B01EB7FE0930B01099158
:105384000895E0910901E47011F40C94CB29E1E053
:105394000895E0E008953D98459A3D98459AE0E0E7
:1053A40008950A930A2F3D98459AE0910A01E06115
:1053B400E0930A01003011F40C94E629E0910B010A
:1053C400E061E0930B0105C0E0910B01EF7EE093F7
:1053D4000B01099108950E9432A9E061E0930A014A
:1053E400003011F40C94FC29E0910B01E061E0938E
:1053F4000B0105C0E0910B01EF7EE0930B010991D5
:1054040008950E9432A9E860E0930A01003011F483
:105414000C94122AE0910B01E860E0930B0105C0A3
:10542400E0910B01E77FE0930B0109910895E0916E
:105434000901E87011F40C94212AE1E00895E0E0F8
:10544400089508950E9432A9E160E0930A010130B1
:1054540011F00C94332AE0910B01E160E0930B010D
:1054640005C0E0910B01EE7FE0930B0109910895D3
:10547400E0910901E17011F40C94422AE1E00895ED
:10548400E0E008950A930A2F829A839A013011F07A
:105494000C944F2A8B988A9A09C0023011F00C940C
:1054A400562A8A988B9A02C08A988B9809910895F3
:1054B4000A930A2FA1E00E94922CA02F0E94442A52
:1054C400099108950A9300E07B9B01C001607A9BD7
:1054D40001C00260E02F099108950A930A2F829A6D
:1054E400003011F40C94782A8A9A01C08A980991A0
:1054F400089583988B9A0E942EA97B9B02C0E1E0B9
:105504000895E0E008950E943AA9E0910701E2605D
:10551400E0930701013011F00C94992AE0910801FD
:10552400E1600E9442A9ED7FE093080115C00230BA
:1055340011F00C94A62AE0910801EE7F0E9442A982
:10554400E260E093080108C0E0910801EE7F0E9448
:1055540042A9ED7FE0930801099108950A9300E0C0
:10556400E0910601E27011F40C94B92A0160E09113
:105574000601E17011F40C94C02A0260E02F099135
:1055840008950E943AA9003011F40C94CF2AE091B6
:105594000801E160E093080105C0E0910801EE7F95
:1055A400E093080109910895E0910701ED7F0E94BD
:1055B40047A9E260E0930801E0910601E27011F46A
:1055C4000C94E62AE1E00895E0E008950E944CA9D5
:1055D400E064E0930701003011F40C94F72AE091A1
:1055E4000801E064E093080105C0E0910801EF7B45
:1055F400E093080109910895E0910801E07411F421
:105604000C94062BE1E00895E0E00895E091070191
:10561400EF770E9447A9E0680E9451A9E091060132
:10562400E07811F40C94182BE1E00895E0E008957B
:10563400E0910701EB7F0E9447A90E9454A911F44D
:105644000C94262BE0E00895E1E00895E091070131
:10565400EB7F0E9447A90E9454A911F40C94342BA7
:10566400E1E00895E0E00895E0910701E77F0E94FA
:1056740047A9E8600E9451A9E0910601E87011F47D
:105684000C94462BE1E00895E0E008950E944CA9B3
:10569400E860E0930701003011F40C94572BE0917B
:1056A4000801E860E093080105C0E0910801E77F84
:1056B400E093080109910895E0910701EF7E0E94AB
:1056C40047A9E0610E9451A9E0910601E07111F43B
:1056D4000C946E2BE0E00895E1E008950E944CA93B
:1056E400E061E0930701003011F40C947F2BE0910A
:1056F4000801E061E093080105C0E0910801EF7E34
:10570400E093080109910895E0910701EF7D0E945B
:1057140047A9E0620E9451A9E0910601E07211F4E8
:105724000C94962BE1E00895E0E008950A930C9818
:10573400149A0E942EA900B104FF03C0E1E009916C
:105744000895E0E0099108950A930D98159A0E942E
:105754002EA900B105FF03C0E1E009910895E0E03E
:10576400099108950A930A2F0D9A003011F40C94AC
:10577400BD2B159A01C01598099108950A93209894
:10578400289A0E942EA903B100FF03C0E0E009910A
:105794000895E1E0099108950A930A2F209A0030B0
:1057A40011F40C94D72B289A01C0289809910895D4
:1057B4000A932198299A0E942EA903B101FF03C0DC
:1057C400E0E009910895E1E0099108950A930A2F10
:1057D400219A003011F40C94F12B299A01C02998D4
:1057E400099108950F98179A0E942EA9079B02C049
:1057F400E0E00895E1E008950E945FA9E068E09385
:105804000401013011F00C940D2CE0910501E068C5
:10581400E093050105C0E0910501EF77E0930501F0
:1058240009910895E0910301E07811F40C941C2C83
:10583400E1E00895E0E008950E945FA9E064E09348
:105844000401003011F40C942D2CE0910501E06466
:10585400E093050105C0E0910501EF7BE0930501AC
:1058640009910895E0910301E07411F40C943C2C27
:10587400E1E00895E0E008950E945FA9E062E0930A
:105884000401003011F40C944D2CE0910501E06208
:10589400E093050105C0E0910501EF7DE09305016A
:1058A40009910895E0910401EF7DE0930401E091F2
:1058B4000501E062E0930501E0910301E07211F457
:1058C4000C94662CE1E00895E0E00895E091030172
:1058D400E07211F40C94702CE1E00895E0E0089576
:1058E4000E945FA9E061E0930401003011F40C947C
:1058F400812CE0910501E061E093050105C0E09190
:105904000501EF7EE093050109910895E0910501F9
:10591400E07111F40C94902CE1E00895E0E0089516
:105924000E945FA9E860E0930401003011F40C9434
:10593400A12CE0910501E860E093050105C0E09128
:105944000501E77FE093050109910895E0910301C2
:10595400E87011F40C94B02CE1E00895E0E00895AF
:105964000E945FA9E460E0930401003011F40C94F8
:10597400C12CE0910501E460E093050105C0E091CC
:105984000501EB7FE093050109910895E09104017D
:10599400EB7FE09304010E942EA9E0910301E470DF
:1059A40011F40C94D72CE1E00895E0E008950A93F3
:1059B4000A2F003011F40C94E12C479A01C0479847
:1059C4003F9A09910895479B02C0E1E00895E0E001
:1059D40008953F9847980E9464A9379B02C0E1E06C
:1059E4000895E0E008956A980E942EA9629B02C07F
:1059F400E1E00895E0E008950E944C2708950A9399
:105A04000A2F0E94D92C099108950E94C82C089548
:105A14009D980E942EA9959B02C0E1E00895E0E0C4
:105A24000895E0910101EB7F0E9437A9E091000104
:105A3400E47011F40C94202DE1E00895E0E0089561
:105A44000A98129A0E942EA9029B02C0E1E00895CE
:105A5400E0E008950A930A2F089A003011F40C9498
:105A6400382DA1E00E94922C109A01C0109809913F
:105A740008950898109A0E942EA9009B02C0E1E0A4
:105A84000895E0E00895A1E00E94922C08950A93FD
:105A94000E940A2D0E2F003011F00C94542DE3E6D1
:105AA400099108950E98169A0E942EA9069B03C088
:105AB400E0E009910895E1E0099108950E98169A9D
:105AC4000E942EA9069B02C0E0E00895E1E008953B
:105AD4000E9468A908950E946FBAA1971A930A9325
:105AE4000E9468A90E946EA9ABA1BCA18DA19EA130
:105AF4000E9474A910F40C94802D10E200E00117A8
:105B040010F00C94952D0E9479A9EA0FFB1F0F0148
:105B1400E02FABA1BCA18DA19EA10E9474A8D001CD
:105B2400EC930F5FECCF0E947EA90E94BF131981F2
:105B34000881A7960895EF9723970E94D9B89D01ED
:105B44000E9468A90E946EA90E9489A90E9474A952
:105B540010F40C94AE2D10E200E0011710F00C9438
:105B6400C12D0E9492A9FF93EF93E02F0E9489A96F
:105B74000E9474A8AF91BF91EC930F5FEECF0E9487
:105B840099A9D9010E94171A1E2F113410F40C94EC
:105B9400CC2D10E400E0011710F00C94D72D0E94D6
:105BA40092A90E94A5A90F5FF6CF0E9499A90E940D
:105BB400E0B8EF962B9608950E94DAB811E020E041
:105BC4002A3010F00C94FC2DA0E00E943226AFE0A5
:105BD4000E94AEA911F40C94F02D10E0A1E00E94F3
:105BE4003226A3E00E94AEA911F00C94FA2D10E025
:105BF4002F5FE6CFE12F0E94E1B823960895EF9737
:105C0400A5970E94B6A90E94BBA90E946912A1E0AF
:105C14000E9460260E94C1A9ACE6B1E080E090E059
:105C24000E946D2DA0E8B1E080E090E00E946D2D0F
:105C34000E94C5A9E1EAF1E060E070E00E94D1A908
:105C44000E940B1CE7EBF1E060E070E00E94D1A938
:105C54000E949D2D0E94C5A9E3ECF1E060E070E094
:105C64000E94D1A90E940B1CE0EDF1E060E070E01D
:105C74000E94D1A90E949D2D0E94C5A9ECEDF1E0DE
:105C840060E070E00E94D1A90E940B1CE9EEF1E0F3
:105C940060E070E00E94D1A90E949D2D0E946A2DAF
:105CA400EF96A5960895AA93EF972F970E94D6A9E9
:105CB40040E00E94DBA9E03011F40C94682EA5EFBB
:105CC400B1E080E090E00E94E0A906C0AFEFB1E04F
:105CD40080E090E00E946D2D0E94E5A9523010F4FE
:105CE4000C947F2E0E94C1A90E94ECA9A3E00E94FB
:105CF400E74E0E94C1A90E94E5A9503011F00C940E
:105D0400BE2EFE01EB5BFF4FE081EA930E94FAA9ED
:105D1400EA93FE01EA5BFF4FE081EA930E94B4A597
:105D2400DE01D4960E948A1EE6E0F2E060E070E0B4
:105D34000E94FFA9FE01E85BFF4FE081EA93FE01A8
:105D4400E85BFF4FE081EA93E0E2EA93FE01E75B60
:105D5400FF4FE081EA930E94B4A5DE01D5960E942C
:105D6400361FE3E1F2E060E070E00E94FFA90E94C8
:105D7400FAA9E093D91106C0A0E2B2E080E090E075
:105D84000E94E0A9A2E00E94394F0E9405AA0E9445
:105D9400BF350E940BAADE01AF5BBF4FAC91A130AF
:105DA40010F40C94DC2EAEE2B2E080E090E00E94AD
:105DB400E0A906C0A2E4B2E080E090E00E946D2D6C
:105DC400A1E00E94DB25A0E00E94D125FE017D9682
:105DD4000E9410AA0E94B44F5E2F503011F40C940C
:105DE400F62E4F5FE1E0EE83E0E0EDA7E3E5F2E0BD
:105DF40060E070E00E946ABADE0191960E949D2DD7
:105E0400E0E0EB8FE4E6F2E060E070E00E946ABA62
:105E1400DE011B960E949D2DA1E00E941C360E946B
:105E24000BAA0E9415AAE03011F00C941B2FE1E09C
:105E3400EE83A1E00E94D125AAE00E94F60EA0E024
:105E44000E944051AAE00E940D0F8F010436E0E049
:105E54001E0710F00C942F2FF2CF0E94F6500E94D0
:105E640043529F010E9443529F010E9443529F014B
:105E74002A5F30402031E7E23E0710F40C94492FAA
:105E84002138EEE33E0710F00C94492F07C0A5E734
:105E9400B2E080E090E00E94E0A90DC03A932A931A
:105EA400DE01AC5BBF4F0E94361CE3E8F2E060E029
:105EB40070E00E941AAA0E9433529F012A50304077
:105EC4002832E0E03E0710F40C946F2F2530E1E017
:105ED4003E0710F00C946F2F07C0A9E9B2E080E0F0
:105EE40090E00E94E0A90FC03A932A930E9421AA4D
:105EF400DE01A85BBF4F0E943119EBEAF2E060E0DB
:105F040070E00E941AAAA1E00E94DB250E942230C0
:105F14000E940BAADE01AF5BBF4FAC91A13010F41D
:105F24000C94A72F0E9415AAF0E0FA93EA93DE01DD
:105F3400AC5BBF4F0E94361CEFEBF2E060E070E018
:105F44000E941AAAE1E0EE8306C0A6EDB2E080E06A
:105F540090E00E946D2DA1E00E943C0FA1E00E9400
:105F6400580F8F01E091D9110E940BAA0E94E5A954
:105F7400503011F00C94C22F0E94FAA90E940BAA6F
:105F84000230E0E01E0710F00C94D52F503011F0D1
:105F94000C94D52F0E9415AAA091D911EA1711F0DB
:105FA4000C94D52F01C001C0D9CF0230E0E01E0708
:105FB40010F40C94E42FA8EEB2E080E090E00E948C
:105FC400E0A919C0503011F40C94EF2FA8EFB2E0FF
:105FD40080E090E00E94E0A90EC00E9415AAA09162
:105FE400D911EA1711F40C94FD2FA6E0B3E080E078
:105FF40090E00E946D2DEE81E03011F00C94093098
:10600400A5E1B3E080E090E00E946D2D06C0A5E21A
:10601400B3E080E090E00E946D2DEE810E94DEB836
:10602400EF96669608950A930A2F003011F00C94A7
:106034001E300E9405AA02C00E9429AA099108954F
:106044000E94DAB80E940D26E093DA11A1E00E94C2
:106054003C0F0E9429AA0E94F52CE03011F00C9408
:1060640036300E942FAA08950E940A2DE03011F0C4
:106074000C943F300E9434AA08950E94132DE030FE
:1060840011F00C944A30E3E00E94E1B8239608959D
:10609400A0E00E9439AA11F40C945530E4E00E9467
:1060A400E1B823960895A1E00E9439AA11F00C9456
:1060B4006030E5E00E94E1B823960895A1E00E94D3
:1060C4006026A0E00E94A026A0E00E9480260E94F4
:1060D4005F350E9441AA11F40C947530EBE00E94E4
:1060E400E1B8239608950E944BAA11F00C947F30D6
:1060F400ECE00E94E1B823960895A1E00E94802676
:106104000E9441AA11F40C948C30EDE00E94E1B895
:10611400239608950E944BAA11F00C949630EEE059
:106124000E94E1B8239608950E9479160E9455AA08
:10613400A0E00E945BAAA0E00E9462AA11F40C9461
:10614400A830EFE00E94E1B823960895A1E00E94F0
:1061540062AA11F00C94B330E0E10E94E1B82396F6
:106164000895A0E00E94EB26A1E00E945BAA0E9491
:1061740025270E2F003011F40C94C530E1E10E9464
:10618400E1B823960895A1E00E9462AA11F00C944C
:10619400D030E2E10E94E1B8239608950E946BAAF0
:1061A4000E9470AA11F00C94DC30E3E10E94E1B883
:1061B40023960895A0E00E9470AA11F40C94E7308D
:1061C400E3E10E94E1B823960895A2E00E94A72883
:1061D4000E94542CA1E00E9436270E94C1A90E946B
:1061E400DC17A0E00E94BE27A1E00E9470280E9454
:1061F40079AA0E9480AA11F40C940531E4E10E946A
:10620400E1B8239608950E9485AA0E9480AA11F0FD
:106214000C941131E5E10E94E1B8239608950E949F
:10622400CB280E2F003011F00C941D31E6E10E94B2
:10623400E1B823960895A0E00E943627A0E00E94CA
:1062440070280E94C1A90E948AAA0E9480AA11F003
:106254000C943131E7E10E94E1B8239608950E943D
:10626400CB280E2F003011F40C943D31E8E10E944C
:10627400E1B823960895A0E00E946427A4E1B0E069
:106284000E947E0E0E948FAA11F40C944E31E9E113
:106294000E94E1B823960895A1E00E9464270E9419
:1062A4005F350E948FAA11F00C945D31EAE10E94DF
:1062B400E1B823960895A0E00E9464270E9494AA5E
:1062C4000E945B270E2F003011F00C946E31EBE12D
:1062D4000E94E1B823960895A1E00E9464270E94D9
:1062E400C1A90E945B270E2F003011F40C947F315A
:1062F400ECE10E94E1B823960895A0E00E9464278F
:106304000E94EB2C0E9498AAA1E00E9470280E948F
:1063140098AA0E947C280E2F003011F00C9497311B
:10632400EDE10E94E1B823960895A0E00E94702850
:106334000E945F350E9494AA0E947C280E2F003090
:1063440011F40C94AA31EEE10E94E1B82396089569
:106354000E946BAA0E94722CA0E00E94D4270E9483
:10636400542C0E949CAAA1E00E94A3AA11F40C94AC
:10637400C031EFE10E94E1B823960895A0E00E94A5
:10638400A3AA11F00C94CB31E0E20E94E1B8239669
:1063940008950E9485AA0E94A8AA11F00C94D731EE
:1063A400E1E20E94E1B8239608950E948AAA0E941D
:1063B400A8AA11F40C94E331E2E20E94E1B8239616
:1063C4000895A0E00E94EF270E945F350E94A8AACA
:1063D40011F40C94F231E3E20E94E1B8239608959B
:1063E4000E949CAA0E94C1A9A0E00E94ADAA11F437
:1063F4000C940132E4E20E94E1B823960895A1E0EE
:106404000E94ADAA11F00C940C32E5E20E94E1B8AE
:10641400239608950E94B6AAA0E00E94D4270E9461
:1064240094AA0E94EB2C0E2F003011F00C941F3212
:10643400E6E20E94E1B823960895A1E00E94D427E1
:106444000E94BDAA0E94EB2C0E2F003011F40C9474
:106454003032E7E20E94E1B823960895A0E00E945A
:10646400D427A1E00E94EF27A0E00E94BE27A0E06D
:106474000E947028A2E00E94D5280E9494AA0E943B
:1064840085AA0E94A8AA11F00C944D32E8E20E9459
:10649400E1B8239608950E948AAA0E94A8AA11F43A
:1064A4000C945932E9E20E94E1B8239608950E94BF
:1064B400F9280E2F003011F40C946532EAE20E94A0
:1064C400E1B8239608950E94B6AA0E9494AA0E9455
:1064D40085AA0E94A8AA11F00C947532EBE20E94DE
:1064E400E1B8239608950E948AAA0E94A8AA11F4EA
:1064F4000C948132ECE20E94E1B8239608950E9444
:10650400F9280E2F003011F00C948D32EDE20E9428
:10651400E1B823960895A0E00E9470280E9494AAEE
:10652400A0E00E9403290E9429290E2F0E94C0AADC
:106534000E94ED29A1E00E94242A0E94BDAA0E9483
:10654400CEAA11F00C94AB32EEE20E94E1B823968D
:106554000895A0E00E94242A0E94BDAA0E94CEAA07
:1065640011F40C94BA32EFE20E94E1B82396089534
:10657400A1E00E948D290E94BDAA0E94CEAA11F01A
:106584000C94C932E0E30E94E1B823960895A0E098
:106594000E948D290E94BDAA0E94CEAA11F40C94D7
:1065A400D832E1E30E94E1B823960895A1E00E9465
:1065B400AD290E94BDAA0E94CEAA11F00C94E73224
:1065C400E2E30E94E1B823960895A0E00E94AD2979
:1065D4000E94BDAA0E94CEAA11F40C94F632E3E301
:1065E4000E94E1B823960895A1E00E94032A0E9424
:1065F400BDAA0E94CEAA11F00C940533E4E30E94D4
:10660400E1B823960895A0E00E94032A0E94BDAA3F
:106614000E94CEAA11F40C941433E5E30E94E1B86D
:1066240023960895A1E00E94ED290E9464A90E9486
:106634005F350E94CEAA11F00C942533E6E30E9444
:10664400E1B823960895A0E00E94ED290E9464A970
:106654000E94CEAA11F40C943433E7E30E94E1B80B
:1066640023960895A0E00E948528A1E00E942D2889
:106674000E9498AA0E949D280E2F003011F40C94B9
:106684004833E8E30E94E1B823960895A0E00E940D
:106694002D280E9498AA0E949D280E2F003011F0E8
:1066A4000C945933E9E30E94E1B823960895A1E0DC
:1066B4000E9443280E9494AA0E9467280E2F00304B
:1066C40011F00C946A33EAE30E94E1B8239608952A
:1066D4000E948AAA0E9480AA11F00C947633EBE3FC
:1066E4000E94E1B8239608950E9485AA0E9480AA78
:1066F40011F40C948233ECE30E94E1B823960895DC
:10670400A0E00E9443280E94C1A90E945F350E9414
:1067140067280E2F003011F40C949533EDE30E949A
:10672400E1B8239608950E948AAA0E9480AA11F0D3
:106734000C94A133EEE30E94E1B8239608950E94DD
:1067440085AA0E9480AA11F00C94AD33EFE30E9455
:10675400E1B823960895A1E00E94D3AA11F00C9405
:10676400B833E0E40E94E1B823960895A0E00E94C3
:10677400D3AA11F40C94C333E1E40E94E1B8239644
:106784000895A1E00E94DCAA11F00C94CE33E2E457
:106794000E94E1B823960895A0E00E94DCAA11F4B7
:1067A4000C94D933E3E40E94E1B823960895A1E060
:1067B4000E94E5AA11F40C94E433E4E40E94E1B8E5
:1067C40023960895A0E00E94E5AA11F00C94EF33FB
:1067D400E5E40E94E1B823960895A1E00E94EEAAA0
:1067E40011F00C94FA33E6E40E94E1B8239608957C
:1067F400A0E00E94EEAA11F40C940534E7E40E9490
:10680400E1B823960895A1E00E94F7AA11F00C9430
:106814001034E8E40E94E1B823960895A0E00E94B1
:10682400F7AA11F40C941B34E9E40E94E1B823960E
:106834000895A1E00E9400AB11F00C942634EAE420
:106844000E94E1B823960895A0E00E9400AB11F4E1
:106854000C943134EBE40E94E1B823960895A1E04E
:106864000E9409AB11F00C943C34ECE40E94E1B8B2
:1068740023960895A0E00E9409AB11F40C944734C8
:10688400EDE40E94E1B823960895A1E00E9412ABC2
:1068940011F00C945234EEE40E94E1B8239608956A
:1068A400A0E00E9412AB11F40C945D34EFE40E945A
:1068B400E1B823960895A1E00E941BAB11F40C9457
:1068C4006834E0E50E94E1B823960895A0E00E94B0
:1068D4001BAB11F00C947334E1E50E94E1B82396EC
:1068E4000895A1E00E9424AB11F40C947E34E2E5F7
:1068F4000E94E1B823960895A0E00E9424AB11F011
:106904000C948934E3E50E94E1B8239608950E942B
:10691400542C0E9479AA0E94542C0E2F003011F49A
:106924000C949934E4E50E94E1B8239608950E94FA
:1069340085AA0E94542C0E2F003011F00C94A73419
:10694400E5E50E94E1B823960895A1E00E942DABED
:1069540011F00C94B234E6E50E94E1B82396089550
:10696400A0E00E942DAB11F40C94BD34E7E50E9425
:10697400E1B823960895A0E00E94D4270E9436AB84
:1069840011F40C94CA34E8E50E94E1B82396089502
:106994000E9436AB11F40C94D434E9E50E94E1B8BA
:1069A40023960895A1E00E946026A1E00E9440ABD6
:1069B40011F00C94E234EAE50E94E1B823960895BC
:1069C400A0E00E9440AB11F40C94ED34EBE50E947E
:1069D400E1B823960895A0E00E941B28A1E00E943C
:1069E40005280E94C1A90E9449AB11F00C94FF3400
:1069F400ECE50E94E1B823960895A0E00E940528E2
:106A04000E94C1A90E9449AB11F40C940E35EDE526
:106A14000E94E1B823960895A0E00E940528A1E011
:106A24000E941B280E94C1A90E9449AB11F00C943A
:106A34002035EEE50E94E1B823960895A0E00E9477
:106A44001B280E94C1A90E9449AB11F40C942F3554
:106A5400EFE50E94E1B823960895A1E00E94580F43
:106A64001E2F2F2F0E940D260E2F1230E0E02E072E
:106A740010F00C944435A091DA110A1711F00C941B
:106A8400443501C001C0E9CF0E940D260E2FA0910C
:106A9400DA110A1711F00C9456351031E0E02E0784
:106AA40010F00C94563501C005C0E0E60E94E1B830
:106AB400239608950E944EAB08950E9453AB089507
:106AC400EF97EF97EF9765970E94D8B84A2F00E0A9
:106AD400242F3327D901E6E00E941BB99F0110E05F
:106AE400103410F00C947D350E9457ABE12FED5F0C
:106AF400EC931F5FF5CF0E945FABDE01AB56BF4F37
:106B04000E942F0D0E945FABDE01A15BBF4F0E946C
:106B14006D0D0E9464A90E9466ABE0E0EA93A6E4CE
:106B24000E946BABE0E4F0E00E9410AA0E942F0DDB
:106B340010E0103410F00C94AE350E9457AB0C905A
:106B4400E12FF0E00E944CA7EC91E01511F40C94B5
:106B5400AC3501E01F5FEDCF0E945FABDE01AB56A9
:106B6400BF4F0E946D0D0E9464A9E02F0E94DFB800
:106B7400EF96EF96EF966A9608951A930A931FE399
:106B8400A12F0E9462350E2F003011F40C94CE35E3
:106B9400E1E0099119910895E0E0099119910895AE
:106BA40028970E94D8B84A2F10E0413011F00C9475
:106BB400DC3516EA423011F00C94E1351EEA2CEF74
:106BC4003FEE0E9471ABE1E2F3E465E070E00E9405
:106BD40033A50E947CAB11F00C94FC350E9471AB80
:106BE4000E948EAB11F00C94FC35E2E00E94DFB8F9
:106BF4002D9608952CEF3FE70E9471ABE4E3F2E198
:106C040060E070E00E9433A50E947CAB11F00C940C
:106C140017360E9471AB0E948EAB11F00C9417369C
:106C2400E1E00E94DFB82D960895E0E00E94DFB80D
:106C34002D960895AA930E94DAB82B81A0E00E94B1
:106C4400F725A1E00E94D2350E2F003011F00C94EC
:106C54003436A5E3B3E080E090E00E946D2D0E94FD
:106C640097AB0895013011F00C944736203011F49D
:106C74000C944236A7E4B3E080E090E00E946D2DCE
:106C8400E1E00E94E1B824960895A2E00E94D23582
:106C94001E2F103011F00C945E36203011F40C9439
:106CA4005936ACE5B3E080E090E00E946D2DE2E05F
:106CB4000E94E1B824960895113011F00C946F36B7
:106CC400203011F40C946C36A1E7B3E080E090E03E
:106CD4000E946D2D0E9497AB0895123011F00C9410
:106CE4008236203011F40C947D36A9E8B3E080E0BC
:106CF40090E00E946D2DE3E00E94E1B8249608958F
:106D04000E9497AB0895A0E00E9410180895AFEF79
:106D14000E94101808950A9300E0023010F00C94B9
:106D2400B636ABE20A9FF001E55DFD4E0E949CABD6
:106D3400E45DFD4E0E949CABE35DFD4E0E949CAB66
:106D4400E25DFD4E0E949CABE15DFD4E0E949CAB5A
:106D5400E05DFD4E0E949CABEF5CFD4E0E949CAB3F
:106D64000E94A2AB0F5FD9CFE1E0E03011F40C94A4
:106D7400C036E03011F40C94C03601C006C0E1E026
:106D8400E0932B12EBE7E0932C12E1E0E03011F4F6
:106D94000C94D236E0E0E03011F40C94D23601C009
:106DA40006C0E1E0E0935612EBE0E0935712E0E016
:106DB400E03011F40C94E336E03011F40C94E33633
:106DC40001C006C0E1E0E0938112E3E3E0938212A4
:106DD400E0E0E0932812E0932A12E093291200E005
:106DE400063210F00C94FC36E02F0F5F0E94A7AB24
:106DF4000F5FF6CFE0E0E0932712099108950E9417
:106E0400DAB8E0912912E03011F00C940C370E94AA
:106E1400B3AB08950E94DB38E03011F00C941537C1
:106E24000E94B3AB0895E0912A12E03011F00C9463
:106E34003A37E0E0E0938212E09381120E947F39B6
:106E44000E2F003011F40C943A370E94BD39A091F2
:106E540028120E94443A1E2F103011F00C94363739
:106E6400E1E0E0932A1204C020E00E944EAB0895B2
:106E7400A0912A12A13011F00C9488370E940A3B89
:106E84000E2F013011F00C9456370E94BCAB0E94B7
:106E9400C5AB0E94CAAB0E94D0AB0E94D5ABEE5CDE
:106EA400FD4EA1E0A0831FC0023011F00C946437A2
:106EB400E2E0E0932A12A0EAB3E080E090E00E94CE
:106EC400609511C0033011F00C946C37E3E0E0934B
:106ED4002A1209C0E2E0E0932A12ACEAB3E080E0AF
:106EE40090E00E946095033011F40C94873720E001
:106EF400263210F00C948437E22F2F5F0E94A7AB48
:106F04002F5FF6CFE0E0E093271284C0A0912A120D
:106F1400A23011F00C94C737E0918212EF5FE09336
:106F24008212A0918212A33010F40C94B3370E9401
:106F3400CAABEE5CFD4EA2E0A0830E94CAAB0E94E5
:106F4400D0AB0E94D5ABE15DFD4EA0E0A083E0E0B4
:106F5400E0932A12ABEBB3E080E090E00E946095EE
:106F640013C0A09128120E94B63A1E2F103011F0BF
:106F74000C94C237E1E0E0932A120E942FAA0895EC
:106F840020E00E944EAB089545C0A0912A12A33080
:106F940011F00C940C38E0918112EF5FE0938112B0
:106FA400A0918112A33010F40C94E6370E94CAAB6E
:106FB400EE5CFD4EA3E0A0830E94CAAB0E94C5AB69
:106FC4000E94BCAB0E94DAAB0E94D2390E2F003073
:106FD40011F40C94F137E1E0E0932A120DC0A09172
:106FE40028120E94183A0E94CAABEE5CFD4EA4E03F
:106FF400A083E0E0E0932A1220E0263210F00C9403
:107004000938E22F2F5F0E94A7AB2F5FF6CFE0E095
:10701400E09327120E942FAA0895A1E00E949127CD
:10702400AEE6B0E00E947E0EA0E00E949127089593
:107034000A930E94132D0E2F003011F40C9429385A
:10704400E0912912E03011F40C94293801C003C0F6
:10705400E1E009910895E0E009910895A0E00E941B
:10706400EF27A0E00E94D4270E94DC17E0E0E09321
:107074002912A7ECB3E080E090E00E9460950895A7
:10708400A0E00E94BE270E946BAA0E94722CA1E07D
:107094000E94D4270E94B6A9E4E00E94DFAB0E94BC
:1070A40052170E94E017E1E0E0932912AFECB3E03D
:1070B40080E090E00E946095E1E008950A930A2F31
:1070C400013011F00C946A38A1E00E94D42715C055
:1070D400023011F00C947C38A1E00E94D4270E9465
:1070E40064A9A0E00E94D4270E9464A9A1E00E94A0
:1070F400D42703C0A0E00E94D427099108950E94D8
:10710400BAA4A0912712A63210F00C949438E091FE
:107114002712EF5FE09327120E94E4ABEA0FFB1FF4
:10712400108321831030E1E02E0714F40C94A1386D
:10713400A0912712A13011F00C94A13801C003C012
:10714400009127120F5F0E94E1B8239608950E94D0
:10715400D1A810F00C94D738003011F40C94C03836
:10716400ABE21A9FF001E35DFD4EA1E0A083A6ED22
:10717400B3E080E090E00E94609517C0ABE21A9FF4
:10718400F001E35DFD4E0E94EBAB0E94DAAB0E947E
:10719400F1AB0E94EBAB0E94C5AB0E94F7ABA8EE2B
:1071A400B3E080E090E00E94609519810881239605
:1071B40008950A9300E0023010F00C94EE38ABE22C
:1071C4000A9FF0010E94FBAB11F40C94EC38E1E04F
:1071D400099108950F5FEFCFE0E0099108950E94AF
:1071E400D1A810F00C940039ABE21A9FF001E25DD3
:1071F400FD4E00830E94F1ABA0E0A08319810881B9
:10720400239608950E94D8B88D012D813E814F8127
:107214001A930A93ABE24A9FF001ED5CFD4EFA9398
:10722400EA93A22FBB270E94061B423010F00C9455
:107234002639ABE24A9FF001E25DFD4E30834A9F5E
:10724400F001E05DFD4E20830E94DFB8289608958A
:107254001A930A931A2F123010F00C94423900E05A
:10726400033210F00C944239ABE21A9FF001ED5C4A
:10727400FD4EDF01EE27A00FBE1FEC930F5FF0CF92
:107284000E94F1AB0E94EBAB0E94C5AB0E94F7AB2E
:107294000991199108951A930A931A2FABE21A9F30
:1072A400F001EE5CFD4E00810E94F7ABE02F0991E6
:1072B400199108950A930A2FABE20A9FF001EF5C3B
:1072C400FD4EE081099108950E94DAB88D012B8169
:1072D400ABE22A9FF001ED5CFD4EFA93EA931A9318
:1072E4000A932A9FF001EF5CFD4EA081B0E00E945A
:1072F400061B0E94E1B8249608950E94D9B82FE095
:1073040030E0A9E00E940D0F8F010217130710F05F
:107314000C949139E0E00E94E0B824960895A9E025
:107324000E94F60E20E030E0E0912812EF5FE09337
:107334002812A0912812A23010F40C94A439E0E091
:10734400E09328120E94CAAB0E94FBAB11F40C9488
:10735400B039E1E00E94E0B824960895F90131962D
:107364009F01339710F00C94B839DECFE0E00E940F
:10737400E0B8249608950E9436A50632E0E01E0780
:1073840014F00C94CD39F8010E9400AC0E9407ACB3
:107394000F5F1F4FF2CF0E94E017099119910895D2
:1073A40022970E94D7B8A0912712A13010F40C9410
:1073B400E239E0912712E150F0E0EE83FF8303C04D
:1073C400E0E0EE83EF8300E010E020E030E0EE81C7
:1073D400FF812E173F0710F00C94F839F9010E9431
:1073E40000AC0E940CAC2F5F3F4FF1CF1070EE81C8
:1073F400FF810E9400AC4D915C9150704017510781
:1074040011F40C940F3AE0E0E093DB11E093DC110B
:10741400E1E00E94DEB828960895EE81FF810E9483
:1074240000AC0E9407AC0E9411AC08950E94DAB827
:107434002A2F10912712113010F40C94223A115073
:1074440000E0011710F00C943A3AABE22A9FF001E5
:10745400ED5CFD4EDF01E02F0E94CCA8E02FABEDE8
:10746400B1E1F0E0EE0FFF1F0E9426A70F5FE9CF06
:10747400ABE22A9FF001EF5CFD4E10830E94E1B85D
:10748400239608950E9416AC11F00C944E3AE1E054
:107494000E94DEB8AD9608950E9424AC0E94FBAB16
:1074A40011F00C945A3AE2E00E94DEB8AD960895C9
:1074B4000E9424ACE25DFD4E1081113010F40C9456
:1074C4006D3A0E9424ACE15DFD4E10830E9424AC11
:1074D4000E94DAAB0CC00E9424ACE15DFD4EBF01FA
:1074E4000E9424ACE45DFD4EE081DB01EC930E943C
:1074F40029ACBF010E9424AC0E942CACE05DFD4E7F
:107504002081103011F00C94883A20E0243210F4D9
:107514000C948D3A23E20E8140E050E0E22F0E9469
:1075240032AC14F00C949F3A0E9424AC0E9437AC05
:107534001083010F4F5F5F4FF1CF0E9429AC00838E
:107544000E94C9A80E943DACE32F0E9432AC14F003
:107554000C94B13A0E944DAC4F5F5F4FF5CFE0E021
:107564000E94DEB8AD9608950E9416AC11F00C94FA
:10757400C03AE1E00E94DEB8AD9608950E9424ACC2
:107584000E94FBAB11F00C94CC3AE2E00E94DEB80E
:10759400AD960895A9EFB3E080E090E00E94609575
:1075A4000E9429ACBF010E9424AC0E942CACE05D77
:1075B400FD4E2081243210F40C94E13A23E20E8132
:1075C40040E050E0E22F0E9432AC14F00C94F33A05
:1075D4000E9424AC0E9437AC1083010F4F5F5F4FB1
:1075E400F1CF0E9429AC00830E94C9A80E943DAC3F
:1075F400E32F0E9432AC14F00C94053B0E944DAC76
:107604004F5F5F4FF5CFE0E00E94DEB8AD9608957E
:1076140025970E9454ACE0E0EC830E94D7A8EAEFDF
:10762400F0E0EE83FF830E9453ABA0912712A130B8
:1076340010F40C94453BE885EA1710F00C942B3BAE
:10764400EE81FF81EC59FF4FEE83FF83E091271217
:10765400E88720E030E0E0912712D901F0E0AE178E
:10766400BF0710F00C94453BF9010E9400AC0E9446
:1076740057BAF17011F40C94423BE22FEF5FEA87A2
:107684002F5F3F4FE8CF0F5F1F4F0E946AA810F093
:107694000C94583BA0912712A83210F00C94583B3C
:1076A400AA85A03011F00C94583B01C001C0BBCF97
:1076B400A091DB11B091DC11A030E1E0BE0711F024
:1076C4000C946B3BA0912712A13011F00C946B3BEE
:1076D40001C005C0E1E00E94DEB82B960895AA859A
:1076E400A03011F40C94823B0E946AA810F00C9410
:1076F400823BA0912712A03011F40C94823B05C068
:10770400E2E00E94DEB82B96089540912712552797
:1077140050704150504020E030E02417350710F0FD
:107724000C949E3BF9010E9400ACEC91A985EA0FF0
:10773400E9872F5F3F4FF1CFE09127120E94E4AB1E
:107744000E94F4A4F070A985B0E0EA17FB0711F4D5
:107754000C94B33B0E948936E2E00E94DEB82B967B
:1077640008950E948536E3E00E94DEB82B960895C2
:107774000E94DEB82B9608950A9300E0083010F0BA
:107784000C94D53BA3E00A9FF001ED57FD4E0E94F7
:1077940058ACEC57FD4E0E9458ACEB57FD4EA0E0A0
:1077A400A0830F5FEBCFE0E0E0939B12E0939D1288
:1077B400E3E6E0939C12E0E0E0939F12E0939E12D4
:1077C40009910895E3E6E0939C120E945EACA4E064
:1077D400B4E080E090E00E9460950895AA970E942A
:1077E400D7B8A0919C12A33611F00C94FE3BE0E0B4
:1077F4000E94DEB8E0960895E0919C12E03011F00A
:107804000C94193C0E941A38E03011F40C94123C88
:107814000E9463AC10F40C94113C0E946BAC02C047
:107824000E9471ACE0E00E94DEB8E0960895A09159
:107834009C12A13011F00C94243C0E9477AC0E945D
:107844006BACCCC1A0919C12A23011F00C943A3CC8
:107854000E9463AC10F40C94393CE0E0EA93A8E78E
:107864000E94F138A5E10E94F60E0E946BACB6C1ED
:10787400A0919C12A33011F00C94783C0E9480AC2F
:10788400013011F40C944B3C043011F40C944B3C37
:1078940004C00E946BAC0E9471ACA5E10E940D0F64
:1078A400AF014536E0E05E0710F40C946E3C0E9494
:1078B40085ACA63010F40C946B3C0E945EACE0E006
:1078C400E0939E12E9ECE093AB12E0E0E0939C12AB
:1078D40003C0E1E0E0939C120E941A38E03011F0FA
:1078E4000C94773CE0E0E0939C1278C1A0919C1248
:1078F400A43011F00C948B3CA5E10E940D0FAF0154
:107904004333E0E05E0710F40C948A3C0E946BACB5
:1079140065C1A0919C12A53011F00C94943C0E9476
:107924008DAC5CC1A0919C12A63011F00C942B3D3F
:107934000E9480AC043011F00C94213D0E9493AC61
:10794400153010F00C94BF3C0E9485ACA53610F4A1
:107954000C94B83C0E945EACE0E0E0939E12EAEC2A
:10796400E093AB12E0E0E0939C1206C0A5E10E9414
:10797400F60EE4E0E0939C1262C00E9498ACE4E04E
:10798400F0E0FF93EF93E985EA93AB850E94BB2077
:10799400AF91BF910E9493BAEB85A0E0B0E00E9442
:1079A4009BBAA1E0B0E0EC850E949BBAA2E0B0E0F3
:1079B400ED850E949BBA20E0203110F00C94F03C3D
:1079C400A8E0B0E0E22F0E94CCA8E22FE25FF0E052
:1079D400DE0118960E949EAC2F5FEECFA8E1B0E0C6
:1079E400E1E00E949BBA0E946BACA5E10E94F60EF6
:1079F400E1E0E093AB12A4E0B0E00E94A5ACECE0BF
:107A0400F4E060E070E00E946ABAAA85BB850E9437
:107A1400AAACA0E0B0E00E947FBA3E2FEAE1F4E015
:107A240060E070E00E94AEACA1E0B0E00E947FBADA
:107A34003E2FE6E2F4E060E070E00E94AEAC0E940B
:107A44001A38E03011F00C942A3DE0E0E0939C12E7
:107A5400C5C0A0919C12A73011F00C94343D0E9433
:107A64008DACBCC0A0919C12A83011F00C94723D56
:107A7400E0919E12E03011F40C944D3DE0919F1280
:107A8400E03011F00C944D3DA0919B12A33010F006
:107A94000C944D3D01C003C0E9E0E0939C12E091D9
:107AA4009E12E03011F40C94643DE0919F12E0309A
:107AB40011F40C94643DA0919B12A33010F00C942B
:107AC400643D01C003C0EAE0E0939C120E941A38AE
:107AD400E03011F00C94713DE0E0E0939C127EC024
:107AE400A0919C12A93011F00C94B33DE0919E1228
:107AF400E03011F00C94813DE8E0E0939C12E091B9
:107B04009F12E03011F40C948A3DEAE0E0939C1259
:107B14000E941A38E03011F00C94933DE0E0E093B9
:107B24009C12A0919B12A83010F40C949C3DE8E0A8
:107B3400E0939C120E9480AC043011F00C94B23D8E
:107B44000E9493AC113010F40C94B23D0E9498AC96
:107B54001A93DE0119960E94FA3FE6E0E0939C1224
:107B64003DC0A0919C12AA3011F00C94F03DE0911C
:107B74009E12E03011F00C94C23DE6E0E0939C12BA
:107B8400E0919F12E03011F00C94CB3DE7E0E093DC
:107B94009C120E941A38E03011F00C94D43DE0E0BD
:107BA400E0939C12A0919B12A83010F40C94DD3D3C
:107BB400E6E0E0939C120E9480AC043011F00C9437
:107BC400F03D0E9493AC113010F40C94F03D0E94EF
:107BD40098AC1A93DE0119960E94FA3FE1E00E94E4
:107BE400DEB8E09608950E94D7B8AD01AAE1B0E0EE
:107BF400EF81F8850E9493BAACE1B0E0EE810E9477
:107C04009BBA00E010E00031E0E01E0710F00C9495
:107C1400203EF801DA010E94B6AC2D913C91AEE110
:107C2400B0E0F801EE0FFF1FAE0FBF1FF9010E9475
:107C340093BA21E030E00F5F1F4FE5CFA8E1B0E039
:107C44000E94BBAC0895A4970E94DAB820E02231C8
:107C540010F00C94373EE22FF0E0DE0113960E9400
:107C6400B6AC0E9407AC2F5FF2CFE5E0F0E0E98FFD
:107C7400FA8FEAE0F0E0E98FFA8FE4E1F0E0EB8FCD
:107C8400FC8FE2E3F0E0ED8FFE8FE4E6F0E0EF8FAF
:107C9400F8A3E8ECF0E0E9A3FAA30FEF1FEF1A93BF
:107CA4000A930E94C3AC0E94F53DE0E00E94E1B853
:107CB400A79608950E941A38E03011F00C94673E9C
:107CC400E0E0E0939C12E1E00895E0E00895E091A3
:107CD4009C1208950A930A2FA0919C12A33611F0C6
:107CE4000C94773EE0E0E0939C12A0919C12A630A5
:107CF40010F00C94803EE0E009910895003011F0FA
:107D04000C948B3E0E945EACE0E0E0939E120991DD
:107D140008950E9477ACE1E00991089526971A939B
:107D24000A93A0919C12A33611F00C949C3EE0E0BF
:107D3400E0939C12A0919C12A63010F00C94A73EE4
:107D4400E1E01981088128960895E0919E12E030BF
:107D540011F00C94B23EE2E019810881289608954E
:107D6400AAE1B0E00E947BBA8F01002E012A11F033
:107D74000C94C43EE0E0E0939F12E3E01981088193
:107D840028960895E1E0E0939F120E94C8AC0E94F7
:107D9400DFACDE0115960E940439A5E3B4E080E06F
:107DA40090E00E946095E0E019810881289608958A
:107DB4002697A0919C12A63010F00C94E43EE1E0CA
:107DC400269608950E94E6AC0E94DFACDE0113966D
:107DD4000E940439E0E0E0939F12A4E4B4E080E060
:107DE40090E00E946095E0E026960895BA93AA93E5
:107DF4000E94D7A80034E0E01E0710F00C94083F5E
:107E0400F8010E9410A60F5F1F4FF4CFA8E1B0E065
:107E14000E947FBAAE81BF81EC93E0919C12AE8147
:107E2400BF811196EC93A2E0B0E00E94EFACA4E015
:107E3400B0E00E94F6ACA0E0B0E00E940CADA1E07E
:107E4400B0E00E9413AD0031E0E01E0710F00C9486
:107E5400373FF80137960E9435A70F01E8E0F0E0BC
:107E64000E941CAD0F5F1F4FEECFAAE1B0E00E944D
:107E740024ADACE1B0E00E942EADE0919E12AE8143
:107E8400BF815A96EC93E0919F120E9435AD003168
:107E9400E0E01E0710F00C945C3FAEE1B0E0F801A6
:107EA4000E94B6AC0E943EAD0E9445AD40830F5F78
:107EB4001F4FEDCFE0E40E94DEB828960895E091CC
:107EC4009B1208950E94C4A4E0919B12E03011F02B
:107ED4000C947F3FAD85BE85E0E00E944CADEFEF92
:107EE400EC93AF81B885E0E0EC93AD81BE81EC9377
:107EF400E1E00E94DFB82F960895E0919B12E150D3
:107F0400E0939B120E9454ADE03011F40C94CC3FEA
:107F14000E9454ADAD85BE850E945DADEC57FD4E0B
:107F2400E081A985BA850E945DADEB57FD4E408185
:107F3400AB85BC854C93403110F00C94B73FAEE157
:107F4400B0E0E42FF0E00E94B6AC0E9464AD10F003
:107F54000C94AE3F980109C0A8E0B0E0EE27A40F4E
:107F6400BE1F0E947FBA2E2F3327AF81B8852C9372
:107F7400E32FF070AD81BE810E945DADED57FD4EE3
:107F84000E946BADEC57FD4E0E946BADEB57FD4E5E
:107F9400A0E0A083E0E00E94DFB82F9608951A9332
:107FA4000A930A2F1A81A0919B12A83010F40C9402
:107FB400E03FE1E019810881239608950E9473ADA2
:107FC400ED57FD4EA1E0A0830E9473ADEC57FD4E2A
:107FD40000830E9473ADEB57FD4E1083E0919B121A
:107FE400EF5FE0939B12E0E01981088123960895E6
:107FF400BA93AA93A2970E94D7B84FEF5FEF3AA51E
:108004000E9479ADE8A5F9A50E94BDA6A32FBB27C0
:108014000E94061B00E0E02FF0E00E94D8A6EC913D
:10802400E07F1E2FE02FF0E00E94D8A6EC91EF70C5
:108034002E2F103711F40C942440103811F40C94A2
:10804400244001C0422F103711F00C943040E2E577
:10805400F4E060E070E00E9483AD0AC0103811F0D3
:108064000C943A40E1E6F4E060E070E00E9483ADF5
:10807400103911F40C944340103A11F40C94434019
:1080840007C0522FAFE6B4E080E090E00E94609514
:108094000F5F031710F00C945040BDCF4A93A52FE7
:1080A4000E94D13FE1E00E94DEB8AB9608950A93A6
:1080B40000E00A3010F00C947040A3E00A9FF00135
:1080C400E354FD4E0E9458ACE254FD4E0E9458AC5D
:1080D400E154FD4EA0E0A0830F5FEBCFE0E0E0931E
:1080E400DB12E093DD12E093DC12E093DF12E09305
:1080F400DE1209910895A8970E94D8B8E091DC1285
:10810400E03011F00C949F400E941A38E03011F4D2
:108114000C9494400E948BAD10F40C9493400E94F4
:1081240094AD06C0E0E0E093DD12A5E10E94F60EF6
:10813400E0E00E94DFB8AD960895A091DC12A13072
:1081440011F00C94B040E1E0EA93A8E00E94F13809
:10815400A5E10E94F60E0E9494AD89C1A091DC12A3
:10816400A23011F00C94C3400E948BAD10F40C9417
:10817400C2400E949AAD0E9494ADA5E10E94F60E01
:1081840076C1A091DC12A33011F00C94FD400E9442
:10819400A3AD013011F40C94D440043011F40C94C8
:1081A400D44005C0E0E0E093DD120E9494ADA5E167
:1081B4000E940D0F3E2F4F2F3536E0E04E0710F48E
:1081C4000C94F3400E94A8ADA63010F40C94F04037
:1081D4000E94B0ADE9ECE093AB1203C0E1E0E093A0
:1081E400DC120E941A38E03011F00C94FC40E0E0FC
:1081F400E093DC123CC1A091DC12A43011F00C9489
:108204000B41E1E0EA93A9E00E94F1380E9494ADA9
:108214002EC1A091DC12A53011F00C9486410E946D
:10822400A3AD043011F00C947C410E94B9AD15301B
:1082340010F00C9430410E94A8ADAB3010F40C94B3
:108244002C410E94B0ADEAECE093AB12E0E0E09385
:10825400DC1203C0E4E0E093DC124CC00E94C3AC27
:108264000E946639A0E4B0E0ED810E949BBAE2E48A
:10827400F0E0FF93EF93EE81EA93A8850E94BB2080
:10828400AF91BF910E9493BAE885AEE3B0E00E943B
:108294009BBAAFE3B0E0E9850E949BBAE4E4F0E066
:1082A400FF93EF93EA85EA93AC850E94BB20AF91DC
:1082B400BF910E9493BA20E0203110F00C947241D7
:1082C400A6E4B0E0E22F0E94CCA8E22FE95FF0E040
:1082D4000E944CA7EC91D0010E949BBA2F5FECCF77
:1082E400A6E5B0E0E1E00E949BBA0E9494ADE1E013
:1082F400E093AB120E941A38E03011F00C948541DF
:10830400E0E0E093DC12B3C0A091DC12A63011F0DF
:108314000C94C441E091DE12E03011F40C949F41BE
:10832400E091DF12E03011F00C949F41A091DB1238
:10833400A33010F00C949F4101C003C0E7E0E09328
:10834400DC12E091DE12E03011F40C94B641E091BD
:10835400DF12E03011F40C94B641A091DB12A3308B
:1083640010F00C94B64101C003C0E8E0E093DC12C5
:108374000E941A38E03011F00C94C341E0E0E0931D
:10838400DC1275C0A091DC12A73011F00C94FF41EF
:10839400E091DE12E03011F00C94D341E6E0E0937A
:1083A400DC12E091DF12E03011F40C94DC41E8E0DF
:1083B400E093DC120E941A38E03011F00C94E5418D
:1083C400E0E0E093DC12A091DB12AA3010F40C94EC
:1083D400EE41E6E0E093DC120E94A3AD043011F01C
:1083E4000C94FE410E94B9AD113010F40C94FE417E
:1083F4000E94C3AC0E94BEAD3AC0A091DC12A8306A
:1084040011F00C943942E091DE12E03011F00C943A
:108414000E42E6E0E093DC12E091DF12E03011F06E
:108424000C941742E7E0E093DC120E941A38E03023
:1084340011F00C942042E0E0E093DC12A091DB12F6
:10844400AA3010F40C942942E6E0E093DC120E9476
:10845400A3AD043011F00C9439420E94B9AD11302F
:1084640010F40C9439420E94C3AC0E94BEADE1E00A
:108474000E94DFB8AD9608950E94D7B8AD01A8E573
:10848400B0E0EF81F8850E9493BAAAE5B0E0EE81EE
:108494000E949BBA00E010E00031E0E01E0710F0FB
:1084A4000C946B42ACE5B0E0F8010E94C5AD0F013D
:1084B400F801DA010E94CAADD0010E9493BA21E00A
:1084C40030E0E02FD9010E941BB99F010F5F1F4FBD
:1084D400E3CFA6E5B0E00E94BBAC08950A930A2F4F
:1084E400A091DC12A63010F00C947B42E0E00991DC
:1084F4000895003011F00C9484420E94B0ADE0E085
:10850400099108950E949AADE1E009910895269792
:108514001A930A93A091DC12A63010F00C9497429F
:10852400E1E01981088128960895E091DE12E03097
:1085340011F00C94A242E2E0198108812896089572
:10854400A8E5B0E00E947BBA8F01002E012A11F049
:108554000C94B442E0E0E093DF12E3E01981088177
:1085640028960895E1E0E093DF120E94C8AC0E94CF
:10857400CEADDE0115960E940439E0E01981088130
:10858400289608952697A091DC12A63010F00C943A
:10859400CE42E1E0269608950E94E6AC0E94CEAD5C
:1085A400DE0113960E940439E0E0E093DF12269680
:1085B4000895BA93AA930E94D7A80034E0E01E0756
:1085C40010F00C94EB42F8010E9410A60F5F1F4FAD
:1085D400F4CFA6E5B0E00E947FBAAE81BF81EC93F0
:1085E400E091DC12AE81BF811196EC93A0E4B0E07F
:1085F4000E94EFACA2E4B0E00E94F6ACAEE3B0E0BF
:108604000E940CADAFE3B0E00E9413AD0031E0E096
:108614001E0710F00C941A43F80137960E9435A7F0
:108624000F01E6E4F0E00E941CAD0F5F1F4FEECF98
:10863400A8E5B0E00E9424ADAAE5B0E00E942EAD0A
:10864400E091DE12AE81BF815A96EC93E091DF1285
:108654000E9435AD0031E0E01E0710F00C943F435A
:10866400ACE5B0E0F8010E94B6AC0E943EAD0E94B9
:1086740045AD40830F5F1F4FEDCFA4E4B0E00E94EF
:108684007BBA0E94D5ADAE81BF81DC96EC930E948B
:10869400DBADAE81BF81DD96EC93E0E40E94DEB8F1
:1086A40028960895E091DB1208950E944BA6E0916C
:1086B400DB12E03011F00C947243AF85B889E0E02E
:1086C400EC93AD85BE85EFEF0E944CADE0E0EC93FA
:1086D400AF81B885EC93E1E00E94DEB8619608951D
:1086E400E091DB12E150E093DB120E94E0ADE35431
:1086F400FD4EE081AF85B889EC930E94E0ADE25471
:10870400FD4EE081AB85BC85EC930E94E0ADE15465
:10871400FD4EE081EE83AD85BE85EC93AE81A03144
:1087240010F00C94B643ACE5B0E0F0E00E94B6ACB7
:108734000E9464AD10F00C94A143980115C0A6E406
:10874400B0E0EE81F0E0AE0FBF1F0E947FBA2E2F83
:108754003327AEE3B0E00E947FBA4E2F5527FA01CB
:10876400D9010E9491B99F01A985BA852C93E32F61
:10877400F070AF81B885EC930E94E0ADE354FD4EF8
:10878400A0E0A0830E94E0ADE254FD4EA0E0A083EF
:108794000E94E0ADE154FD4EA0E0A083E0E00E9421
:1087A400DEB8619608950E94E6ADA091DB12AA306E
:1087B40010F40C94E243E1E00E94E1B82596089598
:1087C4000E94E0ADE354FD4E20830E94E0ADE254EC
:1087D400FD4E00830E94E0ADE154FD4E1083E09114
:1087E400DB12EF5FE093DB12E0E00E94E1B8259634
:1087F4000895BA93AA93A3970E94D7B810E02FEFD5
:1088040030E040E05BA50E94ECAD0E94F1ADE9A52B
:10881400FAA5FA93EA930E94F7ADA52FBB270E940D
:10882400061B00E0E02FF0E0DE011796AE0FBF1F3D
:10883400EC91EE83E07811F40C942944EE81E07716
:108844004E2F42954F70EE81EF702E2F2DC0EE818A
:10885400E07411F40C944944EE81E07FE03711F0A8
:108864000C94364413E00FC0EE81E07FE03511F044
:108874000C943E4412E007C0EE81E07FE03411F036
:108884000C94454411E0EE81EF702E2F0DC0EE8163
:10889400E07211F40C944F4407C0EE81E07111F4BE
:1088A4000C94554401C03E810F5F051710F00C94E1
:1088B4006544103011F40C946444303011F40C9479
:1088C400644401C001C001C0ADCF1A932A93A32F01
:1088D4000E94D543E1E00E94DEB8AC960895089565
:1088E400E0E008950E94FCAD0E94F113A1E00E9413
:1088F4006026A0E00E94802608950E94C1A90E94DB
:10890400F24A0E94C1A90E94ED440E94C1A9A5E0B7
:108914000E9437490E94C1A9A5E00E944B490E94C8
:10892400C1A9EDE0EA93E4E0EA93A2E0B0E080E0DC
:1089340090E00E9401AEEDE0EA93E9E00E9404AE0B
:10894400EEE0EA93E3E00E9404AEE2E1EA93E3E0BE
:10895400EA93A6E9B0E080E090E00E946E49E6E97F
:10896400F0E0E093EF12F093F0120E94C1A9E2E16B
:10897400EA93E7E1EA93AEE1B0E080E090E00E94A0
:1089840001AEE2E1EA93E7E2EA93A8EEB3E080E025
:1089940090E00E9401AEE2E1EA93E8E2EA93A4E601
:1089A400B0E080E090E00E9401AEE8E0EA93AAE043
:1089B4000E9485450E94C1A9A0E00E94D8450E945A
:1089C400C1A9A0E00E94C0450E94C1A9A4E6B0E0EC
:1089D4000E94884B08950E940AAE0E9415AE0E9420
:1089E4001BAEE1E4EC930E9420AEE0E00E9423AED3
:1089F400A2E0B0E00E9480150881659608950E9467
:108A04007444A1E20E949014A1E00E94922CA8EC6C
:108A1400B0E00E947E0E0E94B926E03011F40C945E
:108A240017450E947F440E94ED440895A0E00E94EF
:108A3400922C089526970A930A2F033011F00C9470
:108A44003245ADE00E949014AAE00E949014AAE07E
:108A54000E949014AAE00E949014AAE00E9490142C
:108A6400EBE1E983E3E4EA83013011F40C943F453C
:108A7400033011F40C943F4503C0E0E0EB8306C0DF
:108A8400023011F00C944845E1E0EB83E0E0EC8324
:108A94000E9429AE0E942EAE0881279608956497FD
:108AA4000E940DA90E9432AE0E9415AE0E944CA7EE
:108AB400E6E40E9441AE0E9446AE2083E02FF0E03F
:108AC4000E944CA7E0E0EC930E9466AB0E944BAE80
:108AD400089564970E940DA90E9432AE0E9415AEBB
:108AE4000E944CA7ECE50E9441AE0E9446AE208352
:108AF400E02FF0E00E944CA7E0E0EC930E9466AB0C
:108B04000E944BAE089564970E94DAB81A2F2F89F9
:108B140000E02F3110F40C94904520E0163010F44E
:108B24000C949945153110F00C94994501C01AE044
:108B34000E9453AE0E9415AE0E945BAEE0E5EC933A
:108B44000E9453AEEFEF0E9460AEDE0113960E94C6
:108B540065AEDE011396EA0FFB1F10830E946CAE14
:108B64000E946FAEA5E0B0E00E9480152093E01251
:108B74001093E1120E94E1B8689608950E9476AEBF
:108B8400153010F40C94C74510E00E947CAE0E948E
:108B940084AEE7E50E9460AE0E9489AE0E948FAE6B
:108BA4001093E21219810881669608950E9476AEA8
:108BB400183010F40C94DF4510E00E947CAE0E9443
:108BC40084AEE8E40E9460AE0E9489AE0E948FAE3B
:108BD4001093E31219810881669608950E9476AE77
:108BE4000E947CAE0E9484AEE9E50E9460AE0E94C1
:108BF40089AE0E948FAE1093E412198108816696A3
:108C040008950E9476AE123010F40C940A4610E0D7
:108C14000E947CAE0E9484AEEAE40E9460AE0E9490
:108C240089AE0E948FAE1093E51219810881669671
:108C340008950E9476AE123010F40C94224610E08F
:108C44000E947CAE0E9484AEECE40E9460AE0E945E
:108C540089AE0E948FAE1093E61219810881669640
:108C640008950E9476AE123010F40C943A4610E047
:108C74000E947CAE0E9484AEE9E40E9460AE0E9431
:108C840089AE0E948FAE1093E7121981088166960F
:108C940008950E9476AE1C3611F40C946646133681
:108CA40011F40C946646123711F40C9466461C3485
:108CB40011F40C946646133411F40C946646123580
:108CC40011F40C94664601C001C01CE60E947CAEFF
:108CD4000E9484AEE9E60E9460AE0E9489AE0E94C2
:108CE4008FAE1093E81219810881669608950E9448
:108CF40076AE0E947CAE0E9484AEE3E20E9460AE37
:108D04000E9489AE0E948FAE1981088166960895EB
:108D14000E9476AE0E947CAE0E9484AEEDE60E9474
:108D240060AE0E9489AE0E948FAE1981088166965A
:108D34000895AA93EF9769970E94D7B824E630E084
:108D440040E0FE01E25AFF4F5081FE01B896FA93CB
:108D5400EA930E94F1AD0E9479AD5F3110F40C9456
:108D6400B4465EE100E0051710F00C94C6460E947C
:108D740098AEEA0FFB1F0E949DAEE02F0E94C3A88D
:108D84000E949DAE0F5FEFCFDE01AE59BF4FAC9195
:108D9400A03011F00C94D5460E94ABAEA13011F076
:108DA4000C94D54601C001C012E40E94B0AEA030BC
:108DB40011F00C94E4460E94ABAEA03011F00C9478
:108DC400E44601C001C012E60E94B0AEA13011F029
:108DD4000C94F3460E94ABAEA13011F00C94F34610
:108DE40001C001C013E40E94B0AEA13011F00C9494
:108DF40002470E94ABAEA03011F00C94024701C0B0
:108E040001C013E60E94B0AEA23011F00C941147D9
:108E14000E94ABAEA13011F00C94114701C001C007
:108E240014E40E94B0AEA23011F00C9420470E94CA
:108E3400ABAEA03011F00C94204701C001C014E681
:108E44000E94B0AEA33011F00C942F470E94ABAE39
:108E5400A13011F00C942F4701C001C019E40E9405
:108E6400B0AEA33011F00C943E470E94ABAEA030DC
:108E740011F00C943E4701C001C019E60E94B0AE47
:108E8400A43011F00C944D470E94ABAEA13011F008
:108E94000C944D4701C001C015E50E94B0AEA4304A
:108EA40011F00C945C470E94ABAEA03011F00C940E
:108EB4005C4701C001C015E70E94B0AEA53011F0B7
:108EC4000C946B470E94ABAEA13011F00C946B472D
:108ED40001C001C016E50E94B0AEA53011F00C949B
:108EE4007A470E94ABAEA03011F00C947A4701C0CF
:108EF40001C016E7123411F40C948547123611F4AC
:108F04000C9485471DC000E0051710F00C9493479E
:108F14000E94B5AE0F010E9498AE0E9426A70F5F73
:108F2400F3CFEAE2EE830E94B8AEEAE2EC93E52FD7
:108F3400EE5FF0E00E94D8A6E0E0EC935E5FB6C07E
:108F4400133411F40C94AB47133611F40C94AB475F
:108F54000CC0E52FF0E00E94D8A6EFEFEC930E943E
:108F6400B8AEE0E0EC935F5FA1C0143411F40C944C
:108F7400C047143611F40C94C0471DC00E9479AD4B
:108F84000E94BCAE0E94C3AE5CE000E0051710F086
:108F94000C94DC470E9498AE0E94C7AE11F40C9466
:108FA400DA470E94B5AE0F010E9498AE0E9426A730
:108FB4000F5FECCF7BC0193411F40C94E6471936DB
:108FC40011F40C94E6472CC00E94BCAE0E94CAAEB9
:108FD40000E0051710F00C94FF470E9498AE0E9421
:108FE400C7AE11F40C94FD470E94B5AE0F010E9468
:108FF40098AE0E9426A70F5FECCFE0E0EE835F5FA0
:1090040050FF08C0E52FF0E00E94D8A6EFEFEC93E4
:109014005F5F05C00E94B8AEEFEFEC935E5F46C0A1
:10902400153511F40C941B48153711F40C941B4896
:1090340016C00E9479AD0E94BCAE0E94C3AE00E08F
:10904400051710F00C942F480E94B5AE0F010E9432
:1090540098AE0E9426A70F5FF3CF5CE027C01635B9
:1090640011F40C943A48163711F40C943A481EC083
:109074000E9479AD0E94BCAEA7E0B0E00E94F31B51
:1090840057E000E0051710F00C9458480E9498AE81
:109094000E94C7AE11F40C9456480E94B5AE0F015D
:1090A4000E9498AE0E9426A70F5FECCF0E94CEAE1E
:1090B4000E94D3AE0E9415AE0E94D3AEE3E60E9496
:1090C40060AE0E94D9AE1083E02F0F5FF0E0DE01A6
:1090D400A65BBF4F0E9465AE0E94D9AE3083E02FDD
:1090E4000F5FF0E00E94D9AE4083E02FF0E00E94D1
:1090F400D3AEE0E0EC93FE01E65BFF4FFA93EA9314
:10910400A6E0B0E00E9480150E94DFAEA52FBB2729
:109114000E9480150E94DEB8EF96A4960895649785
:109124000E94BAA400E00E9453AE0E9415AE0E94B1
:109134005BAEE3E6EC930E9453AEEDEFEC93012EAD
:10914400022A11F00C94AE48E02F0F5FF0E0DE012C
:1091540013960E94A6A604C00E9453AEE1E3EC93CA
:109164000E946CAE0E946FAEA4E0B0E00E94801535
:109174000E94E1B86796089564970E94BAA400E03B
:109184000E9453AEECE0EC930E946CAE0E946FAE72
:10919400A1E0B0E00E9480150E94E1B867960895AE
:1091A4001A930A931A2F00E0011710F00C94DF4869
:1091B400AAE00E9490140F5FF7CF099119910895C6
:1091C4000E94D9B89D010E94171A8F013A932A93DD
:1091D400D8010E948015AAE00E9490140E94E0B871
:1091E400249608950E946FBA0E9460BA0E94B31533
:1091F40024960895EF97EF9724970A9300E0023896
:1092040010F00C940B490E9420AEE0E0EC930F5F49
:10921400F6CF00E0013610F00C9417490E9420AEFE
:10922400E02FE05EEC930F5FF5CF0E9429AEA0E63D
:10923400B0E00E94801500E0003810F00C94294939
:109244000E9420AEE02FE058EC930F5FF5CF0E9410
:1092540029AEA0E8B0E00E948015AAE00E94901414
:109264000881EF96EF9625960895AA930A93E981CB
:10927400EE0FEE0FEE0F0E2FE1E1EA93E4E0EA9336
:10928400A02FBB27882799270E946E490881229620
:109294000895AA932497E0ECE883E1E0E9830E942F
:1092A40054AC0A93ED81EE0FEE0FEE0F0E2F0E94D9
:1092B400E4AE0E94F8B8A983BA838B839C83E1E16E
:1092C400EA93E5E0EA93AB81BC818D819E810E94A3
:1092D4006E490881269608950E946FBAAF97E0E020
:1092E400E883E9830E9454AC0E94D7B800E020E0F0
:1092F400EDA9FEA96FA978AD0E94ECAEADA9BEA9F7
:109304008FA998ADA935EEE3BE07EFE08E07E0E044
:109314009E0710F40C949349E1E00E94DEB8EB96AA
:1093240008951AADA12FE4E60E94C9B93E2F0E9408
:10933400F1AE4E2F0E94ECA75E2F305D405D505D74
:1093440019ADA12FE4E60E94C9B9EE8B0E94F1AEDB
:10935400ED8B0E94ECA7EC8BEE89E05DEE8BED8942
:10936400E05DED8BEC89E05DEC8B0E9465A80E94CA
:1093740009A50E94EFB9EB8B0E9465A80E9409A57C
:109384000E94F7AEE0E1F7E260E070E00E94EFB91E
:10939400EA8B0E9400AFE0E1F7E260E070E00E9437
:1093A40005AFE8EEF3E060E070E00E94EFB9E98B0E
:1093B4000E9465A8E8EEF3E060E070E00E94F7AE7A
:1093C400E4E6F0E060E070E00E94EFB9E88B0E9410
:1093D40000AFE4E6F0E060E070E00E9405AF0E94B8
:1093E4000AAF0E94EFB9EF870E9465A80E940FAFF1
:1093F400EE87EB89E05DEB8BEA89E05DEA8BE98936
:10940400E05DE98BE889E05DE88BEF85E05DEF875F
:10941400EE85E05DEE870E9414AFAE0FBF1FEEE154
:109424000E9460AE0E941AAFEBE50E9460AE0E94FB
:109434001AAFE2E30E9460AE0E941AAFEAE3EC9333
:10944400313310F40C942B4A0E9414AFEA0FFB1F23
:109454003083413310F00C94344A313310F00C94BF
:10946400344A05C00E9414AFEA0FFB1F40830E94D8
:1094740014AFEA0FFB1F50830E9414AF0E94A1A6F1
:10948400AE89A13310F40C944D4A0E9414AFEA0F34
:10949400FB1FAE89A083AD89A13310F00C94584A08
:1094A400AE89A13310F00C94584A06C00E9414AF40
:1094B400EA0FFB1FAD89A0830E9414AFEA0FFB1FC4
:1094C400AC89A0830E9414AFAE0FBF1FEAE3EC93F4
:1094D400AB89A13310F40C94754A0E9414AFEA0FBF
:1094E400FB1FAB89A083AA89A13310F00C94804A96
:1094F400AB89A13310F00C94804A06C00E9414AFCB
:10950400EA0FFB1FAA89A083A989A13310F00C9448
:10951400964AAA89A13310F00C94964AAB89A133D8
:1095240010F00C94964A06C00E9414AFEA0FFB1F79
:10953400A989A083A889A13310F00C94B14AA98900
:10954400A13310F00C94B14AAA89A13310F00C9401
:10955400B14AAB89A13310F00C94B14A06C00E9401
:1095640014AFEA0FFB1FA889A083AF85A13310F0C5
:109574000C94D14AA889A13310F00C94D14AA9893A
:10958400A13310F00C94D14AAA89A13310F00C94A1
:10959400D14AAB89A13310F00C94D14A06C00E9481
:1095A40014AFEA0FFB1FAF85A0830E9414AFEA0F2C
:1095B400FB1FAE85A0830E9414AFAE0FBF1FEDE565
:1095C400EC93E02FF0E00E941AAFE0E0EC93FE0190
:1095D40077960E941FAFE0E00E94DEB8EB960895F4
:1095E4000E940AAEEEE10E9460AE0E941BAEEBE563
:1095F4000E9460AE0E941BAEE6E30E9460AE0E9431
:109604001BAEEAE30E9460AE0E9425AF0E9429AF20
:10961400E02F0F5FF0E00E9425AF0E9430AFEAE335
:109624000E9460AE0E9425AF0E9430AFEDE50E941B
:1096340023AEA02FBB270E9480150E94CEAE0E94AD
:109644001BAEEEE10E9460AE0E941BAEEBE50E94F1
:1096540060AE0E941BAEE9E30E9460AE0E941BAEA6
:10966400EAE30E9460AE0E9425AF0E9429AFE02F7A
:109674000F5FF0E00E9425AF0E9430AFEAE30E9442
:1096840060AE0E9425AF0E9430AFEDE50E9423AE8C
:10969400A02FBB270E9480150881659608956497C2
:1096A4000E94D7B82A2F3A8D4B8D5C8D00E015E0CF
:1096B400E02F0F5FF0E00E94D8A6EBE1EC930E944C
:1096C40034AF50830E9434AF40830E9434AF308360
:1096D4000E9434AF2083403011F00C94734B12E09D
:1096E4000BC0303011F00C94794B13E005C02030DE
:1096F40011F00C947E4B14E00E94DFAEA12FBB2727
:109704000E9480150E94DEB86D9608951A930A93FC
:109714008D010530E0E01E0710F40C94984B0B3FCC
:10972400E0E01E0710F00C94984B01C00DC0E2E17C
:10973400EA93E3E0EA93D801882799270E946E49C7
:109744000093EF121093F0120991199108956C97F8
:109754000E94D7B800E030E010E00E949D14E0E0E1
:10976400E093EE120E94CEAE0E9437AF0E9415AE77
:109774000E9437AFEBE6EC93E02FF0E00E9437AFA6
:10978400E0E0EC93FE013E960E941FAFADE00E9424
:10979400F60E00E00E9472150E2FADE00E940D0F30
:1097A400AF01003011F00C94DE4B4436E0E05E076C
:1097B40010F00C94DE4B01C001C0ECCF003011F06E
:1097C4000C94EB4BE0E4E093EE120E94DEB8A29618
:1097D40008950E941E150E9460A8199714F40C9411
:1097E400F54B0E943CAFAE81BF81119714F40C94E9
:1097F400024CAE81BF81199714F00C94024C06C040
:109804001F5F1E3110F00C94084C01C001C0A5CF9D
:10981400AE81BF81119714F00C94194C0E949D14D1
:10982400E0E8E093EE120E94DEB8A2960895FE01ED
:109834003E960E9440AF0E9445AFFE013E96FA93C9
:10984400EA93A4E1B0E00E94431500E0063010F072
:109854000C94344CE02FF0E0DE0118960E9449AFDE
:109864000F5FF4CFAE81BF81169714F40C943E4C75
:10987400E5E0F0E0EE83FF8300E0EE81FF81A02FBE
:10988400B0E0AE17BF0714F00C947B4CE02FF0E06F
:109894000E9437AF2C91E22FE07F1E2F17FF03C0E9
:1098A40016FD01C001C004C0E22FEF73E8871FC09A
:1098B400103C11F00C94624CE22FEF70E98717C052
:1098C400103D11F00C946A4CE22FEF70EA870FC040
:1098D400103E11F00C94724CE22FEF70EB8707C02E
:1098E400103F11F00C94794CE22FEF70EC870F5F6E
:1098F400C4CF00E0053010F00C948D4CA9EEB2E119
:10990400E02F0E94CCA8E12FF0E0DE0118960E941F
:1099140026A70F5FEFCF388530FF02C03E7F01C01E
:109924003160E32F0E94DEB8A29608950E94BAA483
:1099340000E00E944EAFA091E912A0830E944EAFB6
:10994400A091EA12A0830E944EAFA091EB12A083D3
:109954000E944EAFA091EC12A0830E944EAFA09142
:10996400ED12A0830E944EAFA091EE12A0830E943C
:10997400BFA408950E94D7B8AD0100E00E9454AF7F
:10998400A091E012A0830E9454AFA091E112A083A1
:109994000E9454AFA091E312A0830E9454AFA091FF
:1099A400E212A0830E9454AFA091E512A0830E940A
:1099B40054AFA091E712A0830E9454AFA091E61285
:1099C400A0830E9454AFA091E412A0832091EF12CF
:1099D4003091F012122F232F33270E9454AF20838B
:1099E4000E9454AF10830E9454AFA091E812A08348
:1099F400E02F0E94DEB826960895A1E00E94394F18
:109A0400E0E0E093F41208950895BA93AA93A0971E
:109A14000E94D7B8E0E0EE83AE81A73010F00C943A
:109A24001D4DEE81AEA1BFA1F0E00E9449AFEE81D1
:109A3400EF5FEE83F1CFE0E0EE83AE81AA3010F069
:109A44000C942E4DEE81F0E0DE0117960E9449AF92
:109A5400EE81EF5FEE83F1CF0E945AAFE8E00E94FF
:109A64005FAFDE0157960E94C6112E2F213010F4ED
:109A74000C943F4D0E9465AF0895EA89E07811F097
:109A84000C94574DEA89EA8FE068EA8F0E945AAF36
:109A9400E1E00E945FAF0E946AAF10F40C94554D50
:109AA4000E9465AF08950E9498AAED89E07211F0B2
:109AB4000C945E4DED89ED8FED89E07111F40C94F9
:109AC400754DED89ED8FDE015D96EC91EF7E0E9480
:109AD40071AF0E946AAF10F40C94734D0E9465AF8D
:109AE40008950E9498AAED89E87011F00C948C4DA9
:109AF400ED89ED8FDE015D96EC91E8600E9471AF17
:109B04000E946AAF10F40C948A4D0E9465AF0895C8
:109B14000E9498AAEC89E07411F40C94A34DEC898A
:109B2400EA8FEF7BEA8FE2E0F0E00E9478AF0E94D8
:109B34006AAF10F40C94A14D0E9465AF08950E9481
:109B440098AAEA89E093F112EB89E093F212EC8986
:109B5400E093F312ED89E093F412E7703E2F313075
:109B640010F40C94BA4D383010F00C94BA4D01C076
:109B740001C03F83ED89E093F412EC89EF730E94F6
:109B84007CAF2E2F0B89A02F0E946F201E2F1C3319
:109B940010F00C94D04DFE0138961083EA89EF77CB
:109BA4000E947CAF1E2F1C3310F00C94DC4DFE0180
:109BB40039961083283110F00C94E34DFE013A9647
:109BC4002083EF89EF710E947CAF5E2FEE89EF73E3
:109BD4000E947CAFE98BA88D0E946F204E2FFE015E
:109BE4003B964083FE013C965083E989ED87AB8523
:109BF400A43610F40C94034EE2E00E94DEB8A8965A
:109C04000895AC85AD3010F00C940D4EA03011F4D5
:109C14000C940D4E05C0E3E00E94DEB8A8960895AA
:109C2400AD85A03210F00C941C4EA03011F40C94AD
:109C34001C4E05C0E4E00E94DEB8A8960895AA85EB
:109C4400A83110F40C942B4EE5E00E94DEB8A896DF
:109C54000895A885AC3310F40C94354EE6E00E94C8
:109C6400DEB8A8960895AF81A83010F40C943F4E46
:109C7400E7E00E94DEB8A8960895E0E0EE83AE81A6
:109C8400A73010F00C94554EEE81AEA1BFA10E94F6
:109C9400CCA8EE81F0E0DE0117960E9426A7EE81A3
:109CA400EF5FEE83ECCFE0E00E94DEB8A896089563
:109CB40029970E94D7B82A2F3F8548895989583156
:109CC40011F00C94664E50E0583110F40C946D4E23
:109CD4000E9480AF08954C3311F00C94724E40E012
:109CE4004C3310F40C94794E0E9480AF08953C33A9
:109CF40010F40C947E4E30E0E091F412E862E093AC
:109D0400F412EF7EE093F412E32FE068EE83E09127
:109D1400F212EF83E091F312E887E091F412E987FD
:109D2400E0E0EA87EB87EC87ED87503011F00C9484
:109D3400A04E403011F00C94A04E09C0583110F0E0
:109D44000C94A94E4C3310F00C94A94E01C00CC0D5
:109D5400A32F0E948020EE83A42F0E948020EF83F3
:109D6400A52F0E948020E887213010F40C94BF4E68
:109D7400283010F00C94BF4E01C007C01091F412AB
:109D8400187F122BFE0139961083EE81E068EE8372
:109D9400DE011996EC91E862EC930E945AAFE4E07C
:109DA4000E945FAFDE011B960E94F6100E2F0E94E8
:109DB400C1A9003011F40C94E24E0E9480AF0895C2
:109DC400E0E00E94DEB86296089524970E94D9B814
:109DD4001A2F28853985203011F40C94F64E2D3035
:109DE40010F00C94F64E03C00E9485AF0895103015
:109DF40011F40C94024F103210F00C94024F03C073
:109E04000E9485AF0895343110F40C940E4F33330F
:109E140010F00C940E4F01C037E1A12F0E94802056
:109E2400EC83A22F0E948020ED83A32F0E94802028
:109E3400EE83E0E0EF830E948AAFE4E0F0E0FA937F
:109E4400EA93E3E00E945FAFDE0119960E94F610E8
:109E54000E2F0E948AAF003011F40C94344F0E94EC
:109E640085AF0895E0E00E94E0B82A96089522970D
:109E74000E94DAB82A2F022FE02FE03011F00C9460
:109E8400464FE0E0EB830DC0E13011F00C944D4FF0
:109E9400E0E4EB8306C0E23011F00C94534FE4E4A9
:109EA400EB83E0E0EC83E7E0F0E00E9478AFDE01D2
:109EB40018960E94F6101E2F103011F40C94674F60
:109EC400E1E00E94E1B825960895E0E00E94E1B83F
:109ED4002596089522970A93E7E0F0E00E9478AF70
:109EE400DE0116960E94C6110E2F003011F00C945C
:109EF4007F4FE981088123960895EFEF0881239627
:109F040008950881239608952C970E94D9B89D013D
:109F14000E948EAFACE00E946BABE0E3EA930E9438
:109F240091AF0E9495AFDE0119960E94A0AF10F484
:109F34000C94A14FE1E00E94E0B86096089510E00F
:109F4400183010F00C94AF4F0E94A5AFF0E0DE0182
:109F540014960E9426A71F5FF3CFE0E00E94E0B8AA
:109F64006096089568970E94D7B89D014E8D5F8DC5
:109F740005C0E2E00E94DEB8A0960895FE01729644
:109F84000E9440AF0E94C3AE5A934A93E0E3EA931F
:109F9400A0E10E946BABE0E3EA930E9445AF0E940C
:109FA40095AFDE0157960E94A0AF10F40C94DF4FDA
:109FB400E1E00E94DEB8A0960895E98D0E94ACAF5E
:109FC400DA011F96EC93EE85DA011E96EC93E88D88
:109FD4000E94ACAFDA011D96EC93EE85DA011C9673
:109FE400EC93EF890E94ACAFDA011B96EC93EE85FB
:109FF400DA011A96EC93EE890E94ACAFDA01199655
:10A00400EC93EE85DA011896EC93ED890E94ACAFDF
:10A01400DA011796EC93EE85DA011696EC93EC8947
:10A024000E94ACAFDA011596EC93EE85DA01149632
:10A03400EC93EB890E94ACAFDA011396EC93EE85B6
:10A04400DA011296EC93EA890E94ACAFDA01119618
:10A05400EC93EE85DA01EC93EE89FF2766277727E8
:10A064000E94B7AFEF890E94BFAFE88D0E94BFAFD7
:10A07400E98DFF27662777270E9465A80E94FDB80F
:10A084000E94ECAEEA89FF27662777270E94C7AFB4
:10A09400EB890E94D0AFEC890E94D0AFED89FF27F5
:10A0A400662777270E9400AF0E94FDB80E9498A7F8
:10A0B4000E94A8A73A932A930E94D8AF0E946FA83F
:10A0C4000E946ABAFE017696FA93EA930E94D8AF88
:10A0D40013E11A3010F40C9479500E94A5AFEA50A1
:10A0E400F0E0DE0152960E9426A71150F2CF10E054
:10A0F400143110F00C948B500E94B9A5EC91E0300F
:10A1040011F00C9489500E94B9A5E0E3EC931F5F11
:10A11400EFCFE0E00E94DEB8A09608952E970A9350
:10A12400DE0115960E94074D0E2F003011F40C9499
:10A134009E5008812F960895E885E093D011EE8112
:10A14400E093D111EF81E093D211E985E093CC1132
:10A15400EA85E093CD11EB85E093CE11ED81E09398
:10A16400CF11A3EDB1E1E091D011F0E0ED93FC93B8
:10A17400A091D311B091D411ECE30E94B9B9E0934A
:10A18400D311F093D411A091D311B091D411E091D3
:10A19400D111F0E0EA0FFB1FE093D311F093D41137
:10A1A400E091D311F091D411662777270E94E1AF93
:10A1B4000E94F1A80E940EA5E091D2110E94E4AE83
:10A1C4000E94F3B80E94E1AFE093D511F093D61149
:10A1D4006093D7117093D811E0E008812F96089509
:10A1E400E0E0E093F51208951A930A93E3E0EA930A
:10A1F400A3E0B0E00E94BB0BA1E00E94E525A8E02B
:10A20400B0E00E9440BCE1E0E093F712E0E0E093AC
:10A21400F6120E94E5AF00E0053010F00C942751CF
:10A2240010E0123010F00C942551AAE01A9FF001AE
:10A23400E05FFC4EDF01E02FF0E00E94B6AC0E942C
:10A2440007AC1F5FEECF0F5FE7CFEAE0F0E0E093EB
:10A25400F812F093F912A091F812B091F912E2E019
:10A264000E94B9B9E093F812F093F912E0E0E09398
:10A27400FA12E093FB120991199108950E94ECAF30
:10A2840011F40C9448510E94F1AF08950E94F125F5
:10A29400E03011F00C945451A1E00E94E525A3E0B4
:10A2A4000E94F60EA3E00E940D0F8F010630E0E03D
:10A2B4001E0710F40C9498510E94200C9F0144E056
:10A2C400413010F40C947B510E94F6AFDF01E42F6F
:10A2D400F0E00E94C5ADBF010E94F6AFDF01E42F9C
:10A2E400E150F0E00E94CAADDB01ED93FC934150D4
:10A2F400E7CF0E94F6AF20833183E091F612EF5F3F
:10A30400E093F612A091F612A23010F40C948D5141
:10A31400E0E0E093F6120E94E5AF0E94FEAF10F475
:10A324000C949851AAEFB2E10E94DCA40E949F51C0
:10A334000E94D2510E94F1AF08950E94DAB80E949F
:10A34400F125E03011F00C94A9510E9409B00E944B
:10A35400FEAF10F40C94B451E0EEFEE20E94E1B8BA
:10A364002396089500E010E020E0253010F00C94CE
:10A37400C551AAE1B3E1E22FF0E00E94B6AC0E941D
:10A384000CAC2F5FF2CF0E9410B00E9417B0009364
:10A394000C1310930D13F8010E94E1B8239608954D
:10A3A4000E94D8B80E94F125E03011F00C94DC51E1
:10A3B4000E9409B00E94FEAF10F40C94EB51ECE83B
:10A3C400F0E0E0930E13F0930F130E94DFB825968C
:10A3D400089500E010E040E0453010F00C94FC518A
:10A3E400E42FA0E1B3E1F0E00E94B6AC0E940CAC13
:10A3F4004F5FF2CF0E9410B0D8010E9498839F0152
:10A4040020930E1330930F130E94DFB825960895FE
:10A414000E94D9B83A2F323010F40C941752E0E06D
:10A42400F0E00E94E0B82496089500E010E020E0F7
:10A43400253010F00C942C52AAE03A9FF001E05F12
:10A44400FC4EDF01E22FF0E00E94B6AC0E940CAC9F
:10A454002F5FEECF0E9410B0F8010E94E0B824965E
:10A4640008950E94D9B8A1E00E94E525A0E00E94C9
:10A4740026B0D8010E9498839F010E94E0B82496D8
:10A4840008951A930A93A1E00E94E525A1E00E9491
:10A4940026B00E9417B0F8010991199108951A93F2
:10A4A4000A930E9430B0E0E0E093341400E010E03E
:10A4B4000530E0E01E0714F00C946752AFE2B4E1FB
:10A4C4000E94CCA50F5F1F4FF3CF0E94D061E0E044
:10A4D400E0932D14A3E10E943C0FA1E20E94F60E2A
:10A4E400E0E0E0932C14E0930713E0930613099142
:10A4F4001991089524970E94D8B800E010E00E94B2
:10A5040007614E2F403011F00C948C52E8ECE0932C
:10A51400B01203C0E1E0E093B0120E94AF88E030D3
:10A5240011F40C949C52A4E2B4E10E948C881E2F76
:10A5340010930513A0913414AF5FA0933414A53085
:10A5440010F40C94A852E0E0E0933414E091341435
:10A55400F0E0E15DFB4EFF93EF930E948961AF91C0
:10A56400BF91EC93EFE2F4E1FA93EA93A5E00E9441
:10A57400EF233E2F303011F40C94E05200912F144D
:10A584000093071300FF04C0E1E0E093FC1203C052
:10A59400E0E0E093FC1201FF04C0E1E0E093FD126F
:10A5A40003C0E0E0E093FD1202FF04C0E1E0E093A9
:10A5B400FE1203C0E0E0E093FE1201C003E60E9435
:10A5C400D3612E2F203011F40C941853E0E0E09363
:10A5D4002D14113011F40C94F452123011F40C9423
:10A5E400F4520AC00E94D0610E94CE88003011F457
:10A5F4000C94FE520E9430B0003011F40C940653B7
:10A60400A3E20E94F60E0DC0A3E20E940D0F0E9469
:10A6140036B0A83EE3E0BE0710F40C9413530E9436
:10A62400D061E1E00E94DFB829960895113011F05D
:10A634000C942053A1E00E943BB007C0123011F0EB
:10A644000C942753A0E00E943BB0033610F00C9406
:10A654003053013010F40C94305301C005C0E02F86
:10A66400E853E093B5121AC0003011F00C94505323
:10A67400E1E0E093B512E0E0E0930813E0932D14D9
:10A68400AFE00E94580FED83FE83AD81BE815F97DA
:10A6940010F40C945053E0E0E0930613033610F0EA
:10A6A4000C946053E02FE57011F40C946053A09166
:10A6B4000813A03011F00C94605301C018C0E1E0FD
:10A6C400E09308130E94B061113011F40C9471539B
:10A6D400E0910613E03011F00C94715301C003C0F3
:10A6E4000E94BA6102C00E94D0610E94CE880336E3
:10A6F40010F00C94865301FF07C0A0910913A030F9
:10A7040011F00C94865301C01BC0E1E0E0930913DF
:10A714000E94B061123011F40C949753E091061327
:10A72400E03011F00C94975301C003C00E94BA6149
:10A7340005C00E94D061E1E0E0932D140E94CE8810
:10A74400A0912D14A13011F00C94AB5301FF01C062
:10A7540001C020C00E940761E03011F40C94B5538D
:10A76400E1E0E0932E140E940761E03011F00C94B4
:10A77400C253E0912E14E03011F40C94C25301C082
:10A7840008C0E0E0E0932E14E0912D14EF5FE09315
:10A794002D140BC0A0912D14A23011F00C94D7539A
:10A7A400E0912D14EF5FE0932D14013010F40C941C
:10A7B400E053E1E00E94DFB829960895E0E00E94AA
:10A7C400DFB829960895E0912D140895EAE7F4E09E
:10A7D40060E070E00E946ABAA5E3B4E10E94231C21
:10A7E400E3E8F4E060E070E00E946ABAADE3B4E14B
:10A7F4000E94231CECE8F4E060E070E00E946ABA76
:10A80400A5E4B4E10E94231CE5E9F4E060E070E013
:10A814000E946ABAADE4B4E10E94231CEEE9F4E0BC
:10A8240060E070E00E946ABAA5E5B4E10E94231CCE
:10A83400E7EAF4E060E070E00E946ABAADE5B4E1F2
:10A844000E94231CE0EBF4E060E070E00E946ABA2E
:10A85400A5E6B4E10E94231CE9EBF4E060E070E0BB
:10A864000E946ABAADE6B4E10E94231C08951A93CB
:10A874000A93A0918414A33010F40C944A54A5E2D2
:10A884000E9445B010F40C944A54E0E0E093841420
:10A89400A0918414A23011F00C945554A5E20E94A6
:10A8A400F60E0E944CB0A0918414A13010F40C94C4
:10A8B4005F54E1E0099119910895E0E0099119913B
:10A8C40008950A93E1E0E09384140E9471440E9485
:10A8D40001450E943CAF0E94A94B0E2F0E94B9264D
:10A8E400E03011F00C9477540062003011F00C94B5
:10A8F4007F54E1E0E093A6121DC0E02FE07E11F446
:10A904000C948854E8ECE093A61214C0E02FEC7188
:10A9140011F40C949154E9ECE093A6120BC001FFDE
:10A9240004C0EAECE093A61205C000FF03C0E4E60D
:10A93400E093A6120E944CB0E02F09910895EF977E
:10A94400EF97A297E1E0E09384140E9453B0A2EC45
:10A95400B4E080E090E00E94F448A3EDB4E080E02D
:10A9640090E00E94F448A4EEB4E080E090E00E94FD
:10A97400F448A1E00E94D2480E9494AAA2E00E9456
:10A98400C045A3E00E94D845A5EFB4E080E090E084
:10A994000E94F4480E9453B0A1E00E9479460E94AC
:10A9A40094AAA2E00E94C045A2E00E94D845ABEF61
:10A9B400B4E080E090E00E94F4480E9453B00E940A
:10A9C40094AAA1E00E94D2480E945CB0AFEFB4E028
:10A9D40080E090E00E94F448ECE0F5E060E070E094
:10A9E4000E94D1A90E9462B00E9469B0A4E10E94B1
:10A9F4009B460E9494AAA1E00E94D2480E946EB095
:10AA0400A0E00E94C045A0E00E94D845A8E3B5E0BC
:10AA140080E090E00E94F4480E945CB0A1E5B5E0BB
:10AA240080E090E00E94F448A2E00E94D845ADE5A1
:10AA3400B5E080E090E00E94F4480E945CB0A1E0A0
:10AA44000E940346A1E7B5E080E090E00E94F4484C
:10AA5400A0E00E940346A1E00E941B46AEE7B5E0D9
:10AA640080E090E00E94F448A0E00E941B46A1E030
:10AA74000E943346AEE8B5E080E090E00E94F448DE
:10AA8400A0E00E9433460E946EB00E9494AAA3E004
:10AA94000E94D248A1E00E941C45A8EEB3E00E94A7
:10AAA4007E0E0E944CB0EF96EF96A29608950E94F7
:10AAB40074B00E947CB010F00C9463550E9487B06F
:10AAC40002C00E948CB000E010E00030E2E01E07FB
:10AAD40010F00C947455DE0113960E94CCA50F5F00
:10AAE4001F4FF3CF0E9493B00E94DC810E94E1B813
:10AAF4002396DE5F0895AA9323970E94A0B0E98568
:10AB0400EE83F801E07CAF01405C5F4FFA01E01B8B
:10AB1400F10BEF83F887EE810E94A7B010F00C943C
:10AB240096558A010E9487B00E94ADB0AE85BF855C
:10AB34000E94B4B02C960895AA932B97E8E0E8837A
:10AB44000E94A0B0F801E07CAF01405C5F4FDA01E5
:10AB5400A01BB10BEE81F0E0AE17BF0710F00C9410
:10AB6400B6558A010E9487B0EBE1EF83EC89E88750
:10AB7400EB89E987EA89EA87E989EB87E0E2EC87F0
:10AB8400ED87EE870E94ADB0DE011B960E94B4B043
:10AB9400659608950E9474B00E947CB010F00C94E5
:10ABA400D6550E9487B002C00E948CB000E010E02D
:10ABB4000030E2E01E0710F00C94E755DE01139616
:10ABC4000E94CCA50F5F1F4FF3CF0E9493B00E9449
:10ABD400C6B00E9483AD0E9434950E94CDB00E94FD
:10ABE400D2B00E94E1B82396DE5F08950E94D7B8E0
:10ABF4003A2F4E815F81E1E0E0938414E32FE05328
:10AC04000E2F023010F40C94085600E04A93A32F40
:10AC14000E9420241E2F523611F00C941556A02F9A
:10AC24000E94034642C0553711F00C941D56A02FC4
:10AC34000E941B463AC05C3611F00C942556A02F96
:10AC44000E94334632C0513611F00C942D56A42F75
:10AC54000E944B462AC0543611F00C943A561333D2
:10AC640010F40C94365612E3A12F0E94F0451DC037
:10AC7400563611F00C9443561A93ACE00E94854565
:10AC840014C0533711F00C945756A12FEAE00E94D8
:10AC9400C9B92E2FA22F0E94D845A12FEAE00E9405
:10ACA40018BA2E2FA22F0E94C0450E944CB00E94B9
:10ACB400DEB8289608950E943BA5E1E0E093841451
:10ACC400E22FE0530E2F3A93A22F0E9420241E2F2E
:10ACD400E42FE33611F00C947356A1E00E941C4556
:10ACE4005EC0E03711F00C947B56A2E00E941C4534
:10ACF40056C0E53611F00C948356A3E00E941C451F
:10AD04004EC0E23411F00C948C56A8EEB3E00E94CD
:10AD1400BE4845C0EE3611F00C949E56003011F436
:10AD24000C9499560A3010F00C94995601C001E025
:10AD3400A02F0E94D24833C0EC3611F00C94AA56CE
:10AD4400000F000F000FA02FBB270E94514527C002
:10AD5400E23611F00C94B656000F000F000FA02F2E
:10AD6400BB270E946B451BC0ED3611F00C94BE56F8
:10AD7400A12F0E94374913C0E23711F00C94C65634
:10AD8400A12F0E944B490BC0E33711F00C94D1560C
:10AD9400AAE01A9F102DA12FBB270E94884B0E9466
:10ADA4004CB00E94DFB827960895A2970E94D7B8A6
:10ADB4005A2FE1E0E09384140E9479ADA9A5A4344C
:10ADC40011F00C944257E52FE03311F00C94F15636
:10ADD400E5E3F4E10E94BDA60E94E4B04CC0E13377
:10ADE40011F00C94FC56EDE3F4E10E94BDA60E9420
:10ADF400E4B041C0E23311F00C940757E5E4F4E108
:10AE04000E94BDA60E94E4B036C0E33311F00C9456
:10AE14001257EDE4F4E10E94BDA60E94E4B02BC0F9
:10AE2400E43311F00C941D57E5E5F4E10E94BDA64E
:10AE34000E94E4B020C0E53311F00C942857EDE5EE
:10AE4400F4E10E94BDA60E94E4B015C0E63311F0FF
:10AE54000C943357E5E6F4E10E94BDA60E94E4B0E9
:10AE64000AC0E73311F00C943D57EDE6F4E10E947B
:10AE7400BDA60E94E4B00E94E8B00E94EDB008951F
:10AE8400E9A5E33611F00C944C570E94F2B00E94ED
:10AE9400F7B09CC0ED3611F00C9455570E9400B1E8
:10AEA4000E94F7B093C0EC3611F00C946257E8E8B6
:10AEB400F0E00E94BDA6A0E2B0E00E942D1B86C077
:10AEC400E73611F00C946B570E9405B10E94F7B05D
:10AED4007DC0EA3711F00C9474570E940AB10E94A5
:10AEE400F7B074C0E13611F00C947D570E940FB195
:10AEF4000E94F7B06BC0E43711F00C949A57A8A5E0
:10AF0400AC3611F00C94885741E001C040E0E09168
:10AF1400D011EA93E091D111EA93E091D211EA932E
:10AF2400E0E0EA934A93DE011B960E948A1E4EC01B
:10AF3400E43611F00C94B75720E030E0A8A5A5370B
:10AF440011F00C94A75722E031E0E091CE110E9459
:10AF540014B1E0E2EA93E091CC11EA932A933A9394
:10AF6400DE011C960E94361F31C0E73711F00C94A5
:10AF7400E857A091CF11A13010F40C94C857A091B8
:10AF8400CF11A83010F00C94C8570BC0E1ECF5E0D9
:10AF940060E070E00E946ABADE011A960E940B1CFF
:10AFA40015C041E0553611F00C94D95742E0E091B8
:10AFB400CF11EA934A93DE0118960E94DA24A8A5D9
:10AFC400A33711F00C94E857E0E0E8870E94E8B05A
:10AFD4000E94EDB00895EF97EF97A2970E94D9B819
:10AFE4001A2FFE01EC55FF4F2081FE01EB55FF4F58
:10AFF4003081E1E0E09384140E948EAFA0EAB0E0D7
:10B004000E94F31BE32FE23611F00C941C58EDEC74
:10B01400F5E060E070E00E9419B10E9462B00E9405
:10B02400DFAEA4E10E949B460E9494AAA1E00E9484
:10B03400D2481EC0EC3611F00C943158E12FE05385
:10B044000E2F0A3010F40C94285801E0A02F0E940F
:10B0540079460E9494AAA1E00E94D24809C0E1372F
:10B0640011F00C943A580E9494AAA1E00E94D2488C
:10B074000E944CB00E94E0B8EF96EF96A89608950F
:10B084001A930A938D01E1E0E0938414F801E181BD
:10B09400E33711F00C9453580E941EB10E94F855E6
:10B0A4001AC0E63611F00C945C580E941EB10E943E
:10B0B4005D5611C0E63711F00C9465580E941EB11C
:10B0C4000E94D75608C0E73611F00C946D580E94C0
:10B0D4001EB10E94ED570E944CB009911991089538
:10B0E400AA932897D2500E94D7B8E1E0E093841441
:10B0F400A0E00E94F7250E9464A9FE01E25FFD4FD3
:10B1040000811127D801E9E00E941BB98F010030AA
:10B11400EEE31E0710F00C9492580E9487B002C010
:10B124000E948CB000E010E00030E2E01E0710F056
:10B134000C94A358DE0116960E94CCA50F5F1F4FF6
:10B14400F3CFE0918514F09186140E9427B1E0E0DA
:10B15400F2E0FA93EA93DE011C960E94C6B00E94C4
:10B164006ABADE01AE5EBD4FAC910E942EB10E9460
:10B1740034950E94DFAE0E94D2B00E9463544E2FD9
:10B18400423010F40C94CE580E944CB0E42F0E942C
:10B19400DEB82F96DE5F0895A3E00E94D24820E037
:10B1A40030E040E0F9012F5F3F4F0E94D8A65C9148
:10B1B4005B3111F00C94E05841E009C0503011F0BB
:10B1C4000C94E65842E003C0A52F0E94901420344A
:10B1D400E0E03E0710F00C94F458403011F00C9469
:10B1E400F45801C001C0DECF0E94C1A9413011F062
:10B1F4000C94125921503040F901DE0116960E9438
:10B2040033B1FE01E85FFD4FFA93EA930E94E4B084
:10B21400DE01AA5FBD4F0E944258285F3F4F05C020
:10B22400423011F00C94175900C02030E2E03E0780
:10B2340010F00C941E59B5CF0E94C1A90E944CB0C5
:10B24400E0E00E94DEB82F96DE5F08950A9300E0E6
:10B254000E94CB28E03011F40C94315902600E9412
:10B26400F928E03011F40C94385904600E9429291B
:10B27400E03011F40C943F5908600E945529E030E5
:10B2840011F40C94465900610E948329E03011F4B2
:10B294000C944D590062E02F099108950A9300E03F
:10B2A4000E94142CE03011F40C94595901600E944E
:10B2B4003A2AE03011F40C94605904600E94A329E6
:10B2C400E03011F40C94675908600E94C329E030FF
:10B2D40011F40C946E5900610E94192AE03011F4A3
:10B2E4000C9475590062E02F099108950E94D7B813
:10B2F4001A2F2E813F8148855985183010F00C94FF
:10B304008859E1E00E94DEB82A9608950E9438B177
:10B3140000E00E94CA27E03011F40C9492590160B5
:10B324000E947626E03011F40C94995902600E9430
:10B334009626E03011F40C94A05904600E94012771
:10B34400E03011F40C94A75908600E947C28E03086
:10B3540011F40C94AE590061E02FDA01EC930E94D1
:10B364005059DA011196EC9300E00E94682CE03009
:10B3740011F40C94BE5901600E94342CE03011F495
:10B384000C94C55902600E944D26E03011F40C94CF
:10B39400CC5904600E942728E03011F40C94D3594E
:10B3A40008600E941128E03011F40C94DA5900610D
:10B3B4000E943D28E03011F40C94E15900620E948F
:10B3C4005D28E03011F40C94E85900640E94A82C24
:10B3D400E03011F40C94EF590068FA0102830E94E2
:10B3E400642ADA011396EC930E94B02ADA011496C7
:10B3F400EC93D901E8E0EC930E94DEB82A96089514
:10B404002A970E94D7B81A2F288939894A895B89D3
:10B4140000E0183010F00C94145AE1E00E94DEB8F9
:10B42400649608950E9438B10E94DFAE0E941EA95E
:10B4340000E00E94C02BE03011F40C94225A016009
:10B444000E94DA2BE03011F40C94295A02600E9415
:10B45400222DE03011F40C94305A04600E94982B91
:10B46400E03011F40C94375A08600E94A62BE030A7
:10B4740011F40C943E5A0061E02FDA01EC9300E0E1
:10B484000E94362BE03011F40C94495A01600E945A
:10B494001A2BE03011F40C94505A02600E945E2B77
:10B4A400E03011F40C94575A04600E94862BE0306B
:10B4B40011F40C945E5A08600E94082BE03011F4D9
:10B4C4000C94655A00610E94F42BE03011F40C9442
:10B4D4006C5A0064FA0101830E942859DA01129619
:10B4E400EC9300E00E945726E03011F40C947B5A50
:10B4F40001600E947F27E03011F40C94825A0260AC
:10B504000E94B926E03011F40C94895A04600E9418
:10B51400FB27E03011F40C94905A08600E946728CD
:10B52400E03011F40C94975A00610E945B27E030DC
:10B5340011F40C949E5A00620E94CD29E03011F45B
:10B544000C94A55A0064FA01038300E00E94E627E4
:10B55400E03011F40C94AF5A01600E947627E03079
:10B5640011F40C94B65A02600E948E27E03011F454
:10B574000C94BD5A04600E947C28E03011F40C94B1
:10B58400C45A08600E94F52CE03011F40C94CB5A94
:10B5940000610E94FE2CE03011F40C94D25A006237
:10B5A4000E940A2DE03011F40C94D95A00640E94D0
:10B5B400132DE03011F40C94E05A0068FA0104836E
:10B5C4000E94492DDA011596EC935A934A930E94EE
:10B5D40040B10E94E4B0D901E8E0EC93E0E00E94BD
:10B5E400DEB8649608956697FE010E9440AFA6E116
:10B5F400B0E00E94F31BE2EEF5E060E070E00E9430
:10B60400D1A90E9445B166960895A8970A930E940D
:10B6140029AE0E9452B1E8A7E3EFF5E060E070E0E4
:10B624000E945AB1DE0111960E94171A0E2F0E9431
:10B6340020AEE0E2EC93E0E0F6E060E070E00E942F
:10B644006ABA0E9466ABA4E1B0E00E94CA1BDE01A4
:10B6540011960E94171AEA93DE0112960E949A71BB
:10B66400A0E00E948B710881A9960895A8970E9472
:10B67400C5A9EDE0F6E060E070E00E94D1A90E9467
:10B6840045B1A89608956E970E94D8B80A2F1BA1B9
:10B694002CA13DA14EA10E3110F00C94565BE1E0BB
:10B6A4000E94DFB8A79608954A933A93E0E0EA939C
:10B6B400A02FBB270E94F31B0E9466AB0E941EA909
:10B6C400E091A112A32FB42FEC93E091A212A32F27
:10B6D400B42F1196EC93E091A312A32FB42F1296DA
:10B6E400EC93E091A412A32FB42F1396EC93E09162
:10B6F400A512A32FB42F1496EC93E091A612A32FB6
:10B70400B42F1596EC93E091A712A32FB42F16969D
:10B71400EC93E091A812A32FB42F1796EC93E09129
:10B72400A912A32FB42F1896EC93E091AA12A32F79
:10B73400B42F1996EC93E091AB12A32FB42F1A9661
:10B74400EC93E091AC12A32FB42F1B96EC93E091F1
:10B75400AD12A32FB42F1C96EC93E091AE12A32F3D
:10B76400B42F1D96EC93E091AF12A32FB42F1E9625
:10B77400EC93E091B012A32FB42F1F96EC93E091B9
:10B78400B112A32FB42F5096EC93E091B212A32FD1
:10B79400B42F5196EC93E091B312A32FB42F529689
:10B7A400EC93E091B412A32FB42F5396EC93E09151
:10B7B400B512A32FB42F5496EC93E091B612A32F95
:10B7C400B42F5596EC93E091B712A32FB42F56964D
:10B7D400EC93E091B812A32FB42F5796EC93E09119
:10B7E400B912A32FB42F5896EC93E091BA12A32F59
:10B7F400B42F5996EC93E091BB12A32FB42F5A9611
:10B80400EC93E091BC12A32FB42F5B96EC93E32F3F
:10B81400F42F7C96A0E0A083E32FF42F7D96A083E1
:10B82400E32FF42F7E96A0834A933A930E94ECADC3
:10B83400AEE1B0E00E94061BA12FB22FEEE1EC9323
:10B84400E0E00E94DFB8A7960895E6971A930A935A
:10B85400E091D011EE83E091D111EF83E091D21108
:10B86400E887E091CC11E987E091CD11EA87E09176
:10B87400CE11EB87E091CF11EC87E0E2ED870091E8
:10B88400D3111091D4111A930A93A0E00E94A92312
:10B89400EE870E94DBADEF87E0E2E88BE98BE09175
:10B8A400D511F091D6116091D7117091D8110E94E1
:10B8B40060B1EA8B0E9469B1A1E00E94C523EB8BC1
:10B8C4000E9469B1A2E00E94C523EC8B0E9469B179
:10B8D400A3E00E94C523ED8BA091CC110E94E1222C
:10B8E400EE8BA091CC110E94EE22EF8BA091CC1193
:10B8F4000E940923E88FE091CF11EA93A091D0111F
:10B904000E943823E98FE091CF110E9470B10E9408
:10B9140049230E94D5ADEA8F0E94DBADEB8FE09105
:10B92400CE11EA93A091D0110E9457230E94D5AD65
:10B93400EC8F0E94DBADED8FE091CE110E9470B1CF
:10B944000E9465230E94D5ADEE8F0E94DBADEF8F80
:10B954000E9477B1A091CE110E94AA220E94D5AD77
:10B96400E8A30E94DBADE9A30E9477B1E091CE1178
:10B97400EA93A091D0110E9472230E94D5ADEAA34C
:10B984000E94DBADEBA3E0E0ECA3EDA30E9477B152
:10B99400E091CE110E9470B10E9486230E9460B192
:10B9A400EEA30E9469B1A1E00E94C523EFA30E9407
:10B9B40069B1A2E00E94C523E8A70E9469B1A3E08F
:10B9C4000E94C523E9A70E946C4FEAA7E0E0EBA719
:10B9D400ECA7EDA7EA83EB83EC83ED830E9469B1C6
:10B9E400A0E00E94C523EEA70E9469B1A1E00E94D5
:10B9F400C523EFA70E9469B1A2E00E94C523E8AB6A
:10BA04000E9469B1A3E00E94C523E9ABECE2EA938A
:10BA1400DE0117960E949A71A0E00E948B71E0E00B
:10BA240019810881E8960895E0E0E0938714E09393
:10BA34008814E0938914EAE0E0938A14E0938B1469
:10BA44000E947AB1E0E0E0939C14E0939B14E093AD
:10BA54009E1408950E947AB1A0E00E94442AA0E0B6
:10BA64000E94852AA0E00E941B280E9480B1A0E0C9
:10BA74000E94FE2B0E94C0AA0E94E82A08952197E2
:10BA84000E94D6A9A0918714A13011F00C944A5DAC
:10BA9400A0918714A23011F00C94505DA0918814E9
:10BAA400A13011F00C94565DA0918814A23011F0CD
:10BAB4000C945C5DA0919A14A33011F00C946D5D0C
:10BAC4000E94FB27E03011F40C946A5D0E948AB155
:10BAD400EE81E260EE83A0919A14A23011F40C94EA
:10BAE400785DA33011F40C94785D20C020919914F2
:10BAF4003327AAE0A29FF001A39FF00D9F012436F3
:10BB0400E0E03E0710F00C94895D24E630E0A3E108
:10BB14000E940D0F8F010217130710F40C94955D0A
:10BB2400A0E00E941B28EE81E260EE830E9490B1A7
:10BB34005E2F513011F40C94A45D523011F40C9426
:10BB4400A45D77C0A4E10E940D0F8F010E946728B5
:10BB54004E2FA0919B14A23011F00C94B85D0536C1
:10BB6400E0E01E0710F40C94B85D01C002C00E940E
:10BB740080B10333E0E01E0710F40C94CC5D04366E
:10BB8400E0E01E0710F00C94CC5D403011F00C94F2
:10BB9400CC5D0CC0093CE0E01E0710F40C94D75DAA
:10BBA400403011F40C94D75D01C009C0A0919B14DE
:10BBB400A23011F00C94E15DE9ECE093AC12033394
:10BBC400E0E01E0710F40C94F25D0436E0E01E077A
:10BBD40010F00C94F25D403011F40C94F25D01C04D
:10BBE40003C0E1E0E0939C14093CE0E01E0710F47C
:10BBF4000C940D5E0A3FE0E01E0710F00C940D5EFD
:10BC0400403011F00C940D5EE0919C14E03011F47E
:10BC14000C940D5E01C006C0E1E0E093AC12E0E0DC
:10BC2400E0939C14403011F40C941B5EEE81E260AE
:10BC3400EE83AAE10E9445B010F40C94255EA0E0C6
:10BC44000E942C2D03C0EE81E260EE830E9495B128
:10BC54005E2F513010F40C94835EA0919D14A53096
:10BC640010F40C94365E4DC0A0919D14A03011F4D4
:10BC74000C94415EA23011F40C94415E07C00E9402
:10BC8400CD29E03011F00C94485E01C002C00E943E
:10BC94009AB1A0919D14A13011F40C94565EA33076
:10BCA40011F40C94565E07C00E94CD29E03011F4C3
:10BCB4000C945D5E01C002C00E949AB1ABE10E9487
:10BCC4000D0F8F01A0919D14A43011F00C94725E9D
:10BCD400A0E00E94D3290E949AB1E1E0E093AF1260
:10BCE4000D32E1E01E0710F40C94805EA0E00E9487
:10BCF400D3290E949AB1E8ECE093AF12EE81E2609E
:10BD0400EE83A0918914A23011F00C94A85EA7E1EF
:10BD14000E940D0F8F01E0918C140E94A0B110F0CD
:10BD24000C949B5EA0E00E94FE2BA7E10E94F60EFD
:10BD34000DC0E0918B140E94A0B110F00C94A85E89
:10BD4400A1E00E94FE2BEE81E460EE83A0918D14AD
:10BD5400A23011F00C94C95EA8E10E940D0F8F016E
:10BD6400E09190140E94A0B110F00C94C05EA0E089
:10BD74000E94242AA8E10E94F60E09C0E0918F14C3
:10BD84000E94A0B110F00C94C95E0E94A5B1A091CC
:10BD94009414A23011F00C94EA5EA9E10E940D0FF4
:10BDA4008F01E09197140E94A0B110F00C94E15E11
:10BDB400A0E00E94242AA9E10E94F60E09C0E091A5
:10BDC40096140E94A0B110F00C94EA5E0E94A5B1F2
:10BDD400E0917B14E03011F40C94FF5EAAE00E9421
:10BDE400ACB110F40C94FC5EA0E00E943E26E0E0AE
:10BDF400E0937B14EE81E860EE83A091BC12A23044
:10BE040011F00C94155FA9E00E94B3B110F40C94E6
:10BE1400115FA0E00E943E2CE1E0E093BC12EE81B1
:10BE2400E061EE831FC0A091BC12A33011F00C940A
:10BE34002B5FA9E00E94580F8F010A30E0E01E0733
:10BE440010F40C94275F0E94BAB1EE81E061EE8396
:10BE540009C0E091BC12E03011F00C94345FA0E012
:10BE64000E943E2CA0919E14A23011F00C94445FC9
:10BE7400ADE00E94ACB110F40C94435FE0E0E093B9
:10BE84009E141CC0A0919E14A13011F00C94605F0C
:10BE9400ADE00E94580F8F010430E0E01E0710F45B
:10BEA4000C945D5FA0E00E945A2AE2E0E0939E14A5
:10BEB400ADE00E943C0FEE81E160EE83EE810E94D2
:10BEC400DEB8279608950A930A2F00938714A1E0F9
:10BED4000E94E82AA0918714A13011F00C94745F99
:10BEE4000E94C1B1A0918714A23011F00C947C5F20
:10BEF4000E94C1B1E0918714E03011F00C94855F89
:10BF0400A0E00E94442A099108950A930A2F0093FD
:10BF14008814A0918814A13010F40C94945FE1E08B
:10BF2400E0938814A1E00E94E82AA0918814A1302B
:10BF340011F00C94AA5F0E945E2BE03011F00C9477
:10BF4400AA5FA2E10E94F60EA09188140E94852A9D
:10BF5400A0918814A23011F00C94B05FE091881481
:10BF6400E03011F00C94B95FA0E00E94852A099199
:10BF740008950E943BA540938914313010F40C9429
:10BF8400C55F30938A14213010F40C94CB5F209356
:10BF94008B14E0918A14A0918B14EA0FE0938C1413
:10BFA400413011F00C94DD5FA1E00E94FE2BA4E26D
:10BFB4000E94F60E0DC0A4E20E940D0F8F010D32F7
:10BFC400E1E01E0710F40C94EA5FA0E00E94FE2B4F
:10BFD4000E94DFB8279608950E94E6AD20938D1441
:10BFE400113010F40C94F85F10938E14013010F497
:10BFF4000C94FE5F00938F14E0918F14A0918E1423
:10C00400EA0FE0939014213011F00C940D60A1E03C
:10C014000E94242A03C0A0E00E94242A0E94E1B8BE
:10C02400259608950E94E6AD20939114113010F4E2
:10C034000C941E6010939214013010F40C9424603C
:10C0440000939314213011F00C942C60A1E00E9411
:10C054008D2903C0A0E00E948D290E94E1B8259695
:10C0640008950E94E6AD20939414113010F40C94BA
:10C074003D6010939514013010F40C9443600093C8
:10C084009614E0919514A0919614EA0FE0939714F6
:10C09400213011F00C945260A1E00E94AD2903C03C
:10C0A400A0E00E94AD290E94E1B8259608950A9364
:10C0B4000A2F00939814013011F00C946560A1E0EC
:10C0C4000E94032A03C0A0E00E94032A0991089554
:10C0D4000A930A2F003011F40C947760A1E00E94B7
:10C0E4001B28E1E0E0939A1406C0A0E00E941B28FC
:10C0F400E1E0E0939A14099108950E948AB1E2E084
:10C10400E0939A140895E3E0E0939A1408950A934F
:10C114000A2F00939914099108951A930A931A2FD8
:10C124000E9490B10E2F013011F40C949E600230E5
:10C1340011F40C949E6020C0113011F00C94AC608A
:10C14400A0E00E942D28A1E00E944328E1E0E093B2
:10C154009B140FC0123011F00C94B6600E94C8B149
:10C16400E1E0E0939B1405C00E94CEB1E0E0E093CF
:10C174009B14A4E10E94F60E0991199108950A9363
:10C184000E9490B10E2F013011F40C94CE60023055
:10C1940011F40C94CE6008C0A1E00E944328A0E0F2
:10C1A4000E942D280E94D4B1099108950A930E94F7
:10C1B40090B10E2F013011F40C94E560023011F4AB
:10C1C4000C94E56004C00E94C8B10E94D4B10991E6
:10C1D4000895A1E00E942C2DAAE10E94F60E089574
:10C1E4000A930E9495B10E2F013010F40C9405614E
:10C1F4000E94452DA1E00E94D329ABE10E94F60ED6
:10C20400E0E0E0939D14099108950A930E9490B18F
:10C214000E2F013010F40C9426610E94082BE0309C
:10C2240011F40C941A61A1E00E94E82A0E9453AB15
:10C234000E94982BE03011F40C942361E1E0099101
:10C244000895E0E009910895E1E0099108950A93C1
:10C254000E94DDB10E2F013010F40C9448610E944D
:10C26400082BE03011F40C943C61A1E00E94E82A10
:10C274000E9453AB0E94A62BE03011F40C9445614C
:10C28400E1E009910895E0E009910895E1E0099160
:10C2940008950A930E94082BE03011F40C94546121
:10C2A4000E94E2B10E94282B0E2F013011F00C9451
:10C2B4005E61E1E009910895E0E0099108950A932F
:10C2C4000E94082BE03011F40C946A610E94E2B1E0
:10C2D4000E94222D0E2F003011F00C947461E0E0C6
:10C2E40009910895E1E0099108950E94082BE03036
:10C2F40011F40C947F610E94E2B10E94DA2BE030C9
:10C3040011F40C948761E1E00895E0E008951A9334
:10C314000A9310E00E94082BE03011F40C9494610D
:10C324000E94E2B10E94282B0E2F013011F00C94D0
:10C334009C6111600E94222D0E2F013011F00C948B
:10C34400A46112600E94DA2B0E2F003011F00C94BD
:10C35400AC611460E12F099119910895E1E0E09333
:10C364007B14A1E00E943E26AAE00E943C0F08959F
:10C374000A93E1E0E093BC120E94E9B10E2F013070
:10C3840010F40C94C861E2E00E94EEB109910895A2
:10C394000A93E3E00E94EEB1099108950E94BAB1B4
:10C3A4000895E091BC1208950A930A2FE0919E1417
:10C3B400E03011F00C94EF61013010F40C94E6615C
:10C3C400A1E00E945A2A03C0A2E00E945A2AE1E096
:10C3D400E0939E14ADE00E943C0F099108950895E6
:10C3E400E0E00895BA93AA93EF97AD970E94D7B867
:10C3F400FE01EC58FF4F0190F081E02DDE01A059C1
:10C40400BF4FED93FC93FE01EE58FF4F0190F08176
:10C41400E02DDE01A259BF4FED93FC930E9490B131
:10C424005E2FDE01A059BF4FAC910E94CC71FE017A
:10C43400E059FF4F0190F081E02DEA30A0E0FA07C7
:10C4440011F00C9428620E94F55AE4C2E436A0E08C
:10C45400FA0711F00C943A620E94F6B12E2FE1E033
:10C46400EA93ADB7BEB72F930E949A712F91D2C2AF
:10C47400E936A0E0FA0711F00C9450620E94FBB177
:10C48400EA8FE8E0EB8F0E9400B2EC8FE2E0ED8FE0
:10C49400E0E0EE8FE4E00E9405B2BCC2EB30A0E025
:10C4A400FA0711F00C9459620E94075BB3C2EC3096
:10C4B400A0E0FA0711F00C9462620E94385BAAC2F1
:10C4C400E536A0E0FA0711F00C9476620E940AB2F5
:10C4D400EDB7FEB7FA93EA932F93A2E40E94455B6B
:10C4E4002F910E940FB296C2E636A0E0FA0711F02F
:10C4F4000C948A620E940AB2EDB7FEB7FA93EA93EB
:10C504002F93A2E40E94025A2F910E940FB282C27A
:10C51400E736A0E0FA0711F00C949E620E940AB27A
:10C52400EDB7FEB7FA93EA932F93A2E40E947859E9
:10C534002F910E940FB26EC2E836A0E0FA0711F004
:10C544000C94BB62DE01A45ABF4F0E94074D3E2FDC
:10C55400E0E0DE01AD59BF4FEC93303011F00C94A4
:10C56400BA62E8E0EA93DE01A35ABF4F0E949A71CF
:10C5740051C2E331A0E0FA0711F00C94C4620E94A6
:10C58400275C48C2EA36A0E0FA0711F00C94F06286
:10C594000E94D2510E94D5ADEA8F0E94DBADEB8F91
:10C5A4000E949F510E94D5ADEC8F0E94DBADED8FB0
:10C5B400A0E00E940A520E94D5ADEE8F0E94DBAD2E
:10C5C400EF8FA1E00E940A520E94D5ADE8A30E9419
:10C5D400DBADE9A3E8E00E9405B21CC2EE30A0E0A6
:10C5E400FA0711F00C943363A8EAB0E00E947FBA12
:10C5F400EA8F0E9490B1EB8FAAEAB0E00E947FBA62
:10C60400EC8FABEAB0E00E947FBAED8FACEAB0E009
:10C614000E947FBAEE8FADEAB0E00E947FBAEF8F3E
:10C62400AEEAB0E00E947FBAE8A30E9495B1E9A304
:10C63400A0EBB0E00E947FBAEAA30E94DDB1EBA3B5
:10C64400A2EBB0E00E947FBAECA30E94E9B1EDA393
:10C65400A4EBB0E00E947FBAEEA3EDE00E9405B225
:10C66400D9C1E131A0E0FA0711F00C9487630E946C
:10C67400F2B00E9414B2EA8F0E94F2B00E9419B282
:10C68400EB8F0E9400B10E9414B2EC8F0E9400B1A3
:10C694000E9419B2ED8F0E9405B10E9414B2EE8F70
:10C6A4000E9405B10E9419B2EF8F0E940AB10E9444
:10C6B40014B2E8A30E940AB10E9419B2E9A30E942D
:10C6C4000FB10E9414B2EAA30E940FB10E9419B2E2
:10C6D400EBA340E0403210F00C948363E42FE65F58
:10C6E400F0E0DE015A96EA0FFB1F0F01A8E8B0E064
:10C6F400EE27A40FBE1F0E947FBAD001EC934F5FB8
:10C70400E9CFEAE20E9405B285C1E231A0E0FA076E
:10C7140011F00C94A263DE0116960E94864F3E2F00
:10C72400303011F00C949D63E8E0EA93DE01179633
:10C734000E949A7104C0E2E00E941EB208956AC188
:10C74400EF36A0E0FA0711F00C94AF630E946C4F2F
:10C75400EA8FE1E00E9405B25DC1E431A0E0FA078E
:10C7640011F00C94C3630E9423B2FA93EA930E94DB
:10C774002AB2DE015E960E942F0DE0E40E9405B20B
:10C7840049C1E531A0E0FA0711F00C94E1630E947D
:10C7940023B20E9427B10E942AB2DE0190960E9421
:10C7A400EE803E2F303011F00C94DC63E0E40E9404
:10C7B40005B204C0E2E00E941EB208952BC1EB361C
:10C7C400A0E0FA0711F00C94FA630E942FB20E94C1
:10C7D40032B20E941A38EA8F0E94132DEB8F0E9406
:10C7E4008E27EC8FE1E0EC8FE3E00E9405B212C1EA
:10C7F400E631A0E0FA0711F00C941F640E942FB2F6
:10C804000E9432B2E0919F14EA8FE091A014EB8F62
:10C81400A0919F140E944D39EC8FA0919F140E9407
:10C824005C39ED8FE0919F14EA93DE015F960E94DC
:10C834006639E8E20E9405B2EDC0E731A0E0FA07EC
:10C8440011F00C943F64533011F00C942E64DE010B
:10C854005A960E94DB420DC0513011F40C94376497
:10C86400523011F40C94376404C0DE015A960E94CD
:10C87400F83EE0E40E9405B2CDC0EC36A0E0FA0731
:10C8840011F00C947F640E942FB20E9432B2533094
:10C8940011F00C9460640E9454430E9436B20E94CA
:10C8A4003DB2E42FEE5FF0E00E94AFA70E9443B2D6
:10C8B4000E944BB20E9457434B5F1BC0513011F48E
:10C8C4000C946964523011F40C94696412C00E948F
:10C8D400613F0E9436B20E943DB2E42FEE5FF0E069
:10C8E4000E94AFA70E9443B20E944BB20E94643FD1
:10C8F4004B5FE8E00E9405B28DC0ED36A0E0FA0778
:10C9040011F00C948A640E942FB20E9432B282C049
:10C91400E831A0E0FA0711F00C949A64203011F089
:10C924000C94956404C0E4E00E941EB2089572C0A1
:10C93400E931A0E0FA0711F00C94BA640E942FB216
:10C944000E9432B2E4E2F6E060E070E00E946ABA6B
:10C95400FE017E960E9453B2E0E0DE01A55ABF4F6D
:10C96400EC93DE015A960E94171A0E9405B252C037
:10C97400EE36A0E0FA0711F00C94CB640E942FB2BB
:10C984000E9432B20E9459B22F5FE8E00E9405B2C1
:10C9940041C0EA31A0E0FA0711F00C94DD640E9472
:10C9A4002FB20E9432B2DE015A960E94BC4C2E2F46
:10C9B4000E940FB22FC0EB31A0E0FA0711F00C94E3
:10C9C40008650E942FB20E9432B20E94DFAEE0E0FE
:10C9D400EA930E9445AF0E9459B2DE0116960E9466
:10C9E400BC4C2E2F0E94DFAE0E945AAFFE017E96F1
:10C9F400FA93EA93EAE0F0E0FA93EA93AAE0B0E06B
:10CA04000E94A01BE6E10E9405B204C0E1E00E947E
:10CA14001EB20895E0E00E941EB208950895E0E079
:10CA24000895BA93AA932D97D1500E94D7B8FE01C6
:10CA3400E85EFE4F0190F081E02DDE01AF5EBE4F57
:10CA4400ED93FC93FE01EA5EFE4F0190F081E02D30
:10CA5400DE01A15FBE4FED93FC93FE01EB5EFE4F42
:10CA64005081FE01E153FF4F0E9440AFA0E4B0E0CB
:10CA74000E94F31B0E942AB2DE01A95EBE4FAC9154
:10CA8400BB270E9459225E2F20E0251710F00C943A
:10CA94005F65E22F0E9462B2EA0FFB1FBF01DE0155
:10CAA400AD5EBE4F0D90BC91A02DEE27A20FBE1F10
:10CAB400EC91DB01EC932F5FE8CF0E9490B1EAA7E1
:10CAC400DE01AF5EBE4F0D90BC91A02DA130E0E120
:10CAD400BE0710F40C947165E0E0E887E987FE0175
:10CAE400EF5EFE4F0190F081E02DEA30A0E0FA07FE
:10CAF40011F00C949565E0E4F6E060E070E00E94CB
:10CB04006ABADE01AD52BF4F0E9405204E2F40305D
:10CB140011F40C9490650E94200D04C0E2E00E9480
:10CB240067B2089579C5E436A0E0FA0711F00C94D1
:10CB3400A0650E946CB20E94BB5F6EC5E536A0E0A2
:10CB4400FA0711F00C94A76567C5E636A0E0FA076A
:10CB540011F00C94B2650E946CB20E94EE5F5CC549
:10CB6400E736A0E0FA0711F00C94BD650E946CB2A0
:10CB74000E94146051C5E836A0E0FA0711F00C9445
:10CB8400C8650E946CB20E94336046C5E936A0E0D5
:10CB9400FA0711F00C94D3650E9479B20E9459608F
:10CBA4003BC5EA36A0E0FA0711F00C94DA6534C507
:10CBB400EB36A0E0FA0711F00C94E5650E9479B217
:10CBC4000E943E2C29C5EC36A0E0FA0711F00C9423
:10CBD400F0650E9479B20E941E2C1EC5ED36A0E0BD
:10CBE400FA0711F00C94FB650E9479B20E94322678
:10CBF40013C5EE36A0E0FA0711F00C9406660E9405
:10CC040079B20E94702808C5E231A0E0FA0711F059
:10CC14000C9421660E94E2A60E94A7280E947EB27C
:10CC24000E94D5280E9483B20E9403290E9488B2E0
:10CC34000E9431290E948DB20E945F29EDC4E33124
:10CC4400A0E0FA0711F00C943C660E94E2A60E9450
:10CC5400BF280E947EB20E94ED280E9483B20E94E7
:10CC64001B290E9488B20E9449290E948DB20E9409
:10CC74007729D2C4EF36A0E0FA0711F00C94476686
:10CC84000E9479B20E94E82AC7C4E431A0E0FA07FE
:10CC940011F00C947D660E9492B2DE01A752BF4F40
:10CCA400AC910E945A4E4E2F0E94A0B20E9488B2AC
:10CCB4000E94A6B28F010A93FE01EB52FF4FE0815E
:10CCC400EA93DE01A952BF4FAC910E94E74E3E2F7A
:10CCD400403011F00C947366303011F00C9473668C
:10CCE40001C004C0E0E00E9467B20895E1E00E9440
:10CCF40067B2089591C4E531A0E0FA0711F00C94ED
:10CD040090660E9492B2DE01AB52BF4FAC910E947A
:10CD14005A4E4E2F0E9467B208957EC4E631A0E0B9
:10CD2400FA0711F00C94AA660E94ACB20E94A6B253
:10CD34008F010A93FE01EE52FF4FE081EA930E94B5
:10CD44008DB20E94E74E4E2F0E9467B2089564C4CC
:10CD5400E037A0E0FA0711F00C94C0660E94B3B269
:10CD640041E0323010F00C94BB66A32F0E94394F7F
:10CD74004E2FE42F0E9467B208954EC4E137A0E01D
:10CD8400FA0711F00C94C76647C4E237A0E0FA072B
:10CD940011F00C94CE6640C4E337A0E0FA0711F01A
:10CDA4000C94D9660E9479B20E94655F35C4E43759
:10CDB400A0E0FA0711F00C94E4660E9479B20E9494
:10CDC400875F2AC4E537A0E0FA0711F00C94ED66FA
:10CDD4000E94EB6021C4E637A0E0FA0711F00C943E
:10CDE400F8660E9479B20E94D32916C4E737A0E0FE
:10CDF400FA0711F00C9401670E94F2600DC4E73148
:10CE0400A0E0FA0711F00C94BC670E94B3B2323070
:10CE140010F40C940E6731E0E32FA8EAB0E00E940E
:10CE24009BBAFE01E053FF4F3081343010F40C9470
:10CE34001C6731E0A9EAB0E0E32F0E949BBAFE012F
:10CE4400EF52FF4F3081323010F40C942A6731E0F6
:10CE5400AAEAB0E0E32F0E949BBAFE01EE52FF4F14
:10CE64003081323010F40C94386730E0ABEAB0E033
:10CE7400E32F0E949BBAFE01ED52FF4F3081313007
:10CE840010F40C94466730E0ACEAB0E0E32F0E9463
:10CE94009BBAFE01EC52FF4F3081313010F40C94F8
:10CEA400546730E0ADEAB0E0E32F0E949BBAFE0184
:10CEB400EB52FF4F3081313010F40C94626730E054
:10CEC400AEEAB0E0E32F0E949BBAFE01EA52FF4FA4
:10CED4003081313010F40C94706730E0AFEAB0E088
:10CEE400E32F0E949BBAFE01E952FF4F308131309B
:10CEF40010F40C947E6730E0A0EBB0E0E32F0E94C6
:10CF04009BBAFE01E852FF4F3081313010F40C948B
:10CF14008C6730E0A1EBB0E0E32F0E949BBAFE01E6
:10CF2400E752FF4F3081313010F40C949A6730E0AF
:10CF3400A2EBB0E0E32F0E949BBAFE01E652FF4F42
:10CF44003081313010F40C94A86730E0A3EBB0E0EA
:10CF5400E32F0E949BBAFE01E552FF4F308131302E
:10CF640010F40C94B66730E0A4EBB0E0E32F0E9419
:10CF74009BBA52C3EB30A0E0FA0711F00C941A6884
:10CF84000E94ACB20E94BB208F01ACE7B0E00E94CB
:10CF940093BAFE01EE52FF4FE081EA930E9483B2FE
:10CFA4000E94BB208F01AEE7B0E00E9493BAFE015D
:10CFB400EC52FF4FE081EA930E948DB20E94BB20A5
:10CFC4008F01A0E8B0E00E9493BAFE01EA52FF4F3D
:10CFD400E081EA93DE01AA52BF4FAC910E94BB20CC
:10CFE4008F01A2E8B0E00E9493BAFE01E852FF4F1D
:10CFF400E081EA93DE01A852BF4FAC910E94BB20AE
:10D004008F01A4E8B0E00E9493BA20E0203210F02F
:10D014000C941968A8E8B0E0E22F0E94CCA8E22F93
:10D02400E65F0E9462B20E949EAC2F5FEFCFF4C213
:10D03400E837A0E0FA0711F00C942C680E9479B24A
:10D04400A13010F40C9429680E94423802C00E9456
:10D054003038E2C2E937A0E0FA0711F00C943568E1
:10D064000E940F38D9C2EA37A0E0FA0711F00C94F5
:10D0740040680E9479B20E946038CEC2EB37A0E0CB
:10D08400FA0711F00C9450680E94B8B20E94DDA611
:10D09400EA930E947EB20E94F138BEC2EC30A0E056
:10D0A400FA0711F00C9460680E94B8B20E9492B220
:10D0B400DE01AB52BF4F0E940439AEC2E831A0E09A
:10D0C400FA0711F00C94C1680E94ACB20E94BB2014
:10D0D4008F01E3E0F0E0E887F987E0E0EE83EF8397
:10D0E400AE81BF81509710F00C94A068EE81FF814F
:10D0F400DE011A960E94C5ADFF93EF93E885F9858A
:10D104003196DE01A153BF4FAE0FBF1FEC91EA93DE
:10D11400E985FA85DE01A053BF4FAE0FBF1FAC9166
:10D124000E94BB20AF91BF91ED93FC93E885F985F4
:10D134003296E887F9870E9495A5D2CFAAA5A33095
:10D1440011F00C94AE681A930A930E94A0B2DE0107
:10D154001D960E943E4212C0AAA5A13011F40C945F
:10D16400B868A23011F40C94B86808C01A930A93F2
:10D174000E94A0B2DE011D960E94F53D4DC2EC371F
:10D18400A0E0FA0711F00C94E068AAA5A33011F00E
:10D194000C94D1680E9479B20E9470420EC0AAA574
:10D1A400A13011F40C94DB68A23011F40C94DB6808
:10D1B40004C00E9479B20E946C3E2EC2ED37A0E0FA
:10D1C400FA0711F00C94FB68AAA5A33011F00C9493
:10D1D400EE680E9489420CC0AAA5A13011F40C94F7
:10D1E400F868A23011F40C94F86802C00E94903ED2
:10D1F40013C2EE37A0E0FA0711F00C941669AAA541
:10D20400A33011F00C9409690E94C4420CC0AAA571
:10D21400A13011F40C941369A23011F40C94136925
:10D2240002C00E94DA3EF8C1EF37A0E0FA0711F01D
:10D234000C941D69F1C1E038A0E0FA0711F00C94D8
:10D244002469EAC1E138A0E0FA0711F00C942F69CF
:10D254000E9479B20E946A60DFC1E238A0E0FA0756
:10D2640011F00C943C690E9479B20E9489600E947A
:10D274007F60D2C1E338A0E0FA0711F00C94496949
:10D284000E94E2A60E9489600E948560C5C1E438BC
:10D29400A0E0FA0711F00C9467690E94DDA6E17022
:10D2A40011F40C945969A1E00E948F600DC00E9492
:10D2B400DDA6E27011F40C946369A2E00E948F6011
:10D2C40003C0A0E00E948F60A7C1E538A0E0FA0780
:10D2D40011F00C9470690E94C1609EC1E638A0E010
:10D2E400FA0711F00C9479690E94D86095C1E73867
:10D2F400A0E0FA0711F00C948B690E94B3B2A32F3B
:10D304000E94D92CA1E00E946026A1E00E94802600
:10D3140083C1E838A0E0FA0711F00C9496690E94E2
:10D3240079B20E94D32678C1E938A0E0FA0711F057
:10D334000C94A3690E9479B20E94012D0E94C6B286
:10D344006BC1EA38A0E0FA0711F00C94AE690E94B0
:10D3540079B20E94362760C1EB38A0E0FA0711F0D9
:10D364000C94C3690E9479B2A13011F00C94BD6988
:10D374000E94014502C00E941845E0E0E093A11418
:10D384004BC1E931A0E0FA0711F00C94EF69FE01FA
:10D39400EA52FF4FE0810E94CCB2FE01EB52FF4FF4
:10D3A400E0810E94CCB2FE01EC52FF4FE0810E946A
:10D3B400CCB2FE01ED52FF4FE081FF2766277727AD
:10D3C400EBA7FCA76DA77EA70E94DFB2ADA5BEA503
:10D3D4008FA598A90E946E491FC1EA31A0E0FA07FF
:10D3E40011F00C94FE690E9492B2DE01AB52BF4F61
:10D3F400AC910E94514B10C1EB31A0E0FA0711F03F
:10D404000C94196A0E94ACB20E94BB20DF010E94F6
:10D41400884B0E947EB20E94F0450E9483B20E9413
:10D424004B460E9488B2BB270E949148F5C0EC3855
:10D43400A0E0FA0711F00C94376A0E94E2A6A1302A
:10D4440011F00C942B6A0E9479B2BB270E945145BB
:10D454000BC00E94E2A6A23011F00C94366A0E941E
:10D4640079B2BB270E946B45D7C0ED38A0E0FA071C
:10D4740011F00C944D6A0E94DDA6EA930E947EB2DC
:10D484000E9485450E947EB20E94C0450E9483B2DC
:10D494000E94D845C1C0EE38A0E0FA0711F00C9400
:10D4A400606A0E9479B20E9403460E94E2A60E942A
:10D4B40033460E947EB20E941B46AEC0EF38A0E005
:10D4C400FA0711F00C946B6A0E9479B20E941C4511
:10D4D400A3C0ED30A0E0FA0711F00C947B6AFE01C2
:10D4E400E153FF4FFA93EA93A52FBB270E948015BF
:10D4F40093C0E039A0E0FA0711F00C94866A0E9408
:10D5040079B20E94D24888C0E139A0E0FA0711F04C
:10D514000C948F6A0E94FC487FC0EE30A0E0FA07AA
:10D5240011F00C94B76AFE01ED52FF4F308120E0F8
:10D53400231710F00C94AD6AE22FF0E0DE019F9601
:10D54400EA0FFB1F0F01E22FEB5F0E9462B20E9401
:10D5540026A72F5FEDCF0E94DFB2FE01F196FA936A
:10D56400EA93A32F0E949B4657C0EF30A0E0FA072E
:10D5740011F00C94C96AA091A114A33010F00C947A
:10D58400C86AE091A114EF5FE093A11445C0E239A9
:10D59400A0E0FA0711F00C94D06A3EC0E339A0E091
:10D5A400FA0711F00C94DF6A0E94E2A60E948A46F0
:10D5B4000E9479B20E9479462FC0E031A0E0FA07B8
:10D5C40011F00C94EA6AE42F0E9467B2089524C013
:10D5D400E131A0E0FA0711F00C94F56AE42F0E94FF
:10D5E40067B2089519C0E439A0E0FA0711F00C9469
:10D5F400FC6A12C0E231A6E3FA0711F00C94036B43
:10D604000BC0EC31A0E0FA0711F00C940A6B04C0D3
:10D61400E1E00E9467B20895FE01E15FFE4F0190D0
:10D62400F081E02DDE01A15FBE4FED93FC93E0E0BD
:10D634000E9467B208951A930A938D01E2E0EC9375
:10D64400099119910895EA97E0E0EFAB20E030E00A
:10D6540040E050E0E4B7EEABFE01F596EBABFCAB7B
:10D66400ABA9BCA90E941D6BABA9BCA90C91112745
:10D674009924E0E0F2E03E2E4F2EE4E3F2E17E2E28
:10D684008F2EE72DF82DA32DB42DED93FC93E2E01E
:10D69400F0E03E0E4F1EE72DF82DEF5FFE4F7E2E7D
:10D6A4008F2EEEEFF1E23E164F0610F00C945B6BFA
:10D6B400E8CFE0E0F2E03E2E4F2EE4E3F2E17E2EEE
:10D6C4008F2EA32DB42D5D906C907514860411F4E7
:10D6D4000C946E6BE1E09E2EE2E0F0E03E0E4F1EF5
:10D6E400E72DF82DEF5FFE4F7E2E8F2EEEEFF1E249
:10D6F4003E164F0610F00C94806BE3CFE0E0F2E0AE
:10D704003E2E4F2EA32DB42DE0E0F0E0ED93FC93DC
:10D71400E2E0F0E03E0E4F1EEEEFF1E23E164F0661
:10D7240010F00C94966BEECF0E94FB74E4B7E09378
:10D73400BA12992011F00C94A36BE1E0E093A112CA
:10D7440003C0E8ECE093A112E0E0E5BFE5BFE0E848
:10D75400E0936100E0E0E0936100E3BF0E944A0CC3
:10D764000E94070D7894E1E0E0937C14A6E8B0E011
:10D774000E947BBA9F01EAE3FCE5E217F30711F488
:10D784000C947D6CA6E8B0E00E9493BAACE7B0E0DC
:10D79400E9E1F1E00E9493BAAEE7B0E0E8EEF3E02D
:10D7A4000E9493BAA0E8B0E0E1E0F0E00E9493BAEE
:10D7B400A2E8B0E00E9493BAA4E8B0E0E8EEF3E097
:10D7C4000E9493BAECE4F6E060E070E00E946ABA6A
:10D7D400DE0115960E940B1CE0E0EA83FE013196FF
:10D7E400FA93EA93E8E8F0E0FA93EA93A0E2B0E06F
:10D7F4000E94561BA6EBB0E0E1E00E949BBAA7EBA7
:10D80400B0E0E5E00E949BBAA8EBB0E0E0E00E9443
:10D814009BBAA9EBB0E0E3E00E949BBAAAEBB0E0AC
:10D82400E0E00E949BBAA8EAB0E0E1E00E949BBA63
:10D83400A9EAB0E00E949BBAAAEAB0E00E949BBAAF
:10D84400ABEAB0E0E0E00E949BBAACEAB0E0E1E011
:10D854000E949BBAADEAB0E0E0E00E949BBAAEEA57
:10D86400B0E0E1E00E949BBAAFEAB0E0E0E00E94E1
:10D874009BBAA0EBB0E0E1E00E949BBAA1EBB0E060
:10D88400E0E00E949BBAA2EBB0E00E949BBAA3EB3B
:10D89400B0E0E1E00E949BBAA4EBB0E00E949BBA26
:10D8A400ACEBB0E0EFEFFFEF0E9493BAAEEBB0E069
:10D8B400E0E00E949BBAA2EDB0E0E4EFF2E00E9447
:10D8C40093BAA0EDB0E0EAE7F1E00E9493BAAEECBF
:10D8D400B0E0EDEBF0E00E9493BAACECB0E0ECE425
:10D8E400F0E00E9493BAAAECB0E0E6E2F0E00E9415
:10D8F40093BA0E943EA4A3EBB0E0E0E00E949BBA7E
:10D90400ABEAB0E00E949BBA0E949D250E94A40E3F
:10D91400A1E00E94D125A1E00E94B22C0E94757A58
:10D92400EEABAEA9A13010F40C949C6CE953E093D7
:10D93400A51203C0E1E0E093A5120E94DE2DEFAB37
:10D94400E03011F40C94B36CE2E0E0937C140E9498
:10D95400012EA92D0E94552EEEABAEA90E941530C2
:10D96400FCCFE3E0E0937C140E948D360E944238A1
:10D97400A9EAB0E00E947FBAE883A881A33011F03D
:10D984000C94C76C0E9459400CC0A881A13011F4BA
:10D994000C94D16CA23011F40C94D16C02C00E948E
:10D9A400BE3B0E94165D0E9471440E941C710E943D
:10D9B40014860E94F6500E94AD0F0E94FF4C0E94F4
:10D9C400837CE4E0E0937C140E94B8900E94157577
:10D9D4000E947A760E942875E5E0E0937C140E9408
:10D9E4007E700E94F2500E94E8530E9470A20E942E
:10D9F4005152A4E00E943C0FA3E00E943C0FE1E0DE
:10DA0400E0937814E0E0E0937514E0937614E093E7
:10DA14007714E1E0E0937914E0E0E0937B14E09381
:10DA24007A14E0938314ACE00E94F60EE2E0EA93E9
:10DA3400E5E0EA93E3E0EA93E0E0EA93A0E00E9401
:10DA4400F113E1E0E093C814E0E0E093C9147894A2
:10DA5400A1E00E94F60EA8E00E943C0F0E94E40E92
:10DA6400E03011F00C94396D0E94A40E7894E0E03B
:10DA7400E0937D14E0937E14E0937F14E09380148C
:10DA8400E0938114E0938214A3E00E94580F8F0165
:10DA9400ABEAB0E00E947FBAEFABE03011F40C9433
:10DAA4005C6DE0E0E0937614E0917D14E260E09335
:10DAB4007D1403C0E1E0E09376140A30E0E01E0731
:10DAC40010F00C946D6DE0E0E0937614E0917D1419
:10DAD400E460E0937D14A4980E94AD25EFABE030A0
:10DAE40011F40C947D6DE0E0E0937614E0917D14E4
:10DAF400E860E0937D140E94415DEFABAFA9A130D3
:10DB040010F40C948B6DE0E0E0937614EFA9E093AD
:10DB14008014A091C9140E944051EFABE03011F47D
:10DB24000C949C6DE0E0E0937614E0917D14E06247
:10DB3400E0937D140E944871EFABE03011F40C9433
:10DB4400AB6DE0E0E0937614E0917D14E064E09343
:10DB54007D140E941165EFABE03011F40C94BA6DA2
:10DB6400E0E0E0937614E0917D14E068E0937D14A6
:10DB74000E94F261EFABE03011F40C94C96DE0E067
:10DB8400E0937614AEE7B4E1EC91E160EC930E948B
:10DB94007244EFABE03011F40C94D86DE0E0E09304
:10DBA4007614AEE7B4E1EC91E260EC930E946986EE
:10DBB400EFABE03011F40C94EB6DE0E0E0937614FD
:10DBC400AEE7B4E1EC91E460EC93E1E0E09383141C
:10DBD40003C0E0E0E0938314A091C9140E94367559
:10DBE400EFABE03011F40C94FF6DE0E0E0937614B9
:10DBF400AEE7B4E1EC91E860EC930E940137EFAB3F
:10DC0400E03011F40C940E6EE0E0E0937614AEE78D
:10DC1400B4E1EC91E061EC93A9EAB0E00E947FBA30
:10DC2400E883A881A33011F00C94286E0E947D40F3
:10DC3400EFABE03011F40C94276EE0E0E09376143F
:10DC4400AEE7B4E1EC91E062EC9319C0A881A13095
:10DC540011F40C94326EA23011F40C94326E0FC095
:10DC64000E94F03BEFABE03011F40C94416EE0E025
:10DC7400E0937614AEE7B4E1EC91E064EC930E9497
:10DC8400064DA091C9140E949C7CEFABE03011F4C6
:10DC94000C94546EE0E0E0937614AEE7B4E1EC91BA
:10DCA400E068EC930E94F979A09183140E94BC90DF
:10DCB400EFABE03011F40C94676EE0E0E09376147F
:10DCC400AFE7B4E1EC91E068EC930E941626EFAB69
:10DCD400E07111F40C94786EE0E0E0937614AFE711
:10DCE400B4E1EC91E160EC930E945986EFA9E072F3
:10DCF40011F40C948D6EE0E0E0937614AFE7B4E198
:10DD0400EC91E260EC930E942075E23010F00C94E8
:10DD14008D6E0E945986EFA9E07411F40C949A6EEA
:10DD2400E0E0E0937614AFE7B4E1EC91E460EC93C7
:10DD3400EFA9E07811F40C94A76EE0E0E093761478
:10DD4400AFE7B4E1EC91E860EC930E947C52EFAB56
:10DD5400E03011F40C94B66EE0E0E0937614AFE793
:10DD6400B4E1EC91E061EC930E9488A2EFABE03067
:10DD740011F40C94C56EE0E0E0937614A1E8B4E1EC
:10DD8400EC91E160EC930E943954EFABE03011F474
:10DD94000C94D46EE0E0E0937614A1E8B4E1EC9145
:10DDA400E260EC930E948961EFABAFA9A13010F45B
:10DDB4000C94E06EE853E093B51203C0E1E0E09305
:10DDC400B512EFA9E17011F40C94F06EE0E0E09369
:10DDD4007614AFE7B4E1EC91E061EC93EFA9E27063
:10DDE40011F40C94FD6EE0E0E0937614AFE7B4E137
:10DDF400EC91E062EC93EFA9E47011F40C940A6FD7
:10DE0400E0E0E0937614AFE7B4E1EC91E064EC93E6
:10DE1400E0917614E03011F00C94136FA4E00E94AA
:10DE24003C0FA0917714A43011F00C941E6FE1E024
:10DE3400F0E0E8AFF9AF0FC0A0917714A13011F072
:10DE44000C94296FEEE1F0E0E8AFF9AF04C0E3E031
:10DE5400F0E0E8AFF9AFA4E00E94580F8F01E8ADFD
:10DE6400F9AD0E171F0710F40C943F6FA0E00E9449
:10DE74003E260E94EB6F00E010E00E9490500E944A
:10DE8400597CA1E00E94B22CACE00E940D0F8F01DE
:10DE94000536E0E01E0710F40C94536FACE00E94CA
:10DEA400F60EDCCD9901AA01EA96FFCFE0E0E3BFCC
:10DEB4000E94740C0E944E70E1E0E0937914E093A8
:10DEC4007714AEE4B6E080E090E00E9460950E9492
:10DED400B0610E9414860895E0E0E3BF0E94A20CA2
:10DEE4000E944E70E1E0E0937914E2E0E09377144D
:10DEF400ABE5B6E080E090E00E9460950E94B061DE
:10DF04000895E0E0E3BF0E94D00C0E944E70E2E06E
:10DF1400E0937914E3E0E0937714A9E6B6E080E0B7
:10DF240090E00E94609508950A93E0E0E3BF0E94A8
:10DF3400FE0CE3E0E0937914E4E0E09377140E94AC
:10DF44003670E091CA14EF5FE093CA14E091CB14E9
:10DF5400EF5FE093CB14A091CA14A93310F40C948E
:10DF6400C56FA6E7B6E080E090E00E946095E7E028
:10DF7400E0937714A1E00E94DB25E0E0E093CA146B
:10DF84000E94B0610CC0A091CA14A83310F40C9480
:10DF9400D16FA1E00E94DB25E6E0E09377140E94B4
:10DFA40089610E2F013010F40C94DD6F0E94B06172
:10DFB400E5E0E09377140991089508950E94F4111F
:10DFC4000895089508950E94E8B208950E94E8B261
:10DFD4000895F894AEE8B6E080E090E00E94609581
:10DFE400A1E00E94F725A0E00E94D125A0E00E94B4
:10DFF400DB25E0E0E0937714E09378140E942C5D35
:10E004000E9430380E94FC0F0E94EF0D0E94F01213
:10E014000E948C140E9479160E94DC17E0E9E0BF8C
:10E024000E94ED0B0E94F20D0E94AF25A0E00E9419
:10E03400722CE0E8E0936100E8E0E0936100A2E084
:10E044000E944F0CA2E00E947D0CA2E00E94AB0C47
:10E05400A2E00E94D90CE0E0EBB9EAB978940E94FE
:10E064007EA40E9482A408950E94F5B20E947E704C
:10E07400A4E00E943C0FE0E0E0937814E0937A146B
:10E084000E94A40E78940E949990A9E9B6E080E0D9
:10E0940090E00E94609508950E94F5B2A1E00E946C
:10E0A400D1250E947E700E94837C0E948D360E943E
:10E0B4004238A1E00E94F60EA4E00E943C0FA1E0C9
:10E0C4000E94B22C0E94F6500E94A40D0E94AD0F33
:10E0D400E1E0E0937814E0E0E0937A140E94F20D1A
:10E0E4000E94A40E78940E949990A4EAB6E080E07D
:10E0F40090E00E94609508950E94D8B80E94F6B1FD
:10E104000E2F023010F40C948C70A6EBB0E0E1E01A
:10E114000E949BBA0E94FBB11E2F113010F40C9484
:10E124009870193010F00C94987006C0A7EBB0E00A
:10E13400E2E00E949BBA12E00E9400B22E2F2F341C
:10E1440011F40C94AE702E3411F40C94AE7025348A
:10E1540011F40C94AE7001C006C0A8EBB0E0EEE47C
:10E164000E949BBA2EE40E94FBB1E53011F40C949A
:10E17400C070A7EBB0E0E5E00E949BBA0E9400B239
:10E18400EE3411F40C94CB70A8EBB0E0EEE40E94F2
:10E194009BBAE12FE03011F00C94D27040E025C01E
:10E1A400E13011F00C94D87041E01FC0E23011F05E
:10E1B4000C94DE7042E019C0E33011F00C94E4706A
:10E1C40043E013C0E43011F00C94EA7044E00DC055
:10E1D400E53011F00C94F07045E007C0E63011F022
:10E1E4000C94F67046E001C040E0E22FE53411F0F3
:10E1F4000C94FE7031E00DC0EF3411F00C940471F6
:10E2040032E007C0EE3411F00C940A7130E001C022
:10E2140030E00E94FCAD0E946912A1E00E946026D9
:10E224000E94F1610E9410650E94C1A90E94DFB89A
:10E23400259608950A930E947E70E1E0E0932315E9
:10E244000E94011300E0043510F00C943171E02FAA
:10E25400F0E0E453FB4EA0E0A0830F5FF4CFE0E0D6
:10E26400E0932015E0932115E09322150E94C02B22
:10E27400E09324150E94DA2BE0932515E0E0E09367
:10E28400C015A6E00E943C0F099108950E94DAB8D7
:10E2940000E00E94DB710E2FA2E0B0E00E947E0E2F
:10E2A400013011F00C946F71E1E0E09321150E94AC
:10E2B4005B721E2FA12F0E946374103011F00C9416
:10E2C40066710E946B7301C020E00E949773E0E0C6
:10E2D400E09321150E942FAA08950E9491740E2F95
:10E2E400003011F40C9479710E942FAA08950E94B1
:10E2F4004EAB08950A930A2F000F000F000F087108
:10E3040000937715E0917615E260E0937615099114
:10E3140008950A930A2F0295007F000F0076009358
:10E324007715E0917615E460E093761509910895E8
:10E334000E94D8B89D014D8140937F15E0912E1520
:10E34400F0912F15E0937B15F0937C15E091301537
:10E35400F0913115E0937D15F0937E15E42FF0E0F4
:10E36400FA93EA93A0E4B0E00E9459221E2F00E041
:10E37400011710F00C94C871A0E8B5E1E02F0E94D9
:10E38400CCA8D9010E9401B30F5FF2CF0E94DFB87D
:10E39400269608950A930A2F043610F00C94D67129
:10E3A400E1E0E093C01503C0E0E0E093C0150991FB
:10E3B40008950E94DAB80E948B138F01112312F082
:10E3C4000C94E7710E9408B308950635E0E01E0737
:10E3D40014F40C94F0710E9408B3089500240016FC
:10E3E400010614F00C943E7220E0243510F00C94D5
:10E3F4000372E22FF0E0E453FB4EA0E0A0832F5F12
:10E40400F4CFECECF4E1FA93EA93A4E5B0E00E94D3
:10E414008E1300932015E0912015A091C115EA17E1
:10E4240011F40C941C72ACE10E94F60EE0912015DC
:10E43400E093C115A0912015AA3010F40C94297210
:10E44400A091CC14AF3311F00C94297201C003C015
:10E454000E940FB30895A0912015A63410F40C94D3
:10E464003A72A091CC14AD3311F00C943A7201C0FD
:10E4740003C00E940FB30895ACE10E940D0F8F01F9
:10E484000530E0E01E0714F40C944F72A091C115FE
:10E49400A13010F40C944F7201C008C00E94011303
:10E4A400E0E0E093C1150E9434AA08950E944EABA7
:10E4B400089522970E94D7A8E0E0E0932615E0E0B3
:10E4C400F0E0E0932715F0932815E0932915F093D5
:10E4D4002A15E0932B15F0932C15EFEFE0932D15EF
:10E4E400E0E0F0E0E0932E15F0932F15E093301563
:10E4F400F0933115EFEF0E9416B3E0E0E093351589
:10E5040040E050E04034E0E05E0710F00C94937279
:10E51400E6E3F5E1E40FF51FA0E0A0834F5F5F4F52
:10E52400F1CFA091CC14AD3311F40C949E72AF339F
:10E5340011F40C949E7201C005C0E1E00E94DEB8A3
:10E5440028960895A091CC14AD3311F00C94B172B7
:10E55400A0912015A63410F00C94B1720EC0A091B5
:10E56400CC14AF3311F00C94BE72A0912015AA30D4
:10E5740010F00C94BE7201C005C0E2E00E94DEB847
:10E5840028960895E0E0EF83A091CC14AD3311F008
:10E594000C94CF72E0E4EF8308C0A091CC14AF33A5
:10E5A40011F00C94D772E4E0EF83EF81EA5FEE831D
:10E5B400E150F0E0E453FB4EE081EA93EF81E25056
:10E5C400F0E0E453FB4EA0810E94BB209F01EE814A
:10E5D400E250EE8340E050E0EE810E9432AC10F055
:10E5E4000C94FF72ACECB4E1A40FB51FEC91F0E015
:10E5F4000E0F1F1F4F5F5F4FEFCF2017310711F42E
:10E604000C940B7340E050E0E4E00E94DEB82896DE
:10E614000895A091CC14AD3311F00C941473E2E07E
:10E62400E0932615A091CC14AF3311F40C941D7310
:10E63400E1E0E0932615E1E0F0E0E0932715F093A4
:10E644002815A9E2B5E1E091CD14F0E0ED93FC9337
:10E65400ABE2B5E1E091CF14F0E0ED93FC93E0E0A0
:10E66400E0932D15AEE2B5E1E091CE14F0E0ED9328
:10E67400FC93E0912B15F0912C15E0933015F09359
:10E684003115E0E00E9416B3EF81E0933515A091B7
:10E694003515A13410F40C945273E0E4E09335156D
:10E6A40040E050E0E09135150E9432AC10F00C943B
:10E6B4006873E6E3F5E1E40FF51FDF01FA01E053C7
:10E6C400FB4EE081EC934F5F5F4FECCF0E9411ACA7
:10E6D40008950A9300E0E0912915F0912A15FA9320
:10E6E400EA93E0912B15F0912C15FA93EA93E091BB
:10E6F4003515EA93A6E3B5E10E9413650E2FA02F0A
:10E704000E947C7100E0E0912E15F0912F15FA9390
:10E71400EA93A0913015B09131150E94F4610E2F47
:10E72400A02F0E948B7109910895EF9765970E941D
:10E73400D8B8E0917615E03011F00C94A773E0E0BE
:10E744000E94DFB8EF966A960895E0E0EF83E887C9
:10E75400AF81B885A035E0E0BE0710F00C94B97322
:10E764000E941FB3E0E0EC930E9423B3F1CFE09149
:10E77400C015E03011F00C94C373EFE5E98708E0AD
:10E7840003C0EDE5E98700E4A0917F150A1710F0B6
:10E794000C94CE7300937F15E0917715EA87E0E03F
:10E7A400EF83E887E0917F150E94A7B010F00C94E6
:10E7B400ED73EF81F8853296ED83FE830E9429B3D1
:10E7C4000F01E0E8F5E10E9460A6EC91D001EC9322
:10E7D4000E9423B3E7CFED81FE813196ED83FE8362
:10E7E400EF83F887E02FEE5F0E94A7B010F00C943F
:10E7F40002740E941FB3E0E0EC930E9423B3F2CFB3
:10E80400E02FF0E032961E2F2F2F30E040E0E0E0C2
:10E81400EF83E887AF81B885A117B20710F00C9495
:10E824001C740E941FB3EC91F0E03E0F4F1F0E9436
:10E8340023B3F0CFE12FF22F0E9429B33083342F7A
:10E844004427E12FF22F31960E9429B330831E5FB3
:10E854002F4FA985AD3511F00C943674AA85A032DA
:10E8640011F00C94367401C004C0E1E0F0E0EF83D1
:10E87400F887E4E4F0E0E117F20711F40C944A7429
:10E88400ECE0F0E0E117F20711F40C944A7407C0CD
:10E894000E94F7ADA12FB22F0E94DB1303C0E0E06A
:10E8A400EF83E8870E9453ABE0E0E0937615EF81B5
:10E8B400F885EF83F887E1E00E94DFB8EF966A9667
:10E8C40008951A930A931A2F10937715E3E6E093A9
:10E8D4007815E0937915E0E0E0937F1500E00034CB
:10E8E40010F00C947D74A0E8B5E1EE27A00FBE1FD4
:10E8F400EC930F5FF4CFE0917715E03011F00C94B6
:10E904008974E0917615E160E093761505C0E09195
:10E914007615E161E0937615099119910895A09116
:10E924002015AE3010F40C94F974A091CC14A230DC
:10E9340011F00C94EC74A091CD14A13511F00C9449
:10E94400EC74A091CE14A33411F00C94EC74A09147
:10E95400CF14A23211F00C94EC74A091D014A5350C
:10E9640011F00C94EC74A091D114AB3511F00C940B
:10E97400EC74A091D214AD3211F00C94EC74A0910B
:10E98400D314A43311F00C94EC74A091D414A234D5
:10E9940011F00C94EC74A091D514AD3411F00C94D6
:10E9A400EC74A091D614A83511F00C94EC74A091D9
:10E9B400D714A23D11F00C94EC74A091D814A33D8B
:10E9C40011F00C94EC74A091D914A33011F00C94B0
:10E9D400EC7401C00CC0AEEAB6E080E090E00E94A6
:10E9E40060950E9494AA0E94200DE1E00895E0E061
:10E9F40008950E94D7B80DE110E040EA52E120E00A
:10EA040030E0DA01E0E0EC934F5F5F4FF9013196BB
:10EA14009F01E017F10710F00C941175F2CF0E94DA
:10EA2400DEB826960895E0E0E093C215E093C3159E
:10EA34000E949990E3E6E093C4150895E091C3150C
:10EA44000895E2E0E093C315E0E008950E942EB338
:10EA5400A0E00E94D427A0E00E940528A0E00E9424
:10EA6400EF270E945F860895AA9325970E94D7B83E
:10EA7400EB85E03011F40C9442750E9432B3089592
:10EA8400E091C215E03011F00C944B750E9437B33D
:10EA940015C0E13011F00C9452750E943DB30EC0C4
:10EAA400E23011F00C94577509C0E33011F00C9466
:10EAB4005C7504C0E43011F00C946075A091C2152B
:10EAC400AF5FA093C215A53010F40C946C75E0E010
:10EAD400E093C2150E94AF88E03011F40C94AF7536
:10EAE400A5ECB5E10E948C885E2FE091C315E0305F
:10EAF40011F40C948675513010F40C9486755A30C8
:10EB040010F00C94867501C015C0E0E0E093C315C5
:10EB1400A0E00E946A600E94CEB10E9499900E9477
:10EB24002EB3A6ECB6E080E090E00E9460950E94CF
:10EB3400CE8813C0533011F00C94A675E1E0E09335
:10EB4400C3150E94CE8809C0543011F00C94AF75DF
:10EB5400E2E0E093C3150E94CE88A091C315A130D2
:10EB640011F00C94BD750E9499900E94187CE0E00D
:10EB7400E093C315BAC0A091C315A23011F00C9450
:10EB8400EB750E949990A5EDB6E080E090E00E94BC
:10EB94006095A2EFB6E080E090E00E946095A9E164
:10EBA400B7E080E090E00E946095AEE00E943C0FE8
:10EBB400E091C315EF5FE093C3150E9442380E94B1
:10EBC400253EA1E00E946C3E0E9485600E94C8B16F
:10EBD4008CC0A091C315A33011F00C946176AEE003
:10EBE4000E94580F9F012531E0E03E0710F40C9479
:10EBF4000076E091C315EF5FE093C3150E94693E70
:10EC04004E2F483011F00C9409760E94903EE0910A
:10EC1400C415E41711F40C9431764093C4150E9482
:10EC24009990483011F00C941D76AEE2B7E080E084
:10EC340090E00E946095493011F00C942776A0E48E
:10EC4400B7E080E090E00E9460954A3011F00C94A7
:10EC54003176A9E4B7E080E090E00E946095FE017F
:10EC64003A96FA93EA93FE013B960E949FA8FE010E
:10EC74003D96FA93EA93DE011E960E94643F4E2F5E
:10EC8400403011F00C9460760E811127AFEFA09FF5
:10EC9400F001A19FF00D8F01EF81F0E00E0F1F1F17
:10ECA400EFE5F7E060E070E00E946ABAD8010E94E4
:10ECB400AAAC0E943495AEE00E943C0F16C0A0910D
:10ECC400C315A43011F00C947776A0E00E946A601A
:10ECD4000E94CEB10E942EB3AAE6B7E080E090E095
:10ECE4000E946095E0E0E093C3150E9432B308955A
:10ECF400E6970E94D8B800E00E9443B30E9434957E
:10ED04000E9443B3A8E7B7E080E090E00E946095DA
:10ED1400A091A112A13011F00C949776A1E9B7E06B
:10ED240080E090E00E94609506C0A8E9B7E080E02A
:10ED340090E00E9460951091A512113011F00C948E
:10ED4400AA76A8EAB7E080E090E00E94609506C049
:10ED5400E4EBF7E060E070E00E9447B30E94AE7914
:10ED64001E2F113010F40C94BF7601E0E4ECF7E0B0
:10ED740060E070E00E9447B306C0AFECB7E080E00B
:10ED840090E00E9460950E94E2791E2F103011F4E9
:10ED94000C94D47601E0E6EDF7E060E070E00E94C8
:10EDA40047B306C0A1EEB7E080E090E00E94609512
:10EDB4000E944B612E2F203011F40C94E776A8EEBC
:10EDC400B7E080E090E00E9460950E9461613E2F70
:10EDD400303011F40C94F476ABEFB7E080E090E0BF
:10EDE4000E9460950E9477614E2F403011F40C947C
:10EDF4000177AEE0B8E080E090E00E9460952030BA
:10EE040011F00C940E77303011F00C940E774030E2
:10EE140011F00C940E7701C006C0A3E2B8E080E0C4
:10EE240090E00E9460950E9433520E9436B00E9486
:10EE3400477A1E2F103011F40C94287701E0ECE28D
:10EE4400F8E060E070E00E9447B306C0AFE3B8E0CA
:10EE540080E090E00E9460950E9443520E9436B088
:10EE64000E94167A1E2F103011F40C94417701E0A1
:10EE7400EEE4F8E060E070E00E9447B306C0ADE560
:10EE8400B8E080E090E00E9460950E9445791E2FD2
:10EE9400103011F40C94567701E0E8E6F8E060E0F5
:10EEA40070E00E9447B306C0A5E7B8E080E090E0B8
:10EEB4000E9460950E946E791E2F103011F40C94FC
:10EEC4006B7701E0EEE7F8E060E070E00E9447B3A2
:10EED40006C0ABE8B8E080E090E00E9460950E9434
:10EEE400F9781E2F103011F40C94807701E0E4E9D6
:10EEF400F8E060E070E00E9447B306C0A7EAB8E01B
:10EF040080E090E00E9460950E9463541E2F1230AE
:10EF140010F40C94B07701E0E6EBF8E060E070E008
:10EF24000E9447B311FF02C00E944BB315FF02C0F9
:10EF34000E9451B317FD03C016FD01C003C00E9417
:10EF440057B30BC012FD03C014FD01C002C00E94E0
:10EF54005DB313FF02C00E9463B306C00E9469B38D
:10EF640010FF02C00E946FB30E9407611E2F103071
:10EF740011F00C94C877E8ECE093B01201E0A4E23D
:10EF8400B9E080E090E00E94609509C0E1E0E09380
:10EF9400B012A1E3B9E080E090E00E9460950E9485
:10EFA40029611E2F103011F40C94E277E8ECE09301
:10EFB400B112AEE3B9E080E090E00E94609509C030
:10EFC400E1E0E093B112AAE4B9E080E090E00E94AD
:10EFD40060950E9442380E945C3E1E2F113010F44E
:10EFE4000C94FF77E8ECE093AA1201E0A6E5B9E0FF
:10EFF40080E090E00E94609509C0E1E0E093AA12ED
:10F00400A0E6B9E080E090E00E946095E1E0E09342
:10F01400B912E0E0E093AD120E945986ADE10E947E
:10F02400F60EADE10E940D0FED83FE831091AD123B
:10F034000E946986AD81BE81A039E1E0BE0710F06F
:10F044000C942978103011F00C94297801C001C077
:10F05400E8CF0E949990113011F00C943878A7E60B
:10F06400B9E080E090E00E94609507C001E0E4E729
:10F07400F9E060E070E00E9447B3A5E8B9E080E001
:10F0840090E00E946095A0E00E94C27F1E2F0E9423
:10F09400D07BA091AA12A83C10F40C945578E8EC0B
:10F0A400E093AB1239C0E0E0E093AB120E94253E3E
:10F0B400A1E00E946C3E0E94903EADE10E94F60EDB
:10F0C400ADE10E940D0FED83FE831091AB120E94FF
:10F0D40001370E94F03BAD81BE81A83EE3E0BE074C
:10F0E40010F00C947A78103011F00C947A7801C0F6
:10F0F40001C0E6CF113011F00C948778A1EAB9E091
:10F1040080E090E00E94609507C001E0E1EBF9E047
:10F1140060E070E00E9447B3003011F40C949C78D6
:10F12400A1ECB9E080E090E00E946095A1E00E942B
:10F13400DB2509C0A0EDB9E080E090E00E94609575
:10F14400A1E00E94D125E1E0E093BB120E94349536
:10F154000E94F7AD0E9452B1E8ABEAEDF9E060E03D
:10F1640070E00E9475B30E940B1CE0EFF9E060E0D0
:10F1740070E00E9475B30E94BE950E94F7AD0E9494
:10F1840052B1E8ABECEFF9E060E070E00E9475B3D7
:10F194000E940B1CE9E0FAE060E070E00E9475B3A5
:10F1A4000E94BE950E94F7AD0E9452B1E8ABE5E122
:10F1B400FAE060E070E00E9475B30E940B1CE2E28A
:10F1C400FAE060E070E00E9475B30E947AB3E1E077
:10F1D400E093AE12E0E0E093B4120E949990A7E0AD
:10F1E4000E943C0FE02F0E94DFB8EB9608951A931B
:10F1F4000A9300E0E0E0E093AC120E9490B11E2F6D
:10F20400113010F40C9436790E946728E03011F420
:10F214000C940D7901E0A1E00E942D280E943CAFDE
:10F224000E946728E03011F00C94197902E0A0E004
:10F234000E942D280E947EB3A1E00E9443280E94D0
:10F244003CAF0E946728E03011F00C942A7903E067
:10F25400A0E00E9443280E947EB30E946728E03009
:10F2640011F40C94367904E0013010F40C943E79D6
:10F27400E8ECE093AC1203C0E1E0E093AC12E02FC1
:10F284000991199108950A93EFEFFFE0FA93EA9335
:10F29400A9E70E9482B3093711F40C945779E8EC7A
:10F2A400E093A212E1E009910895EFEFFFE0FA93F1
:10F2B400EA93A6E80E9482B3063811F40C946879A4
:10F2C400E8ECE093A212E1E009910895E1E0E09313
:10F2D400A212E0E0099108950A93A0E00E94F725A4
:10F2E4000E9464A9EEEFFFEF0E9427B1A2E10E9401
:10F2F40060810E2F0E9498AA0E948AB3023111F4F1
:10F304000C948A79E8ECE093A312E1E00991089562
:10F31400EEEFFFEF0E9427B1A7E30E9460810E2F5A
:10F324000E9498AA0E948AB3073311F40C94A0791E
:10F33400E8ECE093A312E1E009910895E1E0E093A1
:10F34400A312E0E0099108950E948AAF0895AEE106
:10F35400B0E00E947E0E089562970A93DE01119632
:10F364000E94074D0E2F023010F40C94C7790E94AE
:10F37400C1A90E94ECA9AFE10E94E74E0E94C1A975
:10F38400DE0111960E94074D0E2F003011F00C94EF
:10F39400CF79E1E0E093A4120FC0013011F00C9496
:10F3A400D779E8ECE093A41207C0023011F00C9472
:10F3B400DE79E9ECE093A412E02F088163960895C6
:10F3C400A8970A93FE017796FA93EA93DE011396BF
:10F3D4000E94B44F0E2F003011F40C94F27904C043
:10F3E400E02F0881A99608950881A99608950E949E
:10F3F400D9B820E0A1E00E94E5250E94A9790E94E5
:10F4040037B33E2F313010F40C94097A21E00E9476
:10F414003DB33E2F313010F40C94117A21E0E22FE9
:10F424000E94E0B8249608950E9495B30832E3E25E
:10F434001E0710F40C94257A0939EAE31E0710F02C
:10F444000C94257A05C021E0E8ECE093B21218C0D0
:10F454000033EAE21E0710F00C94357AE9ECE093ED
:10F46400B21222E00DC0003CEBE21E0710F00C9437
:10F474003F7AE4E6E093B21203C0E1E0E093B21213
:10F48400E22F0E94E1B8259608950E9495B30832B0
:10F49400E0E01E0710F40C94567A0530E1E01E07F4
:10F4A40010F00C94567A05C021E0E8ECE093B31216
:10F4B40015C00135E0E01E0710F40C94687A0C3D89
:10F4C400E0E01E0710F00C94687A05C022E0E9EC35
:10F4D400E093B31203C0E1E0E093B312E22F0E9481
:10F4E400E1B8259608951A930A9300E00E947027C4
:10F4F400E03011F40C94837AA0E00E9464270E9407
:10F50400A979A1E00E9464270E94A6790E94762727
:10F51400E03011F00C948F7A01E0013010F40C9477
:10F52400977AE02F0991199108950E94882CE03070
:10F5340011F40C94A27AA0E00E94722C0E94A97982
:10F54400A0E00E94722C0E94A679A1E00E94722C75
:10F554000E94A6790E94132DE03011F00C94B37A26
:10F5640002E0013010F40C94BB7AE02F0991199158
:10F574000895A0E00E949DB311F40C94C27A03E0B4
:10F58400A1E00E949DB311F00C94C97A03E0A0E0BD
:10F594000E94AAB311F40C94D07A03E0A1E00E9473
:10F5A400AAB311F40C94D77A03E0013010F40C944C
:10F5B400DF7AE02F099119910895A0E00E94B7B372
:10F5C40011F00C94E67A04E0A1E00E94722CA1E010
:10F5D4000E94EF270E94A679A1E00E94B7B311F41C
:10F5E4000C94F57A04E0013010F40C94FD7AE02FC9
:10F5F4000991199108950E94E027E03011F40C94C8
:10F60400087BA0E00E94D4270E94A979A0E00E9470
:10F61400BFB311F40C940F7B05E0A1E00E94BFB3CB
:10F6240011F00C94167B05E0013010F40C941E7B51
:10F63400E02F0991199108950E941128E03011F4E6
:10F644000C94297BA0E00E9405280E94A979A0E0DF
:10F654000E94C7B311F40C94307B06E0A1E00E9431
:10F66400722CA1E00E94C7B311F00C943A7B06E01F
:10F67400013010F40C94427BE02F09911991089504
:10F684000E94FE2AE03011F40C944D7BA0E00E940D
:10F69400E82A0E94A979A0E00E94E82A0E94A6799B
:10F6A400013010F40C945A7BE02F099119910895BC
:10F6B4000E94E52CE03011F40C94657BA0E00E94DC
:10F6C400D92C0E94A979A0E00E94D92C0E94A67985
:10F6D400A1E00E94D92C0E94A6790E94F52CE0306A
:10F6E40011F00C94767B09E0013010F40C947E7BCD
:10F6F400E02F0991199108950E94A82CE03011F48B
:10F704000C94897BA0E00E94922C0E94A979A0E02D
:10F714000E94922C0E94A679A1E00E94922C0E9441
:10F72400A6790E940A2DE03011F00C949A7B0AE02D
:10F73400013010F40C94A27BE02F099119910895E3
:10F74400A1E00E94B22C0E94A6790E94C82CE0304D
:10F7540011F00C94AE7B0BE0013010F40C94B67BEA
:10F76400E02F099119910895A0E00E94D0B311F4FB
:10F774000C94BD7B0CE0A1E00E94D0B311F00C947A
:10F78400C47B0CE0013010F40C94CC7BE02F099185
:10F7940019910895E02F099119910895A091A71244
:10F7A400A13011F00C94EF7BAEE2BAE080E090E07F
:10F7B4000E946095A091A912A13011F00C94E87BED
:10F7C400A7E3BAE080E090E00E946095E2E4FAE00A
:10F7D40060E070E00E94D9B328C0AAE4BAE080E0F7
:10F7E40090E00E946095E091A712E83C11F00C941F
:10F7F400027CA1EEB8E080E090E00E94609515C024
:10F80400E93C11F00C940D7CA7E5BAE080E090E0AF
:10F814000E9460950AC0E43611F00C94177CA2E6AD
:10F82400BAE080E090E00E94609508950A93A0E712
:10F83400BAE080E090E00E9460950E9463540E2F2D
:10F84400023010F40C944B7CE6EBF8E060E070E0DE
:10F854000E946ABAA02F0E942EB101FF02C00E942A
:10F864004BB305FF02C00E9451B307FD03C006FD60
:10F8740001C003C00E9457B30BC002FD03C004FDC6
:10F8840001C002C00E945DB303FF02C00E9463B3C3
:10F894000CC00E9469B300FF02C00E946FB30E94B3
:10F8A400F24A0E9494AA0E94A154099108951A93BD
:10F8B4000A93A1E00E9445B010F40C94687CA0E087
:10F8C4000E94D125A1E00E94F60E09C00B35E0E0AC
:10F8D4001E0710F40C94717CA1E00E94D1250991BB
:10F8E40019910895E0918414E03011F00C94827C15
:10F8F4000E94DEB30E94FCAD0E94F1130E949D148D
:10F904000895E0918414E03011F00C949A7C0E94E4
:10F914009B7C0E94747CA1E00E94D92C0E9464A963
:10F92400E0E0E093CD15E093CE15EFEFE093CF1533
:10F93400089508950E94ECAF11F40C94A47C0E94E5
:10F94400F1AF0895E0918414E03011F40C94AD7C8F
:10F954000E94F1AF0895E091CD15A091CF15EA175B
:10F9640011F40C94BA7CE093CF15E1E0E093CE154A
:10F97400E091CD15E03011F00C94D87CE091CE15D7
:10F98400E03011F40C94CB7C0E94E4B340E00E947C
:10F99400747C0E94EAB310F00C94D57C403011F0D2
:10F9A4000C94D57C02C00E94F2B387C0A091CD15FF
:10F9B400A13011F00C94FF7CE091CE15E03011F4ED
:10F9C4000C94EB7C0E94E4B30E94FD7D40E00E9415
:10F9D400DEB30E94B67D8F01D8010E94307E4E2F87
:10F9E4000E94EAB310F00C94FC7C403011F00C94AB
:10F9F400FC7C02C00E94F2B360C0A091CD15A2307D
:10FA040011F00C94237DE091CE15E03011F40C94A8
:10FA14000F7D0E94E4B30E940E7E0E94B67D8F018A
:10FA2400D8010E94727E4E2F0E94EAB310F00C940B
:10FA3400207D403011F00C94207D02C00E94F2B36E
:10FA44003CC0A091CD15A33011F00C943F7DE09102
:10FA5400CE15E03011F40C94327D0E94E4B340E002
:10FA64000E94FBB310F00C943C7D403011F00C94D8
:10FA74003C7D02C00E94F2B320C0A091CD15A430F9
:10FA840011F00C945F7DE091CE15E03011F40C94EC
:10FA94004E7D0E94E4B340E00E94FBB310F00C944E
:10FAA400587D403011F00C94587D06C0E0E0E0939E
:10FAB400CD15E1E0E093CE1500C00E94F1AF0895AA
:10FAC400A0970E94D8B800E010E020E0E0918414F0
:10FAD400E03011F40C94747DE0E0F0E00E94DFB8B3
:10FAE400A59608950E94C1A90E947215E03011F4F0
:10FAF4000C94A27D0E941E151E2F2F2FA12FB22F12
:10FB04000E9403B411F40C948A7DE12FF22F02C0F9
:10FB1400E0E2F0E03E2F4F2F00240116020614F01D
:10FB24000C94A07D0E9466ABA32FB42F0E944315B2
:10FB34000E9466ABA32FB42F0E94FD830E949D14E4
:10FB44000F5F043610F00C94AE7D002401160206FB
:10FB540011F00C94AE7D01C001C0C4CFE12FF22F8F
:10FB64000E94DFB8A5960895EF9721970E94D9B80F
:10FB740000E010E0E0918414E03011F40C94C97DAD
:10FB8400E0E0F0E00E94E0B8EF96259608950E9428
:10FB94007215E03011F40C94F77D0E941E158F014C
:10FBA400D801E0E4F0E00E9485B9F0E0E03011F41F
:10FBB4000C94DE7DF80102C0E0E4F0E09F01002433
:10FBC4000016010614F00C94F57DFE013496FA93A8
:10FBD400EA93D9010E944315FE013496FA93EA93FD
:10FBE400D9010E94FD830E949D14F8010E94E0B88F
:10FBF400EF9625960895E0918414E03011F00C946A
:10FC04000D7E0E94DEB30E949D14A4E8BAE080E059
:10FC140090E00E940AB40895E0918414E03011F059
:10FC24000C941E7E0E94DEB30E949D14ABE8BAE0E1
:10FC340080E090E00E940AB40895E0918414E030DA
:10FC440011F00C942F7E0E94DEB30E949D14A4E94F
:10FC5400BAE080E090E00E940AB4089526970E94DA
:10FC6400BAA40E940FB411F40C943B7E0E9414B405
:10FC740008951B30E0E02E0710F40C946F7EEEE93B
:10FC8400FAE060E070E00E946ABA2A931A930E9434
:10FC940019B411F40C946F7E0E94CDB0A3E00E94BD
:10FCA4007385AD81AC3211F00C94667EEB81E05328
:10FCB400AAE0EA9FF001AC81AE0FE0E30E9477BABC
:10FCC400EA1BE093A81204C0EB81E053E093A8126E
:10FCD400E1E00E94E1B8299608950E9414B40895C1
:10FCE40026970E94BAA40E940FB411F40C947D7E4E
:10FCF4000E9414B408951B30E0E02E0710F40C9415
:10FD0400B87EE5EAFAE060E070E00E946ABA2A93FD
:10FD14001A93A0E00E9443840E2F003011F40C9437
:10FD2400B87E0E94CDB0A3E00E947385AB81A0335E
:10FD340011F00C94AD7EAC81AC3211F00C94AD7E1C
:10FD4400AD81A13311F40C94AC7EA53311F40C9461
:10FD5400AC7E01C001C007C0E1E0E093A9120E949B
:10FD6400E1B829960895E4E6E093A9120E9414B438
:10FD74000895AA93A2970E94D7B838A5E091841455
:10FD8400E03011F40C94CB7EE0E00E94DEB8A9963A
:10FD940008950E94DEB3313011F00C94D67E0E9497
:10FDA400FCAD0E94F1133DC0323011F00C94E27EA0
:10FDB400E2E0EA93EA930E94BBA90E94F11331C0E6
:10FDC400333011F00C94EF7EE2E0EA93E3E0EA933F
:10FDD4000E94DFAB0E94F11324C0343011F00C9464
:10FDE400FA7E0E94B6A90E94BBA90E94F11319C011
:10FDF400353011F00C94077FE2E0EA93E1E0EA93F6
:10FE04000E94BBA90E94F1130CC0363011F00C946F
:10FE1400137FE2E0EA93E4E0EA930E94BBA90E9424
:10FE2400F1130E949D140E947EB300E00E947EB3F1
:10FE3400FE0138960E9440AF0E94CAAE0E949D14F3
:10FE4400ADEABAE080E090E00E940AB410E0A8E0D5
:10FE5400B0E00E947E0E0E947215E03011F40C9402
:10FE6400697F0E941E15AF01DA010E9403B411F4E8
:10FE74000C943E7FFA0102C0E0E2F0E0EE83FF83DF
:10FE840000240416050614F00C94677F0E9440B108
:10FE9400A885B9850E9443150E9440B1A885B985FB
:10FEA4000E94FD830E941FB4EA85FB85FA93EA93BE
:10FEB400A0E00E9443842E2F203011F40C94677F1D
:10FEC400E32F0E94DEB8A99608950E949D141F5F37
:10FED400143610F00C94737F203011F00C94737F5F
:10FEE40001C001C0B4CF0F5F063010F00C947F7FC7
:10FEF400203011F00C947F7F01C001C097CFE0E067
:10FF04000E94DEB8A99608951A930A930E940FB42A
:10FF140011F40C94917FE0E009911991089511E096
:10FF2400A12F0E94BB7E0E2F1F5F163010F00C9481
:10FF3400A07F003011F00C94A07F01C001C0F0CF6D
:10FF4400E02F0991199108950A93E0918414E03007
:10FF540011F40C94C07F0E94DEB30E949D1401E052
:10FF6400A3EBBAE080E090E00E940AB40E947EB362
:10FF74000F5F033010F00C94C07FF2CF0991089505
:10FF8400A0970E94D7B85A2F20E0E0918414E03063
:10FF940011F40C94D27FE0E00E94DEB8A696089596
:10FFA4000E94837C0E94DEB3A8EEB3E00E947E0E22
:10FFB4000E94867F2E2F0E9464A9203011F00C9499
:10FFC400E77FE8EC0E9426B40895E1E0E093A712ED
:10FFD4000E94A67F00E00E94747C0E947EB30E946F
:10FFE400DFAE0E942DB40E949D14A1ECBAE080E023
:0CFFF40090E00E940AB40E9430B40E9409
:020000021000EC
:040000002DB40E9479
:100004009D14A6ECBAE080E090E00E940AB40E943D
:1000140030B40E942DB40E949D14A0EDBAE080E09B
:1000240090E00E940AB40E9435B43B30E0E04E07F1
:1000340010F40C942A80E4EDFAE060E070E00E9491
:100044003AB411F00C942A80E9EC0E9426B4089585
:100054000E94DFAE0E942DB40E949D14ADEDBAE063
:1000640080E090E00E940AB40E9435B43530E0E0AC
:100074004E0710F40C944D800E941FB44A933A9397
:10008400A0E00E9443841E2F103011F00C944D8088
:10009400E4E6E093A7120E94DFAE0E942DB400E0D4
:1000A400503011F40C94578003E6ACE2B1E00E94A6
:1000B4007E0E0E94FD7D0E9435B4A32FB42F0E94B2
:1000C400307E0F5F043110F00C947680A091A8125A
:1000D400AC3010F40C947580A091A812A03210F0EA
:1000E4000C94758001C001C001C0DFCF0E94DFAE57
:1000F4000E942DB40E940E7E0E9435B4A32FB42F0B
:100104000E94727E0E94DFAE0E942DB40E941F7E68
:100114000E9435B43B30E0E04E0710F40C949B8011
:10012400EAE8FAE060E070E00E943AB411F00C945E
:100134009B80E0E00E94DEB8A696089522970E9474
:10014400D8B81A2F2F81388549854A933A93E1E02C
:10015400EA932A931A93DE011A960E94A0AF10F430
:100164000C94B980E0E00E94DFB82A9608950D81CE
:10017400E02F0E94DFB82A96089528970E94D8B8E5
:100184001A2F2D853E854F854A933A93E4E0EA93EE
:100194002A931A93DE011E960E94A0AF10F40C94C9
:1001A400D7800E9417A960960895EC85FF276627DB
:1001B40077270E9444B4EB850E944DB4EA850E94DF
:1001C4004DB4E9850E9426A50E9455B40E9433A52A
:1001D4000E94DFB860960895BA93AA93EF97279781
:1001E4000E94D7B8FE01E05BFF4F5081FE01EE5A3A
:1001F400FF4F11912081FE01E25BFF4F0190F081DE
:10020400E02DE887F987E0E0EE83EF832A931A93E1
:10021400E0E4EA930E94DBA9EA935A93DE011F9675
:100224000E94A0AF10F40C941D81E1E00E94DEB89E
:10023400EF9665960895A885B985A134E0E0BE07D8
:1002440010F40C94398130E040E03034E0E04E07A3
:1002540010F00C9432810E945BB43F5F4F4FF5CF96
:10026400E885F985E054F040E887F98711C030E06B
:1002740040E0E885F9853E174F0710F00C9447815C
:100284000E945BB43F5F4F4FF4CFE0E0E887E9871B
:10029400EE81FF81E05CFF4FEE83FF83105C2F4F04
:1002A400A885B9850E94B0BA10F00C945A81AECFDB
:1002B400E0E00E94DEB8EF966596089522970E94CA
:1002C400D7B81A2F288539854A855B85A5E0B0E023
:1002D4000E945C0E1E835A934A93E1E0EA933A9398
:1002E4002A93DE011B960E94F6100E2F013010F4A3
:1002F4000C948181E1E00E94DEB82C9608950E945E
:1003040032B308950E946FBA28970E94D8B83989E9
:100314004A891B892C89ED85FE856F8578890E9421
:100324001CA5ED81E9870E9470B4EA870E9470B42D
:10033400EB870E9470B4EC872A931A93E4E0EA9363
:100344004A933A93DE011E960E94F6100E2F013056
:1003540010F40C94B281E1E00E94DFB86596089530
:10036400E0E00E94DFB8659608950E94D7B89D0129
:100374004E815F81042F013410F40C94C28100E497
:10038400E885F985FA93EA930A935A93E1E0EA93AC
:10039400D9010E94F6101E2F0E9498AA103011F461
:1003A4000C94D7810E94B2A60895E02F0E94DEB873
:1003B4002A960895BA93AA93EF972F970E94D7B8D5
:1003C400FE01E65AFF4F01911081FE01E65AFF4FEC
:1003D4000190F081E02D662777270E9498A70E945C
:1003E40079B4662777270E9400AF0E94F3B80E9471
:1003F400ECAE0E9479B40E9480B440E050E00E94C8
:1004040086B4A034E0E0BE0710F00C94628220E0D1
:1004140030E00E948DB42E173F0710F00C94178221
:100424000E9494B42F5F3F4FF4CFFE01EE5AFF4F6A
:10043400E081E770EF87E03011F40C942582AF85FA
:10044400E8E0EA1B01C0E0E0EE8720E030E0EE8562
:10045400D901F0E0AE17BF0710F00C943C820E9463
:100464008DB4E20FF31FDE0150960E9449AF2F5F57
:100474003F4FEDCFEE850E9486B4F0E0EA0FFB1FFC
:100484000E9480B41A930A930E94DBA90E94A5B427
:100494000E94A5B40E94ABB4AF85A13010F40C94B3
:1004A40058820E94E8A4EF966D9608950E948DB438
:1004B400E40FF51F9F010E94DEB8EF966D96089534
:1004C40020E030E02034E0E03E0710F00C946F822E
:1004D4000E9494B42F5F3F4FF5CF1A930A93E0E440
:1004E4000E94A5B40E94A5B40E94ABB4AF85A1300C
:1004F40010F40C9482820E94E8A4EF966D960895FD
:100504000E948DB4E054F0400E9480B40E948DB4E7
:10051400309711F00C949482FA010E94DEB8EF96A1
:100524006D960895005C1F4FEE81FF816885798583
:10053400E05CFF4F6F4F7F4F0E9498A7405C5F4F76
:100544000E946FA80E9400AF0E94BFBA10F00C94E2
:10055400AC8255CF0E94E8A4EF966D9608950A9355
:100564000A2FE4E1E09FF00109910895BA93AA9358
:10057400AC978CE2002470E0E8EEFAE060E00E94C0
:10058400E5B80E94D8B809A91AA9ED81FE81E0173F
:10059400F10710F40C94D382E0E00E94DFB8E396F4
:1005A400089541E0E42FF0E0DE0115960E94B6AC18
:1005B4002D913C910217130710F00C94E782E42F5D
:1005C400E1500E94DFB8E39608954F5F453110F083
:1005D4000C94ED82E7CFE4E10E94DFB8E39608953E
:1005E400BA93AA93EF9721978CE2002470E0E4E198
:1005F400FBE060E00E94E5B80E94D7B8FE01EA5B28
:10060400FF4F01911081EEA5FFA50E94B3B40E1710
:100614001F0710F40C941583E0E9F1E00E94DEB8A2
:10062400EF96299608954E815F814017510710F483
:100634000C9421830E94E8A4EF9629960895D8018A
:100644000E94B882EBAFF0E0DE0116960E94B6ACD1
:100654004D915C91EBADEF5FF0E0DE0116960E94E8
:10066400CAAD0E94B3B4E41BF50BEEAFFFAFABAD64
:100674000E94B182DE01AE5BBF4FED93FC93EBAD04
:10068400EF5FEAAFAAAD0E94B182DE01A05CBF4F6A
:10069400ED93FC93DE01AE5BBF4F0D90BC91A02D9A
:1006A400EA1BFB0BECAFFDAFEEADFFAD309711F0E5
:1006B4000C946083E4E1F0E0EEAFFFAFECADFDAD90
:1006C4000E94B9B4DF01CB01EEADFFAD0E94B9B415
:1006D4000E94FCBBEEABFFAB68AF79AFF801E41B43
:1006E400F50B0E94B9B4EAABFBAB6CAB7DABEEA9E6
:1006F400FFA968AD79ADAAA9BBA98CA99DA90E943F
:10070400AEBBEAABFBAB6CAB7DAB0E94F1BA9F0115
:10071400FE01EE5BFF4F0190F081E02D2E0F3F1F95
:10072400F9010E94DEB8EF9629960895BA93AA9328
:1007340066970E94D7B8E0E0F0E46CE975E40E94A3
:10074400ECAE44EE5CE0E0E0F0E46CE17AE40E94BC
:1007540098A70E9400AFE0E0F0E060E874E40E9433
:10076400FCBB0E9498A70E9400AFE0E0F0E06AE7BB
:1007740074E40E94FCBB0E9498A7EC8DFD8D0E943E
:10078400B9B40E94BEB4EE81FF81688579850E9468
:10079400C3B4EE8BFF8B688F798FAE89BF89888D48
:1007A400998D0E946FA80E945DBBEE87FF87688BBE
:1007B400798BAE89BF89888D998D0E94FCBB0E947C
:1007C400BEB4FA010E94B9B40E94C3B40E94BEB47C
:1007D400EA89FB896C897D890E94F1BAEA8FFB8FD3
:1007E400AA8DBB8D0E94F2828F0130969F010E94D8
:1007F400DEB86E9608950E94D7B89D014E815F8140
:100804002A32E3E03E0710F40C940A842AE233E02F
:1008140000E010E00A32E3E01E0710F00C941984A3
:10082400A0EDB5E10E94CCA50F5F1F4FF3CF20933D
:10083400FA183093FB185A934A93E0EDF5E1FA93D2
:10084400EA93A091FA18B091FB180E94061B0E942B
:10085400CAB4E053FA4EA0E0A083E0E0E093FE18AF
:10086400E093FF18E093FC18E093FD18E09300195F
:10087400E0930119E0930219E09303190E9411AC6B
:100884000895AA932697D1500E94D7B8FE01E35F3A
:10089400FE4F0190F081E02DEA87FB87FE01E45FC3
:1008A400FE4F10810E94CFB410F00C945D84E0E000
:1008B4000E94D8B408950E94DDB40E94E4B40E945A
:1008C400EDB40E94F4B410F00C947C84FA01DE01BF
:1008D4001C96EA0FFB1FFF93EF93FA010E94E4B406
:1008E4000E9451A66BBFE691AF91BF91EC934F5F0D
:1008F4005F4FE7CF0E94F9B401E040E050E0FA0115
:100904000E9435A70E9405B511F40C948A8400E076
:100914004F5F5F4F0E94F4B410F00C949684013042
:1009240011F00C94968401C001C0E9CF0E9495A5F2
:10093400AE81BF812A173B0710F40C94A6840030C3
:1009440011F00C94A68401C001C0D6CF0E940FB54B
:1009540011F40C94B0840E9424B502C00E9431B5F5
:10096400003011F40C94BB84103011F40C94BB844B
:1009740001C005C00E943AB50E94D8B40895003061
:1009840011F40C94C984E1E00E94D8B40895E0E025
:100994000E94D8B408950E94D8B40895AA932697C3
:1009A400D1500E94D7B8FE01E25FFE4F0190F08162
:1009B400E02DEA87FB87FE01E35FFE4F10810E9472
:1009C400CFB410F00C94E9840E9444B508950E94B9
:1009D400DDB40E944AB50E94EDB40E94F4B410F054
:1009E4000C940885FA01DE011C96EA0FFB1FFF93A5
:1009F400EF93FA010E944AB50E9451A66BBFE6919B
:100A0400AF91BF91EC934F5F5F4FE7CF0E94F9B472
:100A140001E040E050E0FA010E9435A70E9405B5CC
:100A240011F40C94168500E04F5F5F4F0E94F4B4FC
:100A340010F00C942285013011F00C94228501C031
:100A440001C0E9CF0E9495A5EE81FF81E053FA4EE3
:100A5400A081FE01E45FFE4FE081EA1711F00C94DF
:100A64003E85103011F40C943B85EE81FF810E9489
:100A740053B50E9444B50895AE81BF812A173B0740
:100A840010F40C944A85003011F00C944A8501C08E
:100A940001C0BECF0E940FB511F40C9454850E947E
:100AA40024B502C00E9431B5003011F40C945F8566
:100AB400103011F40C945F8501C005C00E943AB552
:100AC4000E9458B50895003011F40C946D85E1E04E
:100AD4000E9458B508950E9444B508950E9458B5DF
:100AE40008950E94D7B85A2F40E0E52F0E945DB5C3
:100AF4000E9465B52017310710F00C948F85E42F00
:100B04004F5FAE81BF810E94CCA80E946BB5EC916F
:100B1400D001EC932F5F3F4FEDCFAE81BF810E9498
:100B240070B50E94DEB828960895E0910219F091FC
:100B340003190E9453B508950A930A2FE02FA09138
:100B4400FE18B091FF18F0E0EA0FFB1F0E9453B5A6
:100B5400E02F0E945DB5E0930219F0930319099107
:100B64000895AA9321970E94D6A940E0EF810E949C
:100B74005DB50E9465B52017310710F00C94DB8534
:100B84000E946BB55C91523211F00C94D285A88509
:100B9400B9850E9470B5EE810E94DEB82A96089548
:100BA400E42F4F5FA885B9850E9479B52F5F3F4F29
:100BB400E2CF20930219309303190E94B2A608953C
:100BC400AA9321970E94D6A940E0E8850E945DB5CA
:100BD4000E9465B52017310710F00C940B860E9413
:100BE4006BB55C91EF81E51711F00C940286A98531
:100BF400BA850E9470B5EE810E94DEB82B960895E6
:100C0400E42F4F5FA985BA850E9479B52F5F3F4FC6
:100C1400E1CF2093021930930319E0E00E94DEB87B
:100C24002B9608950A93E0E0E0933619E093371980
:100C34000E9455AA0E948FAA11F00C942486A0E168
:100C44000E94F60EA1E00E9464270E94FCAD0E945F
:100C5400F2150E948A160E9464A9E1E0E093361915
:100C6400E0E0E0933819E0933719E8ECE0933519A4
:100C7400E9E3F9E10E9440AF0E9481B5E9E4F9E1BA
:100C84000E9440AF0E9491AFE1E5F9E10E9440AFBC
:100C94000E9491AFE0E0E0935919E0935A19E09370
:100CA4005B19E0935C19E0935D19099108950E9422
:100CB4001486E1E0E09336190895A0E00E946427C9
:100CC400E3E6E0933619A0E10E94F60E08956D97CD
:100CD4000E94D7B8E0913619E03011F00C94778671
:100CE400E0E00E94DEB8A3960895A0913619A336D9
:100CF40011F00C948786E0E00E94DFAB0E94BB5F9A
:100D0400E0E00E94DEB8A3960895A0913619A130C0
:100D140011F00C94A086A0E10E940D0F8F01093CF4
:100D2400E0E01E0710F40C949C86E0E0E093AD1222
:100D34000E9485B5E0E0E0933719E9C1A091361926
:100D4400A23011F00C94AC86E0EF0E948BB50E94A7
:100D540085B5DDC1A0913619A33011F00C94EF864E
:100D6400EDB7FEB7FA93EA935F930E9495B55F914E
:100D74004E2F403011F00C94D686513010F40C9460
:100D8400CA86E1E00E949DB5EAEC0E94A3B50895ED
:100D9400E1E0E093AD12AFE00E94F60EACE00E94F9
:100DA4003C0F0E9485B50BC0423010F40C94E186D0
:100DB400E2E00E949DB5E9EC0E94A3B50895AFE07E
:100DC4000E9445B010F40C94EE86E3E00E949DB5B9
:100DD400E8EC0E94A3B508959AC1A0913619A430F5
:100DE40011F00C943C870E945B274E2F403011F485
:100DF4000C940C870E948A16E1E00E948BB5ACE04B
:100E04000E943C0FE2E0EA93EA93A2E00E94BB5FF7
:100E14000E9485B5E1E00E94DFAB0E94BB5FACE0BD
:100E24000E94580F8F010630E0E01E0710F40C9466
:100E34002287A091BC12A03011F00C9422870EC01E
:100E44000F31E0E01E0710F40C942F87A091BC1220
:100E5400A13010F40C942F8701C00BC0E0E00E9475
:100E6400DFAB0E94BB5FE0E00E949DB50E94AAB583
:100E740008954DC1A0913619A53011F00C947E87C8
:100E8400EDB7FEB7FA93EA935F930E9495B55F912D
:100E94004E2F403011F00C946787513010F40C94AD
:100EA4005987E4E00E949DB50E94AAB50895AFE079
:100EB4000E94F60EE8A1EA93DE0117960E94F18FD4
:100EC4000E94C08C0E9485B50AC0423010F40C9474
:100ED4007187E5E00E949DB50E94AAB50895AFE030
:100EE4000E9445B010F40C947D87E6E00E949DB505
:100EF4000E94AAB508950BC1A0913619A63011F02D
:100F04000C94AC870E94CA8A4E2F413010F40C9482
:100F14009187E7E00E949DB50E94AAB50895AFE0CD
:100F24000E94F60E0E9485B5E0E00E94DFAB0E94AD
:100F3400BB5FAFE00E940D0F8F01053FE1E01E078C
:100F440010F40C94AB87E8E00E949DB50E94AAB50A
:100F54000895DDC0A0913619A73011F00C94CB8709
:100F6400A9E3B9E10E94D98BA9E4B9E10E94EC8B11
:100F7400A1E5B9E10E94FF8B0E94158CE0935919F9
:100F8400F0935A1960935B1970935C190E9485B5AC
:100F9400BEC0A0913619A83011F00C945D88E0E031
:100FA400E0935D190E94DFAE0E94AFB5E0E9FBE07B
:100FB40060E070E00E94B2B5E9E3F9E10E94BDA6E9
:100FC400A0E1B0E00E94F1192E2F0E94DFAE0E9432
:100FD400AFB5E1EAFBE060E070E00E94B2B5E9E49D
:100FE400F9E10E94BDA6A8E0B0E00E94F1193E2FED
:100FF400203011F40C940388303011F40C940388DD
:1010040001C047C0A0914E19A43411F00C9411886A
:10101400A0914F19A53511F00C94118801C004C09A
:10102400E1E0E0935D1935C0A0914E19A43411F0AC
:101034000C942388A0914F19A63511F00C942388A1
:1010440001C004C0E2E0E0935D1923C0A0914E19F1
:10105400A43511F00C943588A0914F19A03511F0E6
:101064000C94358801C004C0E3E0E0935D1911C01D
:10107400A0914E19A43511F00C944788A0914F19F2
:10108400A33411F00C94478801C003C0E4E0E0935A
:101094005D19A0915D19A13010F40C945688A43602
:1010A40010F00C94568801C003C0ABE00E943C0FC2
:1010B4000E9485B52CC0A0913619A93011F00C946A
:1010C4008088A0915919B0915A1980915B19909117
:1010D4005C190E949F8E2E2F203011F40C94798875
:1010E400A0915D19A13010F40C94798801C003C05B
:1010F400E4E6E0935D190E9485B509C0A091361914
:10110400AA3011F00C948988E3E6E09336190E9422
:10111400AAB508951A930A938D01A0915D19A1307F
:1011240010F40C949A88A43610F00C949A8801C098
:1011340009C0E1E5F9E1FA93EA931A930A930E944C
:10114400E4B006C01A930A93E0E0EA930E9491AFD8
:10115400E0915D190991199108951A930A93ABE0EE
:101164000E94B3B110F40C94BA88E0E0E0935D19E6
:10117400A0915D19A13010F40C94C588A43610F028
:101184000C94C58801C004C0E1E009911991089547
:10119400E0E0099119910895E0E0E0935D19089564
:1011A4000E94D7B81A2F2E813F81488559850C8516
:1011B400043010F00C940689A7E00A9FF001EC5F5C
:1011C400F64EAB85A083A7E00A9FF001EB5FF64ED5
:1011D400AA85A083A7E00A9FF001EA5FF64E508338
:1011E4000A9FF001E95FF64E40830A9FF001E85F31
:1011F400F64E30830A9FF001E75FF64E20830A9F84
:10120400F001E65FF64E10830E94DEB82D96089535
:101214000E94D9B89D010C91043010F00C943F89C0
:10122400A7E00A9FF001EC5FF64EA081AB3B11F002
:101234000C942189F9013196ABEBA08304C0F90128
:101244003196AAEAA08310E0163010F00C943E897F
:10125400E12FF0E03296E20FF31FBF01A7E00A9FEF
:10126400F001EB5FF64EDF01EE27A10FBE1FEC91FC
:10127400DB01EC931F5FE8CF12C0F9013196AAEAB3
:10128400A08310E0163010F00C945189E12FF0E0A7
:101294003296E20FF31FAFEFA0831F5FF3CF0E94DC
:1012A400E0B824960895A4970E94D7B85A2F20E056
:1012B400E0E0E093C514E091B214E03011F00C9436
:1012C4006889E1E00E94DEB8AA96089558A3A8A10F
:1012D400A83210F40C947389E2E00E94DEB8AA9656
:1012E4000895A091B314A13011F00C947F89A8A1A2
:1012F400A03110F40C947F8901C005C0E2E00E9483
:10130400DEB8AA960895DE0190960E940A89E0E06C
:10131400E8A740E0E2E0EA93E8E00E94B7B5EDB761
:10132400FEB7FA93EA930F93EDB7FEB7FA93EA93F5
:101334001F930E94BEB51F910F913E2F0E9464A976
:10134400313011F00C94AC892F5F243610F00C94DA
:10135400AC8901C001C0E3CF4F5F453010F00C945D
:10136400B889303011F40C94B88901C001C0D2CFCF
:10137400E09135192E1710F40C94C589E4E00E940D
:10138400DEB8AA960895303011F40C94CE89E5E0C5
:101394000E94DEB8AA9608950093C514023011F491
:1013A4000C94D989E6E00E94DEB8AA960895E8A1D3
:1013B400E093C6140E94EDB00895BA93AA936C9773
:1013C4000E94C2B54CA148A3E0E0E9A350E0E3E0E9
:1013D400EA93E1E00E94B7B5EDB7FEB7FA93EA935A
:1013E4000F93EDB7FEB7FA93EA931F930E94BEB52D
:1013F4001F910F913E2F0E9464A9313011F00C947B
:10140400098A2F5F243610F00C94098A01C001C0A8
:10141400E3CF5F5F553010F00C94158A303011F42F
:101424000C94158A01C001C0D2CFE09135192E1752
:1014340010F40C94228AE3E00E94DEB8A596089585
:10144400303011F40C942B8AE4E00E94DEB8A596A7
:1014540008950093C714003011F40C94368AE5E023
:101464000E94DEB8A5960895103111F40C943F8AB9
:10147400E6E00E94DEB8A596089520E0203110F041
:101484000C94528AE22FAAA1BBA10E94CCA8E22FFD
:10149400F0E00E94D8A6EC91D001EC932F5FEECF40
:1014A400E0E00E94DEB8A5960895BA93AA93AC979B
:1014B4000E94C2B54CA948A320E0203110F00C943E
:1014C400758AE22FEF5FF0E0DE019096EA0FFB1FD2
:1014D4000F01AAA9BBA9EE27A20FBE1FEC91D00150
:1014E400EC932F5FEACFE0E0E9AB50E0E4E0EA936D
:1014F400E1E10E94B7B5EDB7FEB7FA93EA930F9313
:10150400EDB7FEB7FA93EA931F930E94BEB51F91FD
:101514000F913E2F0E9464A9313011F00C94988AE7
:101524002F5F243610F00C94988A01C001C0E3CFD9
:101534005F5F553010F00C94A48A303011F40C9491
:10154400A48A01C001C0D2CFE09135192E1710F43E
:101554000C94B18AE3E00E94DEB8E5960895303039
:1015640011F40C94BA8AE4E00E94DEB8E59608957A
:101574000093C714003011F40C94C58AE5E00E946E
:10158400DEB8E5960895E0E00E94DEB8E596089599
:101594000A93E091B214E03011F00C94D48AE1E0A3
:1015A400099108950E941B8B0E2F0E94588D0130C3
:1015B40010F40C94E08AE2E0099108950E945A8B99
:1015C4000E2F013010F40C94EA8AE3E00991089597
:1015D4000E949E8B0E2F013010F40C94F48AE4E0E8
:1015E400099108950E94768C0E2F013010F40C940A
:1015F400FE8AE5E0099108950E94BA8B0E2F01300E
:1016040010F40C94088BE7E009910895E0E0099147
:1016140008950E9426A60217130710F00C94178B46
:101624000E94F9A60F5F1F4FF6CF0E94DEB82896DE
:101634000895A29780E1002470E0E0E4FBE060E01C
:101644000E94E5B80E94DAB8E4E2F3E1FA93EA937F
:10165400A0E0B1E00E940B8B00E0003110F00C948C
:10166400558B0E946CAE2C912A93DE0154960E94F5
:10167400808D1E2F103011F40C94458BE1E00E94F4
:10168400E1B8A59608950E94C9B5E02FF0E00E9444
:101694005AB9EC5DFC4EFA93EA93A0E1B0E00E94E3
:1016A400061B0F5FDACFE0E00E94E1B8A59608952B
:1016B40062971A930A930E94CEB510F40C94678B28
:1016C400E1E019810881649608951E85EE85ED5F39
:1016D400EE87E0E0EA930E94CDB0A1E00E94ED8D98
:1016E4000E2F043011F00C947C8BE0E019810881FA
:1016F40064960895013010F40C94858BE2E019810E
:101704000881649608950E94CEB510F40C948F8BD2
:10171400E3E01981088164960895EE85E11711F0DC
:101724000C94998BE4E01981088164960895E0E0B3
:10173400198108816496089561970A93EAEAFBE0A7
:1017440060E070E00E945AB1E4E3F3E1FA93EA93B3
:101754000E94CDB0A0E10E94D7B511F40C94B68BD1
:10176400E0E0088162960895E1E0088162960895B8
:101774000E94D7B810914813009149131A93A02FCF
:101784000E94BB209F010E94F2B0AF014217530791
:1017940011F00C94D08B0E94F1AF0895E1E00E9407
:1017A400DEB8269608950E94DEB8269608950E9413
:1017B400BAA400E0003110F00C94E88B0E94DDB56F
:1017C400A4E7B3E10E9401B30F5FF4CF0E94E1B834
:1017D400239608950E94BAA400E0083010F00C94F7
:1017E400FB8B0E94DDB5A4E6B3E10E9401B30F5F59
:1017F400F4CF0E94E1B8239608950E94BAA400E0B1
:10180400083010F00C94118C0E94DDB5A4E6B3E10D
:10181400E02FE85FF0E00E9426A70F5FF1CF0E945F
:10182400E1B8239608952A970A9300E0063010F051
:101834000C94278CE02FF0E00E9457A70F01A4E836
:10184400B3E10E9401B30F5FF1CFEF81EA93E98521
:10185400EA93EB85EA93AD850E94CE200E94E1AF26
:1018640008812B9608950E946FBAEF97299780E418
:10187400002470E0E0E5FBE060E00E94E5B80E942F
:10188400D7B8FE01EE5AFF4F3081FE01ED5AFF4FEB
:101894004191508100E0FE01E25BFF4F0190119005
:1018A40061917081F0010E94E3B5E32F3150E03083
:1018B40011F40C94698C0E9454AF2081E22F0E9491
:1018C400EBB5E22FE295EF700E94EBB5EECFFE018F
:1018D400E65BFF4F0190119061917081F0010E94CD
:1018E400DEB8EF9666960895EF972F970E9412B68A
:1018F4000E941CB6E3E5F3E463E574E50E9402B9D3
:101904000E940EA500E0003310F00C94968CE02F9A
:10191400F0E0DE011D96EA0FFB1F0F01A4EAB3E11C
:101924000E9401B30F5FEFCFFE013D96FA93EA9355
:10193400ECE2EA93AC81BD818E819F810E94358C5B
:101944000E941CA5ECADEA93ECADEA93ECADEA93EE
:10195400ACAD0E94CE20E987FA876B877C870E9412
:101964008EAB11F00C94BB8CE0E00881EF9660968E
:101974000895E1E00881EF96609608956E971A93B2
:101984000E9412B60E9423B6EE8B0E9429B6EF8BFA
:101994000E9429B6E88F0E9429B6E98FEE89EA8F62
:1019A400AA8DEBE40E942FB6E0E50E9438B6E2E48B
:1019B4000E9442B6E7E5EA27D001EC93EAE5EE8F10
:1019C400E5EAEF8F16E000E0063010F00C94F48C9A
:1019D4001150E12FF0E0E05EF64E0F010E944CB68C
:1019E4000F5FF2CFE0E00E9452B6E5E30E942FB60B
:1019F400E2E40E9438B6E4E50E9442B6E1E4EA2754
:101A0400D001EC93E5EAEE8FEAE5EF8F16E000E013
:101A1400063010F00C94188DA7E2B9E11150E12FB3
:101A24000E94CCA80E944CB60F5FF2CFE1E00E9466
:101A340052B6E4E60E942FB6E7E6EA27D001EC931B
:101A4400E88DEC8FE98DED8FE5E1EE8FE8E0EF8F27
:101A540016E000E0063010F00C943A8DAEE2B9E1E5
:101A64001150E12F0E94CCA80E944CB60F5FF2CF18
:101A7400E2E00E9466B6E8E0EA93DE0117960E946F
:101A8400808DED85EA8FEC85EB8FEB85EC8FEA8515
:101A9400ED8FE9E7EE8FE3E2EF8FE3E00E9466B6B5
:101AA400EF8DEF8F19810881A0960895E3E00E94DD
:101AB40076B6E0E2F9E10E947BB60E9482B6E4E5E4
:101AC400F3E10E948DB6E7E00E9476B6E7E2F9E121
:101AD4000E947BB60E9482B6E4E9F3E10E948DB6CF
:101AE400EBE00E9476B6EEE2F9E10E947BB60E943A
:101AF40082B6E4EDF3E10E948DB608950E94D7B852
:101B0400AD013E81303011F00C948A8D20E005C087
:101B1400E32FEC7F2E2F26952695A091C514A23095
:101B240011F00C949C8DA091C6142A1711F00C94FA
:101B34009C8D0AC00E9493B610F40C94A68DE4E028
:101B44000E94DEB8279608953A93DA010E94DF894D
:101B54000E2F053011F00C94CC8D0E9493B610F426
:101B64000C94B98DE4E00E94DEB8279608953A9368
:101B7400DA010E94DF890E2F013010F40C94C78D16
:101B8400E5E00E94DEB827960895E0E00E94DEB802
:101B940027960895013010F40C94D58DE5E00E9449
:101BA400DEB827960895E0E00E94DEB827960895EF
:101BB4000A930A2F003011F40C94E78DE02FE370A0
:101BC400E33011F40C94E78D03C0E0E0099108952B
:101BD400E1E0099108950E94D7B84A2F5885352F1E
:101BE400A32F0E94DA8DE03011F00C94FE8D40306A
:101BF40011F00C94FE8D01C005C0E6E00E94DEB831
